:020000040800F2
:1000000000800020E16B00085D780008BD6B0008EF
:100010005F7800086178000863780008000000003D
:1000200000000000000000000000000031C60008D1
:100030006578000800000000C1C6000805C7000878
:1000400067780008697800086B7800086D78000808
:100050006F78000871780008F1770008F7770008DA
:10006000FD77000803780008097800087378000815
:100070007578000877780008797800087B780008A0
:100080007D7800087F780008817800088378000870
:100090008578000887780008897800080F780008BC
:1000A0008B7800088D7800088F7800089178000818
:1000B00093780008957800089778000899780008E8
:1000C0009B7800089D7800089F780008A1780008B8
:1000D000A37800083D7F000889830008A578000800
:1000E00033780008DD780008A7780008A9780008B0
:1000F000AB780008000000000000000000000000D5
:1001000000000000000000005FF808F110B5054C89
:10011000237833B9044B13B10448AFF300800123B3
:10012000237010BDE802002000000000D8FC010888
:1001300008B5034B1BB103490348AFF3008008BD6A
:1001400000000000EC020020D8FC0108704700000D
:10015000816801480AF070B91CAD010838B5044641
:1001600081680D480AF068F920690C4D0368002188
:100170001B68984701222846032107F0B5F920693A
:10018000002103685B6898472846BDE83840012293
:10019000022107F0A9B900BF02AD0108000002402A
:1001A0000B4B13B51A68B2F5007F04D21A68511CC4
:1001B0001960084B9854084B1C680DF029FE002369
:1001C00002460093072120460EF0ECFC02B010BD61
:1001D00004050020040300200805002010B5044693
:1001E000382115F0CBFD204610BD000070B5154C30
:1001F0002368092B1FD92268134D023A2946134858
:1002000015F0E7FC06462068023828440AF00DFA8B
:100210008642014610D10E4E30680DF0DBF922689F
:100220000023294630680DF021FA10B909480AF078
:1002300003F90023236070BD324607480AF0FCF83A
:10024000F7E700BF0405002004030020040000209D
:100250000C050020ACAC0108DAAC010870B504460E
:100260002048214E60602148C4E90312A060204864
:1002700086B020606361194604F1180004F124057A
:1002800006F06AFA0FCE0FC5336801222B600021F9
:100290004FF400700DF05CF9164B186018B94A2144
:1002A000154806F003FC154B0A210093002314485F
:1002B0001A460EF055FC134B41F221011860012340
:1002C000CDE900334FF6FF7303A81A4615F02EFC54
:1002D0000D4A03AB03CB106020461B88516013818D
:1002E00006B070BD55AD010898AC01085FAD0108BE
:1002F000D4AD01080C05002065AD0108ED01000832
:10030000BFAD010808050020040000200148006876
:100310000DF03ABA0C05002010B50446C068074934
:1003200003685B699847E06804F1240103681B686F
:1003300098470022024B1A6010BD00BFA1010008BF
:1003400004050020C06810B50368084C5B68984736
:1003500001220221204607F0C7F80122032120468E
:1003600007F0C2F80022024B1A6010BD00000240E4
:100370000405002081F001021830082106F0AEBA11
:1003800081F001021830022106F0A8BA81F00102C2
:100390001830042106F0A2BA81F0010218300121C0
:1003A00006F09CBA10B5044681680E480AF044F87D
:1003B00004F1180006F080FA20460021FFF7E6FF5E
:1003C00020460021FFF7DCFF20460021FFF7D2FF87
:1003D00020460121FFF7E0FF2046BDE81040002144
:1003E000FFF7DABFF8AC010810B5044681681A4877
:1003F0000AF022F8A16819480AF01EF820460121E7
:10040000FFF7CAFF01212046FFF7BAFF4FF49670AD
:100410000DF050FE20460021FFF7B2FF01212046DB
:10042000FFF7B4FF4FF496700DF044FE2046002114
:10043000FFF7ACFF01212046FFF79CFF4FF49670B9
:100440000DF038FE20460021FFF794FF2046BDE85E
:1004500010400021FFF7A0BF2BAD01083BAD010804
:1004600008B5034809F0E8FFBDE8084007F0BCBF45
:10047000DEAE010807F0B8BF10B50446C06910B180
:10048000012115F07BFC206910B1012115F076FCEB
:10049000204610BDF8B50025C0E901120570C0E97D
:1004A0000335C0E90555C0E907554562069904467C
:1004B000164600F11C0713F03BFC38B931460748DB
:1004C00009F0BAFF2021064806F0F0FA069A3946EC
:1004D000204613F0F5FB2046F8BD00BFFCAE010836
:1004E00027AF010830B593B014F096FC054603F031
:1004F00003FA294603F0E2FC1E4B08AC1E4A0093A7
:1005000003211E4B2046FFF7C5FF2146284614F065
:100510002FFD2046FFF7B0FF194B1A4A0093032125
:10052000194B2046FFF7B6FF2146284614F020FD60
:100530002046FFF7A1FF2846144B154A154914F031
:10054000DBFB00220521144B0B9208930792134BFF
:10055000134A0993CDE90512124B0A9305AB93E8B0
:1005600007008DE8070094E80F0014F0EFFE13B0C9
:1005700030BD00BF16AE010824AE0108ECAD010885
:100580008AAE010881AE01082DAE0108750400088D
:10059000B4AE0108D8AE010861710008E970000826
:1005A000000008086104000860B1037813F07002CD
:1005B00004D0402A05D003F00F0070474368586804
:1005C000704701207047000010B9034809F034BF9C
:1005D00003C809F097BF00BF43B4010810B926480B
:1005E00009F02ABF0178406801F07002402A01F04A
:1005F0000F030ED004D8A2B10268204809F01CBF36
:10060000502A20D0602AF7D1012B0CD101781C4848
:1006100005E01C491C4B002808BF19461B4809F07F
:100620000BBFFFF7D1BF022B02D101881848F6E7B4
:10063000042B02D101881748F1E7082B01680CBF91
:1006400015481648EBE7012B03D190F90010144828
:10065000E5E7022B03D1B0F900101248DFE7042BC5
:1006600003D1B0F900101048D9E7082B01680CBF7E
:100670000E480F48D3E700BF43B4010827B4010870
:10068000ACB30108A1B30108A6B3010893B00108F7
:10069000B8B30108C5B30108D2B30108E0B301083B
:1006A000ECB30108F7B3010803B401080FB4010863
:1006B0001CB4010870B50020002105F0B3FD04460C
:1006C0000F4D104EC4B16179802911D12279216872
:1006D000306813F02BFF204605F002FF204608216A
:1006E00015F04CFB0020002105F09CFD0446E9E7D5
:1006F000284609F0A1FEEEE7034B187870BD00BF55
:100700001CB30108B40800206009002008B503F0FC
:10071000F3F8BDE8084003F025B910B1042115F045
:100720002DBB704710B1012115F028BB704710B5E3
:1007300004460068FFF7F1FF204610BD1FB5612396
:10074000CDE9013101A9039204F04CFA05B05DF83E
:1007500004FB07B58DF8041001A98DF805208DF86C
:10076000063004F00BFB03B05DF804FB10B50C4C35
:1007700003F0C2F82368DB070FD400F1580300F13F
:10078000440200F148010748FFF768FD0123064ACB
:1007900006490448236016F029F9024810BD00BF3D
:1007A0001005002044070020000000204D01000833
:1007B0002DE9F047FFF7DAFF04460121FFF7ECFDD2
:1007C0002046FFF7A9FD0DF01DFB4EF65F273C4EBE
:1007D0004FF4007233683B49C01AB8424FF47A7341
:1007E000394D204642D8FFF791FDDFF8ECA0DFF845
:1007F000D4902860D5F80080B8F1000F1DD10DF01D
:1008000001FB3368C01AB84217D8504609F014FEED
:1008100001212046FFF7B4FDC8200DF04BFC4146F6
:100820002046FFF7ADFD4FF47A734FF4007249464E
:100830002046FFF76BFD2860DCE72046FFF782FDCE
:100840002B68002B39D001212046FFF79FFD1F4860
:1008500009F0F2FD41F288300DF02CFC0021204619
:10086000FFF794FD1A4B1878BDE8F087FFF74EFDAF
:100870000526DFF86490DFF84C8028602F68002F91
:10088000E1D1013E16F0FF0617D0484609F0D4FD2D
:1008900001212046FFF774FDC8200DF00BFC3946FE
:1008A0002046FFF76DFD4FF47A734FF40072414616
:1008B0002046FFF72BFD2860E0E7064BD3E700BF9B
:1008C0003C070020280500203807002091B30108CC
:1008D000640900206209002069B301082DE9F04194
:1008E0002B4809F0A9FDFFF741FF04460121FFF75E
:1008F00053FD2046FFF710FD41F288334FF400729C
:1009000024492046FFF702FD234D28602046FFF7CB
:1009100019FD2E68B6B9214809F08EFD0121204647
:10092000FFF72EFD4FF47A700DF0C4FB31462046E0
:10093000FFF726FD31462046FFF72EFD184B1878AD
:10094000BDE8F081174809F077FD0026114FDFF868
:1009500060802B68B34206D917F8011B404609F0A6
:100960006BFD0136F5E7104809F066FD01212046D0
:10097000FFF70CFD4FF47A700DF09CFB0021204630
:10098000FFF704FD00212046FFF706FD074BD6E7E1
:1009900042B30108280500203807002069B3010888
:1009A0006209002056B30108B3F001086409002071
:1009B000E9AF0108F8B5334809F03EFDFFF7D6FE70
:1009C00001210446FFF7E8FC2F4B1A786AB1002595
:1009D000012120461D70FFF7CDFC41F288300DF05B
:1009E00069FB29462046FFF7C5FC2046FFF794FC2B
:1009F00041F288334FF4007224492046FFF786FC09
:100A0000234D28602046FFF79DFC2E68AEB9214893
:100A100009F012FD01212046FFF7B2FC4FF4967059
:100A20000DF048FB31462046FFF7AAFC3146204630
:100A3000FFF7B2FC184B1878F8BD01212046FFF7EC
:100A4000A5FC4FF496700DF035FB20460021FFF712
:100A50009DFC20460021FFF79FFC104809F0ECFCAC
:100A600000240A4E0E4F2B68A34206D916F8011B2C
:100A7000384609F0E1FC0134F5E70A4809F0DCFCEE
:100A8000094BD8E742B301081800002028050020D0
:100A90003807002069B301086209002056B3010835
:100AA000E9AF0108B3F00108640900202DE9F04F17
:100AB00087B00BF0D1FF04460BF0D4FF214602466D
:100AC000C34809F0B9FC02F017FF04460BF0C4FF5D
:100AD00005460BF0C7FF29460246BD4809F0ACFCAD
:100AE000BC4809F0A9FCFFF741FE0146204615F07D
:100AF0000DFF204615F0C6FEB74809F09DFC0BF02F
:100B0000ABFF05460BF0AEFF29460246B04809F0A0
:100B100093FCFFF7E7FC0BF09FFF05460BF0A2FFED
:100B200029460246AA4809F087FCAC4809F084FC33
:100B3000FA200DF0BFFA14F089F913F05FFD20469A
:100B400015F0B6FEA64809F077FC0BF085FF0446C9
:100B50000BF088FF214602469D4809F06DFCA14834
:100B600009F06AFC14F072F99F4D06462B689F4C01
:100B700013F0010F04D104F01BF8012320602B6057
:100B8000256802F0B9FE00F16001284603F0D0FEAE
:100B90002068974903F0CEFE96493046256813F049
:100BA000E4FF9549024603A803F0ACFE03A92846DA
:100BB00003F002FF25688DF80600062200238F4906
:100BC00003A803F06DFE03A9284603F0F5FE25688F
:100BD00000230F228A4903A803F062FE03A92846D6
:100BE00003F0EAFE874A8DF8070087492068FFF77F
:100BF000A5FD864A074686492068FFF79FFD834A80
:100C000084492068FFF79AFD834A8DF800008349E4
:100C10002068FFF793FD824A824682492068FFF7E9
:100C20008DFD7F4A834680492068FFF787FD7C4A17
:100C30007E492068FFF782FD70254FF000067C4B4F
:100C40008DF8010003A92068039504938DF81460C2
:100C500003F0C8FF774B03A98DF8020020680493C6
:100C600003958DF8146003F0BDFF8DF80300206834
:100C700005F0FEF870498146206805F0E3F86F4AF8
:100C80008DF804006E492068FFF758FD8046206803
:100C90006C4A80F828706C49FFF750FD6B4A064695
:100CA0006B492068FFF74AFD6A4D8DF805009DF8F5
:100CB00000302A7839462068674FFFF74AFD9DF8D3
:100CC00001302A789DF800102068FFF742FD4B465E
:100CD0003A789DF800102068FFF73BFD4B462A78D4
:100CE0009DF801102068FFF734FD4B463A789DF8D7
:100CF00001102068FFF72DFD43462A7849462068F9
:100D0000FFF727FD53462A7841462068FFF721FD6B
:100D10009DF803303A7841462068FFF71AFD4346B4
:100D20009DF807209DF803102068FFF712FD5B4631
:100D30002A7851462068FFF70CFD5B463A78514609
:100D40002068FFF706FD33462A7859462068FFF7EA
:100D500000FD33463A7859462068FFF7FAFC3F4ACF
:100D60009DF80430314620681278FFF7F2FC9DF8B8
:100D700005302A789DF804102068FFF7EAFC384A0D
:100D800033469DF8051020681278FFF7E2FC9DF8C5
:100D900002302A7831462068FFF7DBFC53469DF885
:100DA00006209DF802102068FFF7D3FC206804F0AD
:100DB00005FA2C4809F040FB24680BF04DFE05466F
:100DC0000BF050FE29460246014809F035FB4BE086
:100DD00049B4010868B401087CB401088DB4010865
:100DE000A4B40108B6B40108180500209C0800202E
:100DF0000D07000824AE0108D3B40108DAC70108C2
:100E0000DCB401085D16000832C90108DD080008DD
:100E1000ECB40108F8B40108B50900080BB50108E5
:100E20009510000810B5010819B5010829B5010889
:100E3000C3C7010840B501081CC80108B107000874
:100E40004EB501088D0E00085AB50108B506000818
:100E500063B50108640900206209002063090020CD
:100E60006009002072B50108074809F0E5FA01227F
:100E70004FF4C871204604F00FF900200CF08EFEEC
:100E800007B0BDE8F08F00BF8CB501082DE9F04F29
:100E900089B0FFF76BFC012106466D4DFFF77CFA28
:100EA000FFF764FC0121FFF765FA4FF496700DF02F
:100EB00001F92B685C68FCB1664809F0BDFA2C6842
:100EC00005F0A8F96449024604AB204613F0E6F8A1
:100ED000614902469DF8100005F070F9FFF746FCE5
:100EE0000021FFF747FA00213046FFF755FA5B4B28
:100EF000187809B0BDE8F08F06F006FE584B6D4635
:100F0000D3E900ABBBF1004F08BFBAF1000F0BD023
:100F1000B0EB0A0861EB0B094FF0000BDFF870A192
:100F2000C2457BEB090255DAC3E9000104AC4D4828
:100F300009F082FA14224C49204614F098FE05F07C
:100F40009FFF804615F002F900210746204614F065
:100F5000B9FE0421204614F0B5FE0121204614F00C
:100F6000B1FE0021204614F0ADFE4049404616F087
:100F700067FC16F051FE01B2204614F0B5FE39466A
:100F8000204614F0B1FE94E80F0085E80F002846D3
:100F900014F0A5FE40B3364809F04EFA13F056FFA0
:100FA000344913F0BFFD00238DF81030C0B98DF81F
:100FB0001100284614F091FE0446284614F08FFED6
:100FC000049BC2B22146012005F00CF9284614F01A
:100FD00088FE83E710222146284617F04DF9D6E710
:100FE00001238DF81130E4E7234814F078FE04461D
:100FF000A0B1214814F073FE0146204809F01CFA04
:101000001D4814F06AFE04461B4814F068FE214691
:10101000C2B2032005F0D2F81748D8E7184F3D7840
:101020003DB1184809F008FA3C7022460A492046AA
:1010300052E7154809F000FAFFF798FB2946FFF739
:1010400099F929463046FFF7A7F9104B50E700BF42
:10105000B40800202FB20108BE0700206309002059
:101060001000002055B20108A008002000007A44BA
:1010700074B2010895B2010828070020A2B2010845
:101080002E0A0020CCB2010801B301086409002037
:10109000085101002DE9F04F89B03222002103AE42
:1010A000A848A94C17F0E8F83222A649304614F0B7
:1010B000DEFD96E80F0007C42370FFF757FBA34B34
:1010C00007461B68102B1DD80021A4F10C0014F05A
:1010D000F9FD01213846FFF75FF901213846FFF796
:1010E0004FF94FF496700CF0E5FF00213846FFF7FA
:1010F00047F900213846FFF74FF9954B187809B0AA
:10110000BDE8F08F0022CDE90522924A103B039200
:101110000493304601F062FE98BB0121304601F095
:1011200065FEDDE904329A42F3D38B4809F084F975
:10113000854814F0D2FD0446834814F0D0FD0146E2
:10114000204609F0DFF9804814F0C9FD014610B9C6
:101150007D4814F0B7FD01213846FFF71DF9012144
:101160003846FFF713F94FF496700CF0A3FF0021F7
:101170003846FFF70BF900213846FFF70DF9774B9A
:10118000BCE7304601F05CFB0546304601F01BFE33
:1011900098B1734809F050F9DDE9043206997148B5
:1011A00009F04AF9704809F047F9DDE9041303989A
:1011B000C91A184409F0A6F9B7E76C4809F03CF9D8
:1011C0006B686B48197809F037F9AB68694819788A
:1011D00009F032F92B696848198809F02DF9674838
:1011E00009F02AF92868FFF7EFF9EB6864481B68F3
:1011F000196809F021F9EB681B681A6840F201735D
:101200009A4243D15F4809F017F9EB68DFF8908103
:101210005B68DFF890911C69DFF88CA1002C35D059
:1012200023682BB1404609F007F92068FFF7CCF995
:1012300063682BB15A6819781278484609F0FCF8AF
:10124000A36813B1504609F0F7F8E36823B11A78A0
:101250004D48114609F0F0F8236923B193F90010C5
:101260004A4809F0E9F8636933B14948197809F047
:10127000E3F86069FFF7B2F9A3692BB1454809F0BB
:10128000DBF8A069FFF7A0F9E469C7E7EB681A6823
:10129000116840F2017291424FD15B68DFF80CB1E6
:1012A00000933D4BDFF8A0805A68D3F800A001926C
:1012B000019A5346524540D0186801F0E5FB81463B
:1012C000584609F0B9F84846FFF77EF9D9E9001207
:1012D000404614F0D9FC009B0AF1040A1C69002C5A
:1012E0007ED022688AB1D2F804C0D9F804309C4577
:1012F0000BD100239C455BDD1068D9F80010C05C61
:10130000C95C884201D10133F4E7E469E7E74B683F
:10131000D3E90012404614F0B7FC216901B1097805
:10132000404614F0CFFC23691C4893F9001009F0E3
:1013300083F8484601F05BFBBAE7284601F068FAFB
:10134000EFE600BF8C0700202807002038070020A8
:101350006209002030050020EBB10108640900207B
:1013600097B00108BFB00108DCB00108E9B001087E
:10137000F7B0010808B101081CB1010829B1010842
:101380003CB101084EB1010894B10108A6B10108B1
:10139000B5B10108C7B101081C050020A9B10108B9
:1013A00063B101086DB1010886B10108D6B1010829
:1013B0000F4809F041F86069FFF710F96069FFF71D
:1013C000F3F8C1B2404614F07DFC61690B7813F06C
:1013D000700F9CD00846FFF7E7F80246496899E786
:1013E000044809F029F82146404614F06BFCA0E7B8
:1013F000FBB1010814B20108F7B502F07DFA0368E9
:1014000004469B6898471F4809F016F81E4809F0E3
:1014100013F80BF057FA05460BF054FA012629464B
:10142000002500F57052194809F006F805F068FA31
:101430002B464FF496721649CDE9006515480CF01D
:10144000BFFA0BF009FB07460BF00CFB39460246CE
:10145000114808F0F1FF23683146DB6820469847C1
:101460004FF4FA7005F01EFE23682946DB6820461B
:1014700098470A4808F0E0FF094808F0DDFF0CF043
:1014800079FCFEE751B80108CEB50108D8B50108CE
:10149000F1B50108AD0A000849B40108FAB5010820
:1014A0000DB60108B1F5705F2DE9F843054602D984
:1014B000184814F027FC066883689B1BB1EBA30F48
:1014C0001CD9D0F804904FEA8108A9EB060759B15E
:1014D000404609F04DF804462346B14506D056F87B
:1014E000042B43F8042BF8E70C46F5E72868FFF7D0
:1014F00014F927442C6044446F60AC602C683CB9FC
:101500002046C5E90144FFF708F92046BDE8F88305
:101510000120FBE7A4B501082DE9F84FD0E90079D7
:10152000A9EB0704A410B4F5705F064688469346FD
:1015300002D1204814F0E6FB002C14BF23460123FF
:10154000E418A1EB070515D2B4F5705F12D8A4B169
:10155000A00009F00DF88246DBF80030AAF1040281
:101560004AF805303B46984509D053F8041B42F829
:10157000041FF8E74FF47054EAE7A246ECE725F0C1
:1015800003050435554441462B46494504D051F8DE
:10159000042B43F8042BF8E7A1EB08010D4438466F
:1015A0000AEB8404FFF7B9F8C6E900A5B460BDE80A
:1015B000F88F00BFB4B5010810B50A46D0E9011490
:1015C000A14204D0126841F8042B416010BDFFF71E
:1015D000A3FFFBE72DE9F0410368551A174682681F
:1015E0000446D21A95420E4615D9284608F0C0FF87
:1015F00080460346B74204D016F8012B03F8012BAE
:10160000F8E720684544FFF78DF8C4E90155C4F8B0
:101610000080BDE8F0814268D21A95420BD825B10E
:1016200018462A4616F00EFE03461D446368AB4278
:10163000EFD06560EDE7164412B1184616F002FED1
:10164000636832461946974204D012F8010B01F83C
:10165000010BF8E7BE1B1E446660DAE72DE9F04196
:101660007A48AAB008F0E8FE13F0F0FB784D044683
:101670002B68DB0706D401468022764812F0B4FCC2
:1016800001232B60744B734A204674491A6013F08F
:101690006CFA00240546724E724FDFF8DC81002D93
:1016A00044D00EAB03930BAB02930AAB019309AB8F
:1016B000009307AA08AB3146284617F0D5FC062848
:1016C00008D0694808F0B8FE40F2B621674805F036
:1016D000EDF92FE00E9B11A804930B9BC4F164015C
:1016E00003930A9B20440293099B3A460193089B6B
:1016F0000093079B17F064FC0444622C04DD214630
:101700005B4808F099FEDFE728462C2117F01BFD07
:10171000054658B111ABC4F16401181942460134B1
:1017200017F04EFC632CEAD00135B8E711A95148F7
:1017300008F082FE11A817F025FD0023002878D0BC
:10174000441C2046CDE90B330D9308F011FF0546EC
:101750000B98FEF7E7FF2B19CDE90B550D93002DE4
:101760003BD128460D95FEF7DDFF3A213F4805F0B5
:101770009DF9002309AA40490B98CDE90E33109337
:1017800017F097FD0546394F3B4E7DB3284617F0BD
:10179000F9FCD8B1441C204608F0EAFE0A9018B9BA
:1017A0004621384605F082F9294622460A9816F065
:1017B0003BFDDDE90E31C91A891001310EA8FFF792
:1017C00071FE18B10AA90EA8FFF7F6FE09AA314664
:1017D000002017F06EFD0546D7E711AA4FF0000371
:1017E000224411A90BA8FFF7F5FEC2E728460E9E7A
:1017F0000F9C0E95CDE90F55FEF78FFF0B98FEF766
:1018000091FF0CF0FFFA1D4B354618601C4808F09C
:1018100013FEDFF878801B4FA5420DD055F8041B4E
:1018200040460E9108F008FE0EA93846FFF7C4FEA8
:10183000F2E704460646E4E7134B30461C78FEF711
:101840006CFF20462AB0BDE8F08100BF60AF010800
:10185000140500207C070020B408002081AE010898
:1018600073AF0108D5AF010885AF010844B0010886
:10187000EEAF01082AB0010828B001083C0700209B
:1018800083B001081C0500206409002091B0010804
:10189000FF22054B05481A700023054AC0E90033B2
:1018A0008360044915F0A2B8400700201C05002001
:1018B000000000202F07000808B5102008F058FE8F
:1018C0001022002116F0D8FC08BD10B5044680B1E6
:1018D000006801F08CF8606801F089F8A06801F0F8
:1018E00086F8E06801F064FD2046BDE8104008F08D
:1018F00029BE10BD38B50446FFF7DEFF0546204679
:1019000001F066FA702806D00123E3602846FFF74D
:10191000DCFF002528E0204601F035FA0428F3D149
:10192000204601F071F82860204601F04CFA0028AA
:10193000ECD1204601F068F86860204601F043FAD7
:101940000028E3D1204601F05FF8A860204601F0AE
:101950003AFA0028DAD1204601F0D1FDE8602046AD
:1019600001F031FA0028D1D1284638BD10B504461F
:10197000012008F0FDFD047010BD70B5044601F0B3
:1019800039FA30B9204601F023FA402803D0012368
:10199000E360002070BD204601F0F5F901280546FE
:1019A000F5D1204601F01AFA06462946204636B1FE
:1019B00001F01CFAFF20BDE87040FFF7D7BF01F02F
:1019C00015FA3046F7E708B108F0BCBD704708B516
:1019D000042008F0CDFD0023036008BD10B50446C7
:1019E00038B1006801F003F82046BDE8104008F067
:1019F000A9BD10BD38B50446FFF7E9FF05462046EE
:101A000001F0E6F9702806D00123E3602846FFF7CD
:101A1000E5FF00250DE0204601F0B5F90128F3D1DE
:101A2000204600F0F1FF2860204601F0CCF90028A4
:101A3000ECD1284638BD08B5042008F099FD0023F4
:101A4000036008BD10B5044638B1006800F0CFFF50
:101A50002046BDE8104008F075BD10BD38B50446FD
:101A6000FFF7E9FF0546204601F0B2F9702806D0DD
:101A70000123E3602846FFF7E5FF00250DE020463F
:101A800001F081F90128F3D1204600F0BDFF286064
:101A9000204601F098F90028ECD1284638BD10B551
:101AA000044698B1006800F0A2FF606800F09FFF54
:101AB000206900F09CFFA06800F099FFE06800F04A
:101AC00096FF2046BDE8104008F03CBD10BD38B57B
:101AD0000446142008F04CFD14220021054616F09F
:101AE000CBFB204601F074F9702806D00123E36097
:101AF0002846FFF7D4FF002531E0204601F043F9E6
:101B00000528F3D1204600F07FFF2860204601F031
:101B10005AF90028ECD1204600F076FF6860204694
:101B200001F051F90028E3D1204600F06DFFA860D4
:101B3000204601F048F90028DAD1204600F064FF81
:101B4000E860204601F03FF90028D1D1204600F09E
:101B50005BFF2861204601F036F90028C8D12846ED
:101B600038BD08B51C2008F003FD1C22002116F02A
:101B700083FB08BD10B50446C8B1006800F037FF0C
:101B8000606800F034FFA06800F031FFE06801F009
:101B900088F9206900F0E6FC606900F028FFA06980
:101BA00001F07FF92046BDE8104008F0CBBC10BD25
:101BB00038B50446FFF7D5FF0546204601F008F981
:101BC000702806D00123E3602846FFF7D3FF0025E5
:101BD00043E0204601F0D7F80728F3D1204600F073
:101BE00013FF2860204601F0EEF80028ECD12046D3
:101BF00000F00AFF6860204601F0E5F80028E3D114
:101C0000204600F001FFA860204601F0DCF8002823
:101C1000DAD1204601F054F9E860204601F0D3F80B
:101C20000028D1D1204600F0A7FC2861204601F011
:101C3000CAF80028C8D1204600F0E6FE68612046B8
:101C400001F0C1F80028BFD1204601F039F9A861A0
:101C5000204601F0B8F80028B6D1284638BD08B5AE
:101C6000142008F085FC1422002116F005FB08BDA5
:101C700010B5044698B1006800F0B9FE606800F045
:101C8000B6FEA06800F0B3FEE06801F064F92069D8
:101C900000F0ADFE2046BDE8104008F053BC10BD7A
:101CA00038B50446FFF7DBFF0546204601F090F803
:101CB000702806D00123E3602846FFF7D9FF0025EE
:101CC00031E0204601F05FF80528F3D1204600F00E
:101CD0009BFE2860204601F076F80028ECD12046D3
:101CE00000F092FE6860204601F06DF80028E3D114
:101CF000204600F089FEA860204601F064F8002824
:101D0000DAD1204601F042F9E860204601F05BF8A4
:101D10000028D1D1204600F077FE2861204601F04E
:101D200052F80028C8D1284638BD08B50C2008F064
:101D30001FFC002202604260826008BD10B50446AC
:101D400068B1006800F053FE606801F004F9A06813
:101D500001F02EFB2046BDE8104008F0F3BB10BD9B
:101D600038B50446FFF7E1FF0546204601F030F89C
:101D7000702806D00123E3602846FFF7DFFF002527
:101D80001FE0204600F0FFFF0328F3D1204600F0BB
:101D90003BFE2860204601F016F80028ECD12046D2
:101DA00001F0F4F86860204601F00DF80028E3D156
:101DB000204601F0A4FBA860204601F004F80028AA
:101DC000DAD1284638BD08B5242008F0D1FB2422FA
:101DD000002116F051FA08BD10B50446F8B10068AC
:101DE00000F005FE606801F05CF8A06800F0E4FD1A
:101DF000E06801F0B0F8206901F053F8606900F084
:101E0000DBFDA06900F0DCFAE06900F0F0FD206A7B
:101E100000F0EDFD2046BDE8104008F093BB10BD7A
:101E200038B50446FFF7CFFF0546204600F0D0FF47
:101E3000702807D001232846E360FFF7CDFF002577
:101E4000284638BD204600F09EFF0928F2D12046E2
:101E500000F0DAFD2860204600F0B5FF0028E9D147
:101E6000204601F02DF86860204600F0ACFF002805
:101E7000E0D104226021204600F055FDA8602046F4
:101E800000F0A1FF0028D5D1204601F07FF8E860DE
:101E9000204600F098FF0028CCD1204601F010F831
:101EA0002861204600F08FFF0028C3D1082260215E
:101EB000204600F038FD6861204600F084FF0028CD
:101EC000B8D10F4A0F49204600F0A3FAA861204676
:101ED00000F079FF0028ADD1204600F095FDE861C3
:101EE000204600F070FF0028A4D1204600F08CFDB1
:101EF0002862204600F067FF0028A1D09AE700BFC3
:101F000029330008E933000808B5242008F030FB25
:101F10002422002116F0B0F908BD70B5044638B38C
:101F2000006800F064FD606800F061FDA06800F0EA
:101F30005EFDE068FFF747FD206900F0B2FF6069D1
:101F400000F0AFFFA06901F006F8E56945B1D5E9F9
:101F5000000600F04CFD284608F0F4FA3546F5E797
:101F6000206A01F025FA2046BDE8704008F0EABA80
:101F700070BD2DE9F8430446FFF7C6FF054620462D
:101F800000F026FF702806D00123E3602846FFF703
:101F9000C4FF002550E0204600F0F5FE0928F3D1EB
:101FA000204600F031FD2860204600F00CFF00289C
:101FB000ECD1204600F028FD6860204600F003FFC9
:101FC0000028E3D1204600F01FFDA860204600F065
:101FD000FAFE0028DAD12046FFF7CFFCE860204661
:101FE00000F0F1FE0028D1D1204600F069FF286101
:101FF000204600F0E8FE0028C8D1204600F060FF2F
:102000006861204600F0DFFE0028BFD1204600F0C6
:10201000BDFFA861204600F0D6FE0028B6D12046BC
:1020200000F0E8FE58B1204601F069FA2862204627
:1020300000F0C9FE0028A9D12846BDE8F883204653
:1020400000F0C6FE70289FD1204600F09CFE4FF0A5
:1020500000080746C146002FE5DD082008F088FA91
:102060000646C0F80090C0F80490204600F0CCFC72
:102070003060204600F0A7FE002887D1EB691BB92D
:10208000EE61013FB046E6E7C8F80460F9E710B535
:10209000044668B1006800F0AAFC606800F08CFC9F
:1020A000A06800F089FC2046BDE8104008F04ABA5C
:1020B00010BD10B5044680B1006800F0F2FE606803
:1020C00000F07AFCA06800F07BF9E06800F08FFC7B
:1020D0002046BDE8104008F035BA10BD10B50446E2
:1020E00050B1006801F05EFA606800F080FC2046A4
:1020F000BDE8104008F026BA10BD08B5202008F051
:1021000037FA2022002116F0B7F808BD10B50446B2
:10211000E0B1006800F06BFC606800F0C2FEA068EF
:1021200000F04AFCE06800F016FF206900F048F972
:10213000606900F045F9A06900F059FCE06900F021
:1021400056FC2046BDE8104008F0FCB910BD000068
:1021500038B50446FFF7D1FF0546204600F038FEAB
:10216000702807D001232846E360FFF7CFFF002542
:10217000284638BD204600F006FE0828F2D1204649
:1021800000F042FC2860204600F01DFE0028E9D146
:10219000204600F095FE6860204600F014FE0028FE
:1021A000E0D104226021204600F0BDFBA86020465B
:1021B00000F009FE0028D5D1204600F0E7FEE860D7
:1021C000204600F000FE0028CCD1144A14492046D5
:1021D00000F01FF92861204600F0F5FD0028C1D16C
:1021E000104A1149204600F014F96861204600F0B9
:1021F000EAFD0028B6D1204600F006FCA861204682
:1022000000F0E1FD0028ADD1204600F0FDFBE861C3
:10221000204600F0D8FD0028AAD0A3E78F200008B0
:102220003F220008B3200008C122000808B50C2096
:1022300008F09EF9002202604260826008BD38B555
:102240000446FFF7F3FF0546204600F0C1FD702865
:1022500007D001232846E360FFF719FF0025284631
:1022600038BD204600F08FFD0328F2D1204600F053
:10227000CBFB2860204600F0A6FD0028E9D1012212
:102280006021204600F04FFB6860204600F09BFD77
:102290000028DED101225021204600F044FBA86036
:1022A000204600F090FD0028D9D0D2E708B51020D4
:1022B00008F05EF91022002115F0DEFF08BD0000D5
:1022C00038B50446FFF7F2FF0546204600F080FDD2
:1022D000702807D001232846E360FFF7EAFE0025B7
:1022E000284638BD204600F04EFD0428F2D1204695
:1022F00000F0E6FD2860204600F065FD0028E9D1E9
:1023000008226021204600F00EFB6860204600F0A5
:102310005AFD0028DED10A4A0A49204600F079F821
:10232000A860204600F04FFD0028D3D1204600F0E1
:102330006BFBE860204600F046FD0028D0D0C9E7DE
:10234000DD2000085923000808B5082008F010F91E
:1023500000220260426008BD38B50446FFF7F4FF72
:102360000546204600F034FD702807D0012328469A
:10237000E360FFF7B3FE0025284638BD204600F095
:1023800002FD0228F2D1204601F022F92860204601
:1023900000F019FD0028E9D1204600F035FB686007
:1023A000204600F010FD0028E6D0DFE710B5044617
:1023B0000C2008F0DDF8002202604260846010BD4D
:1023C00038B5044688B938BD50F82500A368984749
:1023D0000135D4E90003AB42F6DC08B108F0B2F8ED
:1023E0002046BDE8384008F0ADB80025F1E738B523
:1023F00004460D464168013141608900006816F0CD
:10240000C7FD6368206003F18043013B40F823501F
:1024100038BD2DE9F84305468846164600F0D8FC3D
:1024200070281AD13046FFF7C1FF0446284600F055
:10243000AAFC00260746BE4202DB2046BDE8F88320
:102440002846C0478146284600F0BDFC28B94946C9
:102450002046FFF7CCFF0136EDE701232046EB6075
:10246000FFF7AEFF0024E8E708B5202008F080F869
:102470002022002115F000FF08BD38B5044600F009
:10248000A7FC702804D001230025E360284638BD4E
:10249000204600F078FC0728F5D1FFF7E5FF054658
:1024A000204600F0B1FA2860204600F08CFC00289D
:1024B000E9D1204600F0BCFC6860204600F083FCB7
:1024C0000028E0D1204600F0FBFCA860204600F088
:1024D0007AFC0028D7D101226021204600F023FA9F
:1024E000E860204600F06FFC0028CCD1012250218A
:1024F000204600F018FA2861204600F064FC00280D
:10250000C1D1204601F064F86861204600F05BFC10
:102510000028B8D1204600F077FAA861204600F0E4
:1025200052FC0028B2D0AEE710B50446C8B100682E
:1025300000F05DFA606800F06FFCA06800F0B1FC8C
:10254000E06800F039FA206900F036FA606901F0BD
:1025500029F8A06900F04BFA2046BDE8104007F0CA
:10256000F1BF10BD10B530B1C469FFF7DDFF14B184
:102570002046E469F9E710BDF8B5054600F03AFCDD
:10258000044608B1002406E0284600F021FC70282B
:1025900003D00123EB602046F8BD284600F0F3FB92
:1025A000061EEFDD2846FFF768FF0446284600F0C8
:1025B0000AFC70B92746013E002EECD02846FFF7F2
:1025C0005CFFF861284600F0FEFB10B9FF69013E90
:1025D000F2E701232046EB60FFF7C4FFD2E70000DB
:1025E00038B50546082007F0C3FF00230446036002
:1025F0004360284600F0ECFB702806D00123EB6016
:10260000204607F09FFF002459E0284600F0BBFB5E
:102610000228F3D104226021284600F084F92060CA
:10262000284600F0D0FB0028EAD123681968B1F5EC
:10263000806F52D01DD8B1F5007F46D00AD8B1F5D1
:10264000807F38D040F2011399423AD02F4816F0DB
:102650002FFC34E0B1F5407F3FD040F20133994286
:1026600037D040F201239942F0D12846FFF7F6F91E
:1026700024E0B1F5C06F3CD00ED8B1F5A06F30D0DA
:1026800040F20153994230D040F201439942DDD1EA
:102690002846FFF7C5FB11E040F2017399422CD0A8
:1026A0004FF6017399422CD0B1F5E06FCED1284698
:1026B000FFF70DFA02E0284600F032FA606020468B
:1026C00038BD284600F0A9FAF8E72846FFF792F946
:1026D000F4E72846FFF73CFDF0E72846FFF749FC02
:1026E000ECE72846FFF7DCFAE8E72846FFF738FB77
:1026F000E4E7284600F002FBE0E72846FFF758FA37
:10270000DCE72846FFF7F6F8D8E700BF73B6010804
:1027100010B50446002875D003681A68B2F5806FBA
:1027200054D01ED8B2F5007F4CD00BD8B2F5807FC4
:1027300039D040F201139A4240D03349334816F061
:10274000B7FB33E0B2F5407F40D040F201339A420C
:1027500040D040F201239A42EFD14068FFF772F96E
:1027600024E0B2F5C06F41D00ED8B2F5A06F35D0DD
:1027700040F201539A4235D040F201439A42DCD1F3
:102780004068FFF729FB11E040F201739A4231D013
:102790004FF601739A4231D0B2F5E06FCDD1406867
:1027A000FFF77DF902E0406800F09CF9206800F036
:1027B00003F92046BDE8104007F0C4BE406800F0B1
:1027C00011FAF3E74068FFF709F9EFE76068FFF7F0
:1027D000A4FBEBE74068FFF799FCE7E74068FFF7E9
:1027E00047FAE3E74068FFF7A9FADFE7406800F03F
:1027F0006DFADBE74068FFF7BDF9D7E74068FFF700
:1028000064F8D3E710BD00BF3EB6010854B6010816
:1028100010B5044698B1006800F0E9F8606800F06F
:10282000CBF8A06800F0C8F8E068FFF771FF2069F6
:1028300000F0C2F82046BDE8104007F083BE10BD8E
:1028400038B50446142007F093FE142200210546F3
:1028500015F012FD204600F0BBFA702806D00123C7
:10286000E3602846FFF7D4FF00253FE0204600F054
:102870008AFA0628F3D1204600F0C6F828602046E0
:1028800000F0A1FA0028ECD101226021204600F0DE
:102890004AF86860204600F096FA0028E1D101224B
:1028A0006021204600F03FF8A860204600F08BFA37
:1028B0000028D6D12046FFF793FEE860204600F0BE
:1028C00082FA0028CDD102226021204600F02BF8A8
:1028D0002861204600F077FA0028C2D1204600F097
:1028E0007DFA18B90121204600F080FA284638BD4B
:1028F000B0B5CB1D23F0070300AFADEB030D0A46C7
:102900000C4605460146684615F08EFC00230DEB8B
:1029100004029C4202F1FF3201DCBD46B0BD1178D9
:10292000E9540133F5E72DE9F84305460C4617460F
:1029300000F060FA064638B9284600F049FAA0428D
:10294000814603D00123EB6000242FE0284600F0ED
:102950001AFAB0F10008F5DBB845F3DC384607F0A9
:1029600007FE31463A46044615F086FC284600F03C
:1029700035FAB9F1500F08BFC0F3C016284600F071
:1029800031FAA7EB0809A14401464246484615F032
:102990004BFC1EB12346FF224B450AD13946204647
:1029A000FFF7A6FF4146284600F020FA2046BDE882
:1029B000F88303F8012BEFE708B107F0C3BD7047B8
:1029C00070B5064608200D4607F0D2FD00239D4253
:1029D00004460360436008DD284607F0C9FD2A4627
:1029E0002060314615F020FC6560204670BD10B5B2
:1029F000044640B1006808B107F0A4FD2046BDE8D8
:102A0000104007F09FBD10BD70B5044600F0F2F90C
:102A100028B9204600F0DCF918B10123E360002555
:102A20000FE0204600F0AFF9061EF6DB204600F06E
:102A3000D9F93146FFF7C4FF31460546204600F07C
:102A4000D5F9284670BD03463038C0B209280DD9E3
:102A5000A3F16102052A02D8573BD8B27047A3F10F
:102A60004102052A01D8373BF7E70020704710B52F
:102A700004460078FFF7E7FF01466078FFF7E3FFC1
:102A800040EA0110C0B210BD2DE9F84300AF044682
:102A900016F078FBC3071AD44510EB1D23F007038B
:102AA000ADEB030DE8460DF1FF3604EB45094C454F
:102AB00006D129464046FFF783FFBD46BDE8F883AF
:102AC0002046FFF7D4FF023406F8010FEFE700209D
:102AD000F3E708B51C2007F04BFD1C22002115F080
:102AE000CBFB08BD10B50446C8B10068FFF77FFFF7
:102AF0006068FFF77CFFA068FFF779FFE068FFF7E9
:102B000076FF2069FFF773FF6069FFF770FFA06928
:102B1000FFF752FF2046BDE8104007F013BD10BD7F
:102B200038B50446FFF7D5FF0546204600F050F9BA
:102B3000702806D00123E3602846FFF7D3FF002565
:102B400045E0204600F01FF90728F3D12046FFF7A3
:102B50005BFF2860204600F036F90028ECD12046C3
:102B6000FFF752FF6860204600F02DF90028E3D1FE
:102B70002046FFF749FFA860204600F024F900280E
:102B8000DAD12046FFF740FFE860204600F01BF94D
:102B90000028D1D12046FFF737FF2861204600F0FA
:102BA00012F90028C8D12046FFF72EFF68612046A1
:102BB00000F009F90028BFD1012260212046FFF76B
:102BC000B2FEA861204600F0FEF80028B4D12846E5
:102BD00038BD08B5182007F0CBFC1822002115F0ED
:102BE0004BFB08BD10B50446B0B10068FFF7FFFE0F
:102BF0006068FFF7FCFEA068FFF7F9FEE068FFF7EA
:102C0000F6FE206900F04DF96069FFF7D5FE204619
:102C1000BDE8104007F096BC10BD38B50446FFF77C
:102C2000D8FF0546204600F0D3F8702806D00123CF
:102C3000E3602846FFF7D6FF00253CE0204600F081
:102C4000A2F80628F3D12046FFF7DEFE28602046D2
:102C500000F0B9F80028ECD12046FFF7D5FE6860F7
:102C6000204600F0B0F80028E3D12046FFF7CCFE64
:102C7000A860204600F0A7F80028DAD12046FFF728
:102C8000C3FEE860204600F09EF80028D1D120461F
:102C900000F016F92861204600F095F80028C8D108
:102CA000012260212046FFF73EFE6861204600F0C9
:102CB0008AF80028BDD1284638BD08B5142007F091
:102CC00057FC1422002115F0D7FA08BD10B50446B0
:102CD00098B10068FFF78BFE6068FFF788FEA06878
:102CE000FFF785FEE06800F036F9206900F060FB30
:102CF0002046BDE8104007F025BC10BD38B504469D
:102D0000FFF7DBFF0546204600F062F8702806D08A
:102D10000123E3602846FFF7D9FF002531E0204674
:102D200000F031F80528F3D12046FFF76DFE28604A
:102D3000204600F048F80028ECD12046FFF764FE5A
:102D40006860204600F03FF80028E3D12046FFF7F6
:102D50005BFEA860204600F036F80028DAD1204655
:102D600000F014F9E860204600F02DF80028D1D1D9
:102D7000204600F0C4FB2861204600F024F800281B
:102D8000C8D1284638BDF0B5836805680022EB5CE1
:102D9000466803F07003703B18BF4FF0FF33816843
:102DA000B14201F1010402D38460D018F0BD695C26
:102DB00001F00F07090647EA0212F5D58460002BDF
:102DC000EDD0013BEBE7C068003018BF0120704731
:102DD00002688368D05C00F0700070470268836806
:102DE000D05C70470268806810447047836819445B
:102DF00081607047826803689B5C012B03BF0132CE
:102E0000826018460020704708B5082007F0B0FB24
:102E100000220260426008BD10B5044638B1406827
:102E2000FFF7CAFD2046BDE8104007F08BBB10BD80
:102E3000F8B50646FFF7DEFF30BB3046FFF7C8FFA8
:102E400005463046FFF7CAFF0746FFF7DDFF602D56
:102E5000057004464FF0010519D107F00F07013F37
:102E600000E06D00AF42FCDC2A4660213046FFF7EF
:102E70005AFD237860601D4325703046FFF7A3FF9D
:102E800018B12046FFF7C8FF00242046F8BDF560C2
:102E9000F3E708B5082007F06BFB002202604260F0
:102EA00008BD10B5044650B10068FFF785FD6068A5
:102EB000FFF782FD2046BDE8104007F043BB10BD80
:102EC00038B50446FFF796FF60B9FFF7E2FF054605
:102ED0002046FFF77DFF702806D00123E3602846D7
:102EE000FFF7DFFF00251AE02046FFF74CFF02281E
:102EF000F3D1012260212046FFF715FD286020460E
:102F0000FFF761FF0028EAD1042260212046FFF785
:102F10000AFD68602046FFF756FF0028DFD12846EB
:102F200038BD08B5082007F023FB0022026042608C
:102F300008BD38B504460D460168013101608900BD
:102F4000406816F025F82368606003F18043013B78
:102F500040F8235038BD38B50446B0B143687BB162
:102F60000368002B0CDD0025636853F82500FFF78C
:102F70003EFD23680135AB42F6DC606807F0E2FAFB
:102F80002046BDE8384007F0DDBA38BDF8B5054643
:102F9000FFF730FF48B9FFF7C4FF04462846FFF7A4
:102FA00017FF702803D00123EB60002405E02846BA
:102FB000FFF7E9FE0646002E01DC2046F8BD284654
:102FC000FFF722FD07462846FFF7FDFE28B1012343
:102FD0002046EB60FFF7BFFFE7E71FB13946204609
:102FE000FFF7A7FF013EE6E708B5102007F0C0FA9B
:102FF0001022002115F040F908BD38B504460D46F1
:10300000C1680131C1608900806815F0C1FFE368C3
:10301000A06003F18043013B40F8235038BD08B560
:10302000082007F0A5FA00220260426008BD08B53A
:103030005C2007F09DFA5C22002115F01DF908BD07
:1030400010B50446002849D00068FFF7D0FC60683E
:10305000FFF727FFA068FFF7AFFCE068FFF7ACFCC5
:103060002069FFF7A9FC6069FFF7A6FCA069FFF7DC
:10307000A3FCE069FFF7A0FC206AFFF79DFC606AF3
:10308000FFF79AFCA06AFFF797FCE06AFFF794FC51
:10309000206BFFF7ACFC606BFFF78EFCA06BFFF7BB
:1030A0008BFCE06BFFF788FC206CFFF785FC606C05
:1030B000FFF782FCA06CFFF77FFCE06CFFF77CFC65
:1030C000206DFFF779FC606DFFF776FCA06DFFF7D0
:1030D0008EFC2046BDE8104007F034BA10BD38B56C
:1030E0000446FFF787FE60B9FFF7A1FF05462046BB
:1030F000FFF76EFE702806D00123E3602846FFF735
:103100009FFF002505E12046FFF73DFE1728F3D17C
:103110002046FFF779FC28602046FFF754FE002880
:10312000ECD12046FFF7CCFE68602046FFF74BFE4F
:103130000028E3D1082260212046FFF7F4FBA860B5
:103140002046FFF740FE0028D8D10122602120460A
:10315000FFF7E9FBE8602046FFF735FE0028CDD1F8
:10316000012250212046FFF7DEFB28612046FFF7B1
:103170002AFE0028C2D1082250212046FFF7D3FBA7
:1031800068612046FFF71FFE0028B7D101226021A9
:103190002046FFF7C8FBA8612046FFF714FE002871
:1031A000ACD1012250212046FFF7BDFBE86120464B
:1031B000FFF709FE0028A1D1082250212046FFF781
:1031C000B2FB28622046FFF7FEFD002896D10122BF
:1031D00060212046FFF7A7FB68622046FFF7F3FD5A
:1031E00000288BD1012250212046FFF79CFBA862CA
:1031F0002046FFF7E8FD002880D108225021204614
:10320000FFF791FBE8622046FFF7DDFD00287FF421
:1032100075AF2046FFF7F8FB28632046FFF7D3FD84
:1032200000287FF46BAF012260212046FFF77BFB73
:1032300068632046FFF7C7FD00287FF45FAF0122D7
:1032400050212046FFF76FFBA8632046FFF7BBFD28
:1032500000287FF453AF082250212046FFF763FB7C
:10326000E8632046FFF7AFFD00287FF447AF012257
:1032700060212046FFF757FB28642046FFF7A3FD97
:1032800000287FF43BAF012250212046FFF74BFB83
:1032900068642046FFF797FD00287FF42FAF0822CF
:1032A00050212046FFF73FFBA8642046FFF78BFD27
:1032B00000287FF423AF012260212046FFF733FB73
:1032C000E8642046FFF77FFD00287FF417AF012256
:1032D00050212046FFF727FB28652046FFF773FDA6
:1032E00000287FF40BAF082250212046FFF71BFB7C
:1032F00068652046FFF767FD00287FF4FFAE204693
:10330000FFF782FBA8652046FFF75DFD00287FF4EC
:10331000F5AE284638BD08B5142007F029F9142267
:10332000002114F0A9FF08BD10B5044698B100684B
:10333000FFF75DFB6068FFF73FFBA068FFF73CFB12
:10334000E06800F02FF92069FFF751FB2046BDE847
:10335000104007F0F7B810BD10B5044638B3D0E9F7
:103360000030FBB11B78013B032B16D8DFE803F0DC
:10337000020C0F1200F016F92068FFF71DFB204623
:10338000BDE8104007F0DEB8FFF7CEFFF4E7FFF727
:1033900057FEF1E7FFF785FDEEE70028ECD007F0D8
:1033A000D1F8E9E70028EAD007F0CCF8E7E710BD4C
:1033B00038B50446B8B10068FFF719FB6068FFF73D
:1033C000CBFF0025D4E90203AB4206DC07F0BAF8D4
:1033D0002046BDE8384007F0B5B850F82500FFF7A3
:1033E000E7FF0135EEE738BD38B50446FFF702FDCB
:1033F00060B9FFF790FF05462046FFF7E9FC70280B
:1034000006D00123E3602846FFF78EFF002535E054
:103410002046FFF7B8FC0528F3D12046FFF7F4FA61
:1034200028602046FFF7CFFC0028ECD10122602164
:103430002046FFF778FA68602046FFF7C4FC0028B2
:10344000E1D1012250212046FFF76DFAA860204605
:10345000FFF7B9FC0028D6D1204600F0B9F8E860A3
:103460002046FFF7B0FC0028CDD12046FFF7CCFA6C
:1034700028612046FFF7A7FC0028C4D1284638BDA4
:1034800038B50546FFF7B6FC60B9FFF7C8FD04463E
:103490002846FFF79DFC702806D00123EB602046EC
:1034A000FFF75AFF00241CE02846FFF76CFC0228B7
:1034B000F3D1012260212846FFF735FA2060284623
:1034C000FFF781FC0028EAD123681B78013B032B1E
:1034D000E3D8DFE803F002080C10284600F078F883
:1034E0006060204638BD2846FFF77EFFF8E7284693
:1034F000FFF7F5FDF4E72846FFF7E2FCF0E7F8B543
:103500000446FFF777FC60B9FFF76EFD05462046DD
:10351000FFF75EFC702806D00123E3602846FFF722
:1035200047FF002525E02046FFF72DFC0328F3D1B7
:103530002046FFF769FA28602046FFF744FC002880
:10354000ECD12046FFF79CFF68602046FFF73BFC6C
:103550000028E3D12046FFF74DFC50B92046FFF785
:1035600037FC7028D8D12046FFF70DFC0646002E08
:1035700001DC2846F8BD2046FFF7C1FF074620467C
:10358000FFF721FC0028C9D11FB139462846FFF7B3
:1035900034FD013EEBE708B5082006F0E9FF002303
:1035A000036008BD10B5044688B10378406823B1B4
:1035B000402B09D0FFF700FA01E0FFF718FA204688
:1035C000BDE8104006F0BEBFFEF7FDF9F7E710BDFD
:1035D000F8B50546FFF70EFC38BB2846FFF7F8FBA9
:1035E00006462846FFF7FAFB0746FFF7D4FFF1B27D
:1035F000402E044601701BD003DC5EB10123EB605A
:103600000CE0502E01D0602EF8D107F00F070126F4
:10361000013F12E02846FFF7F7F960602846FFF700
:10362000D2FB18B12046FFF7BDFF00242046F8BDAD
:103630002846FEF7A2F9F0E77600B742FCDC3246F6
:103640002846FFF770F9237860601E432670E5E78F
:1036500038B50A4C05460121204603F0C9FF002376
:1036600020461A46012103F001FF85F001022046A1
:10367000BDE83840012103F0C7BF00BF0000024091
:1036800008B50120FFF7E4FFBDE80840032004F07F
:10369000BBBE0846FFF7DCBF10B50446024B036013
:1036A00013F04EF9204610BDACB6010810B5044623
:1036B000054B503040F8503C044B40F8083CFFF7B5
:1036C000EBFF204610BD00BFA4BA0108B0BC010842
:1036D00010B50446FFF7E0FF2046082112F04EFB2C
:1036E000204610BD10B50446FFF7E0FF20467421C8
:1036F00012F044FB204610BD024B012118680368FC
:103700001B681847C4080020021C18BF01220321AF
:10371000014803F079BF00BF0004024010B50C4619
:103720000AF058FF022808D14FF47A704443B4FBE2
:10373000F0F0BDE810400AF0BDBC2046BDE81040E6
:1037400003F0B0BC0321014803F067BF000402404E
:1037500010B5094C094806F06FFE20460B2103F016
:1037600047FF002320461A460B2103F07FFEBDE8E9
:10377000104003F07DBC00BF0000024041BA0108C8
:1037800008B5022003F0D8FB03F03AFC00F04CFC33
:1037900003F060FC00F036FE04F0C0F90C4803F0C2
:1037A0004BF94FF4E13004F0A3FC0A4B1A680AB954
:1037B000094A1A60094B1A680AB9074A1A60084888
:1037C00006F03AFEBDE80840064806F035BE00BFE8
:1037D00081360008940B0020A57F0008980B00207C
:1037E0001CB7010834B701082DE9F3470446264603
:1037F0004FF01B0913F03CF8274B04F1210846F861
:10380000113B10220021304614F036FD4A460021BB
:10381000404614F031FD00252146204BC4E90F55E8
:1038200004F1480041F8443F00F0AEFF1C4B1D4F2F
:10383000A3651D4B84F85C5023661C4BC4E91A55E4
:10384000636684F870501A4806F0F6FD3B68DFF8AE
:103850006CA00193DAF80030164D00932B68164ADD
:103860004946404615F0ACFB2968304606F0E1FEBB
:10387000DAF8001004F1150006F0DBFE396804F1F7
:10388000190006F0D6FE296804F11D0006F0D1FEED
:10389000204602B0BDE8F087A4BA010890BB010839
:1038A000E0BB01086400F81F10BC0108FCBB010864
:1038B00075BA01085000F81F8ABA01085400F81FB1
:1038C00010B5094CFFF75CFF2368DB0709D40748F4
:1038D000FFF78AFF0123064A06490448236013F0D4
:1038E00085F8024810BD00BFBC080020C8080020B1
:1038F00000000020AD36000838B5064D064C2B6898
:1039000013F0010F04D1FFF7DBFF012320602B60D0
:10391000206838BDC00800203C09002008B50B21F4
:10392000054803F07FFE28B1BDE808400B2102489E
:1039300003F08CBE08BD00BF0000024008B519B1FD
:10394000BDE80840FFF704BF044806F075FDBDE878
:10395000084002220B21024803F0C6BD5DBA0108EF
:103960000000024070B504462E4804F1440506F0FC
:1039700063FD2846002100F06DFD0021284600F07F
:103980007FFD204612F0A4FF0CF08AFD20460021A6
:10399000FFF7D4FF0BF00EFC01220C21224803F0AC
:1039A000A3FD04F0D9F904F1480000F0CFFE23682C
:1039B0002046DB6804F16405002198471B4E002176
:1039C000284600F0E3FD03F09DFE194806F034FDA3
:1039D00004F086FA03F03EFB304601220D2103F08D
:1039E00083FD012230460E2103F07EFD00210846B2
:1039F00004F070F904F1580000F058FD0121284648
:103A000000F0C4FD4FF4E13004F072FB094806F009
:103A100013FD0BF0F5FA04F09DF92046BDE8704067
:103A200012F063BF0FBA0108000402400000024018
:103A300033BA0108BDC9010838B50546FFF76EFF66
:103A4000044628B100212846FFF778FF03F010FB59
:103A500003F016FA05460CB1FFF77AFE284638BD8A
:103A600070B50C4606461549204614F0A5F820B955
:103A70000021204614F082F870B11149204613F05D
:103A8000DFFE14F0A3F801460E4806F0D5FC40F224
:103A90007D110D4803F00AF83046FFF73FFF054659
:103AA00048B93046FFF7C8FF0146204614F084F8B5
:103AB00008B1FFF74DFE284670BD00BF33335340B9
:103AC00000007A444AB7010879B7010870B52D4A59
:103AD000D6B013680546DB0705D42B4900F1640313
:103AE0000B600123136029492846FFF7B9FF0646FA
:103AF000274806F0A1FC002105F1440000F0C0FCBD
:103B0000244C254BE360254B2361254BA360254BBB
:103B10006360254B2360254B6361254BA361254BD7
:103B2000E36104F110030FCB8DE80F0094E80F0060
:103B300012F0EEFB002305A8EB632B6412F070FB80
:103B40009DF8143005F13C04012B14D1DDF815303B
:103B500005A8EB63DDF819302B6412F031FB164831
:103B600006F06AFC0821204606F0CCFCBDF91611CF
:103B7000124806F061FC31462846FFF7DFFE56B0DA
:103B800070BD00BFB8080020C408002000004040FD
:103B9000B5B6010854540020A57000082D70000827
:103BA000F9360008453700080937000839A400082D
:103BB00055C6000895C60008D6B60108FCB601082F
:103BC0007FB5F82300F15805064628468DF80F30DA
:103BD00000F072FC02230DF10F0100930122A123DA
:103BE000284600F06DFC4FF400430822009306F1D4
:103BF0006801A1230446284600F08CFC0440E4B28E
:103C0000284600F05BFC204604B070BD30B58BB098
:103C1000044604F027FC0146574806F00DFC5748BF
:103C200006F00AFC204600F0A3FB04F1580500F062
:103C3000D5FA00F081FA5248524906F0FDFB2846B9
:103C400000F034FC38B9504806F0F6FB4FF49D7193
:103C50004E4802F02BFF03F00BFA2046FFF7B0FFAF
:103C600020B940F23F11494802F020FF94F86F302C
:103C700094F86920049394F86E3094F868100393D4
:103C800094F86D304248029394F86C30019394F8A4
:103C90006B30009394F86A3006F0CEFB284600F0B3
:103CA0004DFA284600F0ACFA04F14405002184F8EE
:103CB0007000284600F0CEFB012000F073FD0021CB
:103CC000284600F0DDFB012000F08AFD2046FFF7CA
:103CD000FDFE00F0E1FA2F4806F0AEFB4FF4FA705B
:103CE00014F076FA054600283ED12B4806F0A4FBD6
:103CF0002A4806F0A1FB2A4806F09EFB294806F058
:103D00009BFB294806F098FB284806F095FB2848BD
:103D100006F092FB274806F08FFB274806F08CFB45
:103D2000264A2749274806F087FB2749274806F0F7
:103D300083FB274806F080FB04F12101254806F0AB
:103D40007BFB2549254806F077FB07A803F07EFE9C
:103D500007A806F0C7FA0146214806F06DFB104897
:103D600006F06AFB0BB030BD1E4806F065FB284626
:103D700014F036FABCE700BFB9B70108CFB70108A5
:103D8000E6B70108A086010001B8010879B701086B
:103D900017B801084CB801087FB80108B2F0010853
:103DA000B3B80108E4B80108F3B8010815B901086F
:103DB00038B901085CB90108B3F001087FB90108FE
:103DC00085B9010890B90108A0B90108A7B901088F
:103DD000B2B90108D2B90108DDB90108E3B9010897
:103DE000FDB90108CEB501082DE9FF4100F15805E4
:103DF000284600F061FB04240226284F013C14F001
:103E0000FF0433D0A123012239460096284600F052
:103E100057FB4FF40043804600930422A12302A9DC
:103E2000284600F077FBB8F1000F01D10028E5D05B
:103E30009DF80830442B20D19DF809306E2B1CD101
:103E40000DF10A0006F0E3FB0223013084B22146A3
:103E50000DF109008DF8083006F0F4FB0023032271
:103E60000093A02302A9284600F02AFB284600F070
:103E700025FB204604B0BDE8F0814FF488430024C0
:103E8000ADF808306E2300210DF10B008DF80A30DB
:103E900006F0D8FB0094A0230522E3E7B4B601089E
:103EA00038B50C46113105460CF0B6F9214651F8EB
:103EB000683F28462B604B686B6038BD30B50D46B7
:103EC0009DB0044601466846FFF7EAFF694628466A
:103ED0000BF0DCFE04F1110321346B632C631DB085
:103EE00030BD0000024B186803685B68184700BFCC
:103EF0004C090020024B186803689B68184700BFF4
:103F00004C0900200023F0B5137014460222054628
:103F10000C4E85B030688DF80F1003680092DF6892
:103F200001222B460DF10F01B84748B14FF4004272
:103F300030682146036800921E6901222B46B04773
:103F400005B0F0BD4C09002030B585B08DF80D20CE
:103F50000022074B8DF80C101C6803A923680092FF
:103F6000DD68022203462046A84705B030BD00BFE9
:103F70004C09002037B54FF40045064B1C682368F8
:103F800000951D6913460A4601462046A84703B01E
:103F900030BD00BF4809002037B50025054B1C681F
:103FA00023680095DD6813460A4601462046A84767
:103FB00003B030BD4809002037B50225054B1C6809
:103FC00023680095DD6813460A4601462046A84747
:103FD00003B030BD48090020024B186803681B6815
:103FE000184700BF48090020024B186803685B6847
:103FF000184700BF48090020024B186803689B68F7
:10400000184700BF480900204FF47A735843B0FBAB
:10401000F3F00AF04FB810B50446FFF76DFC2146E7
:10402000BDE81040FFF7E0BE10B5424C0BF014F9AC
:1040300020460222002103F057FA012220461146B1
:1040400003F052FA20460122022103F04DFA2046E5
:104050000222032103F048FA20460022042103F043
:1040600043FA20460222082103F03EFA20460122AC
:10407000092103F039FA204601220A2103F034FA1B
:10408000204602220B2103F02FFA02F0E3FF002367
:1040900020461A460C2103F0E9F9204600220C21A3
:1040A00003F0B2FA2046002204F580640F2103F0E9
:1040B0001BFA20460122002103F016FA20460022B6
:1040C000022103F011FA20460022032103F00CFA2A
:1040D00020460222062103F007FA2046002208218A
:1040E00003F002FA20460022092103F0FDF92046E0
:1040F00001220C2103F0F8F9204602220D2103F0E1
:10410000F3F9204602220E2103F0EEF920460222A6
:104110000F2103F0E9F9002304F5806420461A46D4
:104120000D2103F0A3F92046BDE8104000220D2127
:1041300003F06ABA0000024003F0F0BC1C4B00B56B
:104140001A6889B0D2075FBF1A4A106001221A604C
:10415000194B0493194B0593194B0393194B029375
:10416000194B0793194B069308AB13E903008DE82D
:10417000030002AB0FCB11F079FF90B1144806F0A9
:104180005BF900221348114603F0AEF90F23022217
:104190000021104803F048F809B05DF804EB11F075
:1041A000FFBE69210C4809B05DF804EB02F07EBC4B
:1041B000440900204C090020E53E0008F53E0008B7
:1041C000053F0008493F000839A4000809400008DD
:1041D00036BB01080000024047BB0108002307B5B9
:1041E000ADF8043001238DF8063001980AF090FFF5
:1041F00002F030FF03B05DF804EB0AF0DBBF000013
:10420000194B10B51A688CB0D2075FBF174A1060FF
:1042100001221A60164B0793164B0593164B069313
:10422000164B0893164B0993164B0A93164B0B9398
:104230000CAB13E907008DE8070005AB0FCB11F0BD
:1042400039FE044601220F21104803F04DF93CB11C
:104250000F4806F0F1F811F00BFE20460CB010BD2F
:104260000C4806F0E9F8F8E740090020480900206A
:10427000753F0008993F0008B93F0008D93F000882
:10428000E93F0008F93F000839A400080000024097
:10429000B8BA0108EBBA01082DE9F0479EB00BF05F
:1042A000C5FBDFF8C890284C284E294F16AD50B9F1
:1042B000CDE91944CDE91776CDF85890009495E8EA
:1042C0000F000BF0B9FB234B4FF0000A1793224B62
:1042D0004FF001081693214B09A91893204B28464B
:1042E0001993204BCDE91C76CDE91A340423CDE98E
:1042F000093A8DF8298006F08BFD06F07DFD14F05B
:10430000EFFD514610220CA813F0B6FF164BCDE975
:104310001044159303238DF836800B9302AC0BAD3C
:104320000FCDCDE91376CDF848900FC42B682360EC
:1043300014AB93E803008DE8030010AB0FCB0BF038
:10434000ADFF1EB0BDE8F08739A4000845A5000800
:1043500071A5000839F1000801F0000811EF00080C
:10436000A9EE0008BDEE000817400008097B000810
:104370002DE9F047044602F083FD1E49054613F07F
:104380005FFA13F023FC01461B4806F055F84FF086
:104390008041284613F0F2FB48B30025DFF8609017
:1043A000DFF85080154E02F06BFD4946074613F0CA
:1043B000F9FBA8B94146384613F042FA13F006FC5F
:1043C0000146304606F038F8236885F0010520469E
:1043D000DB68294698474FF47A7002F063FEE2E703
:1043E00023682046BDE8F047DB6800211847BDE898
:1043F000F08700BF00007A4409BB01081BBB01081D
:104400000000204008B50D49012003F0DFF90C49F8
:104410000B2003F0DBF90B490A2003F0D7F90A4916
:10442000042003F0D3F90949072003F0CFF9BDE8D0
:1044300008400749052003F0C9B900BF39C1000889
:1044400081C40008F1C20008A1C50008F5C4000835
:104450007DC50008002310B50C461A460D210748FB
:1044600003F004F814B1012C00D010BD2246BDE8C1
:1044700010400D21014803F0C7B800BF00080240FA
:10448000002310B50C461A460C21074802F0EEFF37
:1044900014B1012C00D010BD2246BDE810400C2103
:1044A000014803F0B1B800BF00000240014803F02A
:1044B00017B900BFA086010003F0E2B803F0FCB812
:1044C0002DE9F041069F1E4607F00303032B8046AB
:1044D0000C46154603D12F210D4802F0E7FA20467D
:1044E000BC07324629460AD503F034F910B1012041
:1044F000BDE8F0810123002088F80430F8E7FB07CD
:1045000002D503F035F9F1E703F016F9EEE700BF45
:1045100098BB01082DE9F041069C0D46E107804655
:1045200016461F4603D54C210D4802F0BFFAA207DC
:1045300003D54F210A4802F0B9FA23043A4631461E
:1045400028460AD503F022F910B10120BDE8F08118
:104550000123002088F80430F8E703F0DFF8F3E7E0
:1045600098BB010808B50321034803F056F8003052
:1045700018BF012008BD00BF000402400A460248DF
:10458000032103F041B800BF0004024008B581B127
:10459000012303211A460A4802F068FF0321084854
:1045A00003F026F8BDE8084003220548114602F052
:1045B0003DBF0122BDE808400321014802F094BF3D
:1045C0000004024003F0A0BA1FB501A805F04CFE9C
:1045D00001A803F02BFA05B05DF804FB1FB501A894
:1045E00005F042FE01A803F06FFB05B05DF804FB87
:1045F00003F0D8BA03F0F0BA084603F069B9DFB5A2
:104600000023CDE90133ADF80C3001238DF80730DC
:104610008DF808306FF01D038DF80930072304462C
:1046200001A88DF80A3005F044FE236806461B6891
:1046300020460F469847864277EB0103B4BF01201E
:10464000002004B0D0BD7047704700007FB500F176
:104650000806054630460C4612F09CF960BB33480C
:1046600005F0EAFEA27C617C314805F0E5FE637C42
:104670003BB16868002103681B689847022000F07E
:1046800091F8A37C3BB16868002103685B68984798
:10469000022000F0A5F861684E2918D04F2916D0E5
:1046A000452914D01521234802F000FA1621224B87
:1046B000224A204813F08AFC6421304612F056F951
:1046C0000028CFD142211B4802F0F0F9CAE7A368C5
:1046D000073B022B15D81A4AD25CE3680A2B18D084
:1046E00009DC052B16D03321124802F0DFF9124BFA
:1046F000144A3421DDE70F2B0CD0142BF3D1022305
:1047000008E023210B4802F0D1F90B4B0E4A24217B
:10471000CFE70123A07C0290607C0190207C009078
:10472000206803F01FFD04B070BD00BF2FBC01085E
:1047300088BC010848BC0108A6B30108D0BC010828
:104740002CBC010800BD010834BD010810B50446A9
:1047500003F0DAFC04F10800BDE8104012F01DB9C6
:10476000084603F0CFBD38B50C468D18AC4204D0D6
:1047700014F8010B03F0C6FDF8E738BD03F0EABCFE
:10478000084603F0EFBD000010B50446044BC0E935
:1047900000310121083012F00BF9204610BD00BF96
:1047A000B0BC0108042817D8DFE800F00309100E98
:1047B0001200002303211A46084802F057BE0022C7
:1047C0000321064802F090BE0222F9E70122F7E732
:1047D0000321024802F0AEBE704700BF0000024055
:1047E000042817D8DFE800F00309100E1200002398
:1047F00002211A46084802F039BE0022022106486A
:1048000002F072BE0222F9E70122F7E70221024814
:1048100002F090BE704700BF000002401FB5536811
:104820000293137801934B6800930B6842680178F8
:10483000024805F001FE05B05DF804FB6CBD0108FF
:1048400010B50446C06908B105F07CFE206908B1C6
:1048500005F078FE606808B105F074FE204610BDD2
:1048600010B50446006808F0B9FD204610BD0000F0
:10487000CB21014802F01AB98ABD0108FE2307B511
:104880008DF80430054B01A91868002300681A460A
:1048900008F090FA03B05DF804FB00BF5C0900204B
:1048A000D0B51F467423C0E900310023044683605D
:1048B0000820164611F042FAC0E90067A0602046C1
:1048C000D0BD0000036837B5632B05460C4601D008
:1048D000FFF7CEFF002301AAA9682046019305F047
:1048E00091FB019A3AB12146044805F0A5FD382113
:1048F000034802F0DBF803B030BD00BFCCBD0108B7
:10490000F9BD010870B563230025C0E900310446F4
:1049100085601A20164611F011FA1A22294613F062
:10492000ABFC3146A0602046FFF7CCFF204670BDAF
:1049300081647047C16470472DE9F843D0E9017381
:10494000884600254FF00C09DB1B0A4E9B105E4386
:10495000ECB2B4420BD209FB04724146506814F029
:10496000FFFB01350028F3D12046BDE8F8834FF066
:10497000FF30FAE7ABAAAAAA2DE9F843D0E90473FD
:10498000884600254FF00C09DB1B0A4E9B105E4346
:10499000ECB2B4420BD209FB04724146506814F0E9
:1049A000DFFB01350028F3D12046BDE8F8834FF046
:1049B000FF30FAE7ABAAAAAA2DE9F0470E464968EC
:1049C0000446FFF7B9FFC0B2FF2807D071682E4830
:1049D00005F032FD7C212D4802F068F8D4E901236E
:1049E0002B4F9B1A9B107B437E2B03D97F2127489B
:1049F00002F05CF8D4E901120C25E068531A9B1010
:104A0000121A7B4392107A430133934205FB03F859
:104A10000ED84144A160D4E9013496E80700E31AB6
:104A200004E907001A489B1058430138BDE8F08795
:104A3000404605F09DFD054618B96921154802F06C
:104A400035F8D4E901C300274FF00C0AA3EB0C039F
:104A50000F4A9B1002FB03F9A9EB0703002B0ADDA9
:104A60000AFB07F305EB030E634493E807000137E5
:104A70008EE80700F0E7604605F064FD6560454498
:104A8000C4E90255C7E700BF41C30108F9BD0108E9
:104A9000ABAAAAAA61C301081FB56E23CDE90131F3
:104AA000002301A90393FFF787FF05B05DF804FB1E
:104AB000FF22F8B5002380F8282004464FF0FF3588
:104AC0006FF07F42C0E90033C0E90233C0E904332C
:104AD000C0E90633C0E908334FF000410020052645
:104AE0000027C4E91052234DC4E90C012A68C4E927
:104AF0000E0112F00102C4E91233C4E91467A36580
:104B0000C4E9180113D101211B4E084632607160BF
:104B100008F076F8306018B91221184801F0C6FF85
:104B20000123174A174914482B6011F05FFF164BF9
:104B30001A680AB9104A1A6014492046FFF7ACFFF8
:104B4000134B144918702046FFF7A6FF124B134968
:104B500018702046FFF7A0FF114B1249187020462D
:104B6000FFF79AFFFE22104B1870104B20461A7068
:104B7000F8BD00BF58090020E00900209CC40108CE
:104B800000000020614800085C090020D6C401082C
:104B900064090020DEC4010862090020E6C401089F
:104BA00060090020EBC401086309002061090020AE
:104BB00010B5084C2368DB0709D40748FFF778FFD6
:104BC0000123064A06490448236011F00FFF0248FA
:104BD00010BD00BF5409002078090020000000200B
:104BE000414800082DE9F0470E4649680446FFF7A2
:104BF000C3FEC0B2FF2807D071682E4805F01CFC28
:104C000087212D4801F052FFD4E904232B4F9B1A32
:104C10009B107B437E2B03D98A21274801F046FF56
:104C2000D4E904120C25A069531A9B10121A7B4375
:104C300092107A430133934205FB03F80ED84144A6
:104C40006161D4E9043496E80700E31A04E9070037
:104C50001A489B1058430138BDE8F087404605F0DC
:104C600087FC054618B96921154801F01FFFD4E9F2
:104C700004C300274FF00C0AA3EB0C030F4A9B1050
:104C800002FB03F9A9EB0703002B0ADD0AFB07F37C
:104C900005EB030E634493E8070001378EE8070035
:104CA000F0E7604605F04EFC25614544C4E9055532
:104CB000C7E700BF99C30108F9BD0108ABAAAAAABA
:104CC00061C3010838B5D0E901239B1A074A9B103C
:104CD0005343CDB29D42044603D3A621044801F0BC
:104CE000E5FE0C20636800FB053038BDABAAAAAA1C
:104CF000F9BD010838B5CCB2114905460B6813F06F
:104D0000010307D10F4A70201372012310600E486F
:104D10000B605060FF2C10D0D5E904239B1A0B4A7E
:104D20009B1053439C4203D3B221094801F0BEFEBD
:104D30000C23286903FB040038BD0248FCE700BFD0
:104D4000500900206809002079BE0108ABAAAAAA70
:104D5000F9BD010810B5D0E90730C9B2D2B283421B
:104D600009D01C788C4204D15C78944201D19878A7
:104D700010BD0333F3E74FF0FF30F9E72DE9F041C1
:104D8000D0E904239B1A534A9B1053430D460978DC
:104D90000446994203D393214F4801F087FED4E99A
:104DA00001239B1A4B4A9B1053436978994203D3C2
:104DB0009421494801F07AFED4E904239B1A454A1C
:104DC0009B105343A978994205D3FE2903D095211E
:104DD000414801F06BFE6A7829782046FFF7BAFF58
:104DE000C3B2FF2B06462CD03C4805F025FB2978A2
:104DF0002046FFF77FFF697807462046FFF762FFEE
:104E0000314680462046FFF775FF41460246384648
:104E1000FFF704FD29782046FFF76CFF6978064606
:104E20002046FFF74FFFA97807462046FFF762FFAD
:104E3000394602463046FFF7F1FC9C21264801F036
:104E400035FED4E90723234F9B1A7B437E2B03D9DE
:104E50009F21214801F02AFED4E90721606A8B1ABC
:104E60007B43091A4F430133BB4203EB43080AD883
:104E7000424422622A88236A23F8032CAA7803F882
:104E8000012CBDE8F081404605F072FB064618B9DA
:104E90006921134801F00AFED4E907010B1A0D49F4
:104EA00059430023CA1A002A0DDD03EB4302871879
:104EB000B7F800E006EB020C26F802E0BA780133FE
:104EC0008CF80220EEE705F03DFBE6614644C4E9BC
:104ED0000866CFE7ABAAAAAAF9BD01085EBE010821
:104EE00061C3010813B5FF24074B8DF804401B680C
:104EF0000A46186801A908F001F8012814BF2046E5
:104F00009DF8040002B010BD5C09002038B581682E
:104F100000681D46144605F0CDFB0346201845EBFE
:104F2000E37138BD2DE9F0410E681046722E1F4620
:104F300027D0742E08D0632E12D000244FF00045E5
:104F400020462946BDE8F0818B68D3E90023B3F100
:104F5000004F08BF002A19D0841847EB0305EFE77C
:104F6000886805F00FF9002871F1000304460D462A
:104F7000E6DA084805F060FADD21074801F096FD01
:104F8000DEE78868BDE8F041FFF7C0BF14461D4664
:104F9000D6E700BFC0BF0108F9BD01082DE9F04701
:104FA0000F460646FFF7A6FE0024DFF85C90426835
:104FB0000178FFB2124805F03FFAD6E90758454597
:104FC00016D02B78BB4211D169783046FFF77AFEB4
:104FD000016869290AD1D0E9012A484605F02CFA6E
:104FE000DAF8003003B198470134E4B20335E6E75C
:104FF0002146044805F020FA2046BDE8F08700BFAE
:10500000E6BF01082FC001080DC001082DE9F347D4
:1050100007468846FFF76EFE0025426801781B4868
:1050200005F00AFAFC693E6ADFF86890033403363B
:105030005FFA88F8A64220D0234633F8032D9B78E8
:10504000ADF804208DF8063014F8033C984512D1D1
:105050009DF805103846FFF735FE016869290AD129
:10506000D0E9012A484605F0E7F9DAF8043003B13F
:1050700098470135EDB20334DCE72946044805F0D2
:10508000DBF9284602B0BDE8F08700BF4DC001083B
:105090009AC0010876C00108836C73B504460D46BA
:1050A000164623B94FF48C710D4801F0FFFC0D49F1
:1050B000CDE9006423462A460B4808F081FC01280C
:1050C00001460AD0094805F0B7F94FF48F7104483A
:1050D00002B0BDE8704001F0E9BC02B070BD00BF95
:1050E000F9BD01080FC30108B15900081AC301082E
:1050F00038B590F847300446032B0D4604D940F2EA
:105100003111064801F0D2FC94F847305A1C84F85B
:1051100047201C4484F8425038BD00BFF9BD010847
:1051200010B590F84730044623B94FF49B710648F8
:1051300001F0BCFC94F84730013BDBB284F8473007
:105140001C4494F8420010BDF9BD0108CBB2FE2BFF
:1051500037B5054605D1104803B0BDE8304005F02D
:105160006BB9FFF7C7FD016804466D290DD1017ABF
:105170002846FFF7BFFD436800930368D4E9001297
:10518000064805F059F903B030BD4268044803B041
:10519000BDE8304005F050B935C401083DC40108F0
:1051A000A0C1010808B5FFF78DFDBDE80840D0E9B2
:1051B0000012014805F040B9B9C301082DE9F74FC5
:1051C00004462A4805F038F94FF00008284FDFF868
:1051D000B0A0DFF8B090D4E90431C91A891079433E
:1051E0005FFA88F6B14231D9504605F025F92046DC
:1051F0003146FFF7ABFF94F82830DFF88CB0B342AC
:105200000CBF1C48484605F017F9D4E907531A4A61
:10521000AB4218D02978B14213D11046019305F062
:105220000BF969782046FFF7BDFF584605F004F9F1
:10523000A9782046FFF78AFF484605F0FDF8019B54
:105240000D4A0335E4E708F10108C4E7D4E9072370
:105250009B1AD4E90102121A92107B437A43074841
:1052600003B0BDE8F04F05F0E7B800BFC1C30108C7
:10527000ABAAAAAAD9C30108E5C30108F6C301086D
:10528000D0C30108B3F00108F2C301082DE9F843C7
:105290000422054690F84710114805F0CDF8002487
:1052A000DFF848900F4F05F1420695F84730A342CA
:1052B00010DD16F8011B2846FFF71CFDD0F804800E
:1052C00014B1484605F0B8F84146384605F0B4F840
:1052D0000134EAE70448BDE8F84305F0ADB800BF83
:1052E0002AC4010878EE010832C4010828B0010878
:1052F00000232DE9F04FC0E90833884619464FF0E6
:1053000000430446C0E90613C0E90013C0E90213D4
:10531000C0E90413FF2085B0CDE90013DDE90E6775
:1053200084F820005FFA82F9D8E907500390039BC4
:10533000D4E900AB9D4221D02B784B451CD1697834
:105340004046FFF7BFFC32463B4601464046FFF76A
:10535000E9FDDDE90023994208BF90420CD09B454E
:1053600008BF924503D0504571EB0B0304DA6B780C
:10537000C4E9000184F820300335D8E7BBF1004FC1
:1053800008BFBAF1000F05D0BAEB06066BEB0707B2
:10539000C4E90467204605B0BDE8F08FF8B50D46B6
:1053A0000E4B896906464B434FF47A71B3FBF1F11A
:1053B000FFF798FD0446C7B2B06C03681B689847B6
:1053C000C6E90E0104F0B8FF0146054805F034F8BF
:1053D000FF2F0CBF95F820002046F8BD40420F007B
:1053E0003BBE010838B5C36C04460D4643B920489E
:1053F00005F022F829462046BDE83840FFF7CEBF29
:10540000806C1C4903685B699847A06C0368DB6883
:105410009847D5E9020104F08FFF0146164805F0D0
:105420000BF8A06C03689968D5E902238847A06C43
:1054300003681B699847E36C9847A06C0368DB68B6
:105440009847A06C03681B689847C4E90E0104F0F4
:1054500073FF0146094804F0EFFF00212046FFF7E3
:1054600041FDC0B2FE2808BF95F8200038BD00BF3E
:105470004BC401087D48000869C401087CC40108C8
:105480002DE9F84FD1E90689B9F1004F08BFB8F10D
:10549000000F05460C4608D11AB1BDE8F84FFFF7DA
:1054A0007DBFBDE8F84FFFF79DBFB8F1010F79F15F
:1054B00000030CDA58EA090302D0294804F0BCFFC3
:1054C000284804F0B9FF94F82000BDE8F88F12B323
:1054D000254804F0B1FF21462846FFF75FFF94F806
:1054E00020305FFA80F8434536D1D5E90EABD4E9D8
:1054F000002392457BEB03011DDAB2EB0A0063EB5C
:105500000B0104F02FFF0146184804F095FF4FF0FF
:10551000FF084046D9E7D0E91423904579EB03030F
:1055200001DA1348D5E7134804F086FF21462846E0
:10553000FFF758FFD3E7BAEB02066BEB0307022E27
:1055400077F10003E5DB3946304604F00BFF0146F6
:10555000094804F071FFDCE7084804F06DFFD8E764
:1055600025C201084AC2010862C20108BAC2010884
:1055700082C20108A0C20108D9C20108F8C201080C
:105580002DE9F04F8FB004468A46FFF7B3FB03685E
:105590000546702B04D04FF49E716D4801F086FAD9
:1055A000A06C03681B6898475246C4E90C01CDE91A
:1055B0000001214604A8FFF79BFE51462046FFF755
:1055C000EDFC9DF830308346FF2B0AD148B929788D
:1055D00060486A6804F030FF40F247115C4801F00F
:1055E00065FAD4E90C0104F0A7FE01465A4804F01C
:1055F00023FF5946594804F01FFF9DF83010FF293A
:105600007DD1574804F018FF00224FF00043CDE948
:105610000823DDE90423CDE90623DDE90823CDE9EC
:105620000A23A36D13B39847DDE90423D4E91801D5
:10563000B3F1004F08BF002A09D0DDE9082310F1BB
:105640000B0841F10009904579EB03030EDAD4E928
:105650000C321B1841EB0202CDE90A01CDE90632FA
:1056600004F080FE01463F4804F0E6FE4FF00008DB
:105670004FF000492A7A04A92046FFF701FFA36DE5
:10568000834603B198475FFA8BF3FF2B57D1DDE9CF
:105690000432D4E90E01181A62EB0101CDE9063299
:1056A000CDE90801CDE90A0104F05CFE01462E486F
:1056B00004F0C2FEA36D002BDCD0DDE90423D4E9A5
:1056C00018014B4508BF424509D0DDE9082310F118
:1056D0000B0641F10007964277EB0303CADAD4E9DF
:1056E0000E321B1841EB0202CDE90A01CDE9063268
:1056F00004F038FE01461B4804F09EFEBAE720463F
:10570000FFF7E0FAD0E900B2DDE90401039204F00A
:1057100013FE039A03465946144804F08DFED4E95B
:105720000C2304980599801A61EB0301CDE9080167
:1057300004F018FE01460E4804F07EFE69E751466B
:105740002046FFF763FC58460FB0BDE8F08F00BF5E
:10575000F9BD0108B8BE0108EBBE01080ABF010887
:1057600025BF010880BF010898BF01083EBF01089E
:1057700062BF010870B504460D46FFF7BBFA036827
:105780006D2B11D0702B09D0612B0DD1836894F84B
:10579000411094F84000BDE8704018472946204663
:1057A000BDE87040FFF7ECBE40F22B11024801F05B
:1057B0007DF94FF0FF3070BDF9BD01082DE9F74FBD
:1057C00004466B4804F038FE6A4804F035FE6A4827
:1057D00004F032FE674804F02FFE94F82830FF2BC7
:1057E00004D14FF4E371654801F060F994F8281092
:1057F0002046FFF77FFA42680178614804F01CFEFA
:1058000094F82830DFF8A4B1DFF8649184F84630CA
:1058100094F846102046FFF76DFA036880466D2B1A
:105820001BD14168574804F007FE94F84610204603
:10583000FFF75EFC98F80810204684F84610FFF742
:1058400059FA42680178504804F0F6FD2046FFF707
:105850001DFD484604F0F0FDDAE794F846102046B6
:10586000FFF788FFC3B2FF2B06460ED1474804F06E
:10587000E3FD40F2DB11414801F018F940F2DB1181
:10588000434B444A3D4812F0A1FB024694F84610AF
:105890002046FFF75FFAC5B2FF2D0CD13E4804F059
:1058A000CBFD40F2E111354801F000F9384B394A9F
:1058B00040F2E111E6E794F84610FE2D204636D17D
:1058C000FFF72EFC014607462046FFF713FAD8F8EB
:1058D000042098F800108246304804F0ADFD3246AE
:1058E00039462046FFF736FAC5B2FF2D12D13146B0
:1058F0002046FFF7E7F9D0E90012294804F09CFDA3
:1059000040F2ED111D4801F0D1F8214B214A40F23F
:10591000ED11B7E7DAF80410584604F08DFD204683
:10592000FFF7B4FC484604F087FD3946C5E7FFF7AA
:10593000E1F9314607462046FFF7C4F9294680467B
:105940002046FFF7D7F90190164804F075FD164878
:1059500004F072FD019A41463846FEF75FFF94F865
:10596000463084F8416084F8403084F846504FE770
:10597000B3F00108BAC00108D9C00108F9BD010897
:10598000F8C0010816C1010835C101084CC1010861
:10599000A6B30108F3C401086FC1010889C1010859
:1059A000A8C10108FFC1010815C20108E9C1010829
:1059B00008B5FFF7FDF8FFF701FF00002DE9F843F8
:1059C0001F461646FFF77EF9B7F1004F08BF002EBD
:1059D000D0E9005884681AD0742D01D0FEF748FF32
:1059E000D4E9000104F0BEFC39468146304604F09B
:1059F000B9FC4A46034641460A4804F01DFD742D91
:105A000001D0FEF735FFC4E90067BDE8F883742DC7
:105A100001D0FEF72DFFD4E9000104F0A3FC024BF6
:105A20000246E8E787BE0108ACBE0108836C10B5EA
:105A3000044623B940F29721024801F037F8A06CE0
:105A400010BD00BFF9BD0108FF23054A1370054AC8
:105A50001370054A1370054A1370054A1370704796
:105A60006409002062090020600900206309002009
:105A70006109002010B50446006807F0AFFC20461D
:105A800010BD00002DE9F04385B00AF04FFD4FF640
:105A9000FF712E4A2E4C13888B421CBF013313809A
:105AA000FFF786F8FFF7C2FF03681B689847637823
:105AB00006460F46FBB9274BDB88E3B1264AD2E9FD
:105AC0000001B1F1004F08BF00280FD0B04271EBC8
:105AD000070210DA214AB6EB000802FB03F267EB7B
:105AE0000109D317904579EB030304DB1C4804F04C
:105AF000A3FC012363700023ADF80C3063782BB155
:105B000001238DF80C30144BC3E900672378154C42
:105B1000BBB1012514488DF80D5004F08DFC2570A3
:105B20000023124A1249134800931278039B097804
:105B300000680AF039FE30B10F4B187805B0BDE8A7
:105B4000F0832370ECE70D4BF7E700BF2A0A002033
:105B50000C0A0020180A00203000002080510100AB
:105B600030C60108150A002059C601080F0A002096
:105B70000E0A0020080A00206009002062090020A7
:105B80001D4B10B5DB882BB91C4804F055FC1C4B91
:105B9000187810BD1B4BD3E90023B3F1004F08BFA9
:105BA000002A01D01848F0E7184C23780133DBB203
:105BB000032B237001D91648E7E7012B0BD90A21E3
:105BC000002004F077FD134B58434FF47A73B0FB79
:105BD000F3F008F06FFA21780F4804F02DFC002351
:105BE0000E4A13700E4A13700E4A13600E4A137059
:105BF000012353700D4BCBE7180A00206EC6010835
:105C000060090020280000208AC60108400A002000
:105C1000A4C6010840420F00BBC601080F0A0020BD
:105C20000E0A0020080A00200C0A00206309002048
:105C300008B500231A4607F0BDF8431E58425841E4
:105C400008BD000007B50B78012B11D05AB22AB15C
:105C5000022B11D00A4804F0EFFB06E00192094B39
:105C600001A91B681868FFF7E3FF03B05DF804FBA8
:105C70004FF0FF330193F2E7024B04311B68F1E769
:105C800021C70108F80900201FB57023CDE90131B3
:105C9000002301A98DF80C30FEF7A4FF05B05DF8D4
:105CA00004FB00002DE9F04F4A4B85B01A780446FA
:105CB000002A40F08B80012747491F70FEF7ECFE59
:105CC000464B474918702046FEF7E6FEDFF868A10C
:105CD00044498AF800002046FEF7DEFEDFF85C91BA
:105CE0000A22002389F800003F4901A8FEF7D8FDE9
:105CF00001A92046FEF760FE3C4E3D49307020462B
:105D0000FEF7CAFE3B4B3C4918702046FEF7C4FE26
:105D10003A4B3B4918702046FEF7BEFE394B3A49D4
:105D200018702046FEF7B8FE384B394A18703949CA
:105D30002046FAF703FDDFF808B1374A8BF8000078
:105D400036492046FAF7FAFC354905462046FFF762
:105D50009BFF70230193334B804601A92046029399
:105D60008DF80C70FEF73EFF07462F4A2B4612783F
:105D70009BF800102046FAF7ECFC43469AF8002006
:105D800029462046FAF7E5FC3B4699F800202946CB
:105D90002046FAF7DEFC2B46327841462046FAF7D9
:105DA000D8FC2B46327839462046FAF7D2FC1F4AF7
:105DB0002B46127829462046FAF7CBFC1C4B1D4A8D
:105DC0001B78127829462046FAF7C3FC05B0BDE8D7
:105DD000F08F00BF410A0020B4C70108100A00205C
:105DE000BEC70108C9C70108D5C70108F1090020CD
:105DF000E2C70108290A0020F0C70108280A00208C
:105E0000FCC701082C0A002009C801082D0A00203F
:105E1000855A000817C801087966000821C80108DA
:105E200035C8010848C8010860090020630900203E
:105E30006109002064090020140A0020F0090020F4
:105E4000120A002030B5044685B00D46FFF72AFF40
:105E50006D22064B01A91B782046CDE901258DF85E
:105E60000C30FEF7BFFE05B030BD00BF120A0020A7
:105E70002DE9F84F434B04461A68434D12F0010FC9
:105E800079D1FF222A7001221A602046FFF70AFF0B
:105E90003E4A3F492046FAF751FC3E4A28703E49A7
:105EA0002046FAF74BFC3D4F3D4A38703D492046AD
:105EB000FAF744FC3C4E3D4930702046FFF7C2FFE4
:105EC0003B4982462046FFF7DFFE3A49834620469B
:105ED000FFF7DAFE8146384A3B7829782046127867
:105EE000FAF737FC354ADFF8E8803378297820461E
:105EF0001278FAF72EFC337898F80020397820468B
:105F0000FAF727FC2B7898F8002031782046FAF72A
:105F100020FC2B4A5B46397820461278FAF719FCA8
:105F200028493B780A7820465946FAF712FC264A57
:105F30004B46397820461278FAF70BFC21493B781A
:105F40000A7820464946FAF704FC1C4A5346317841
:105F500020461278FAF7FDFB337898F80020514676
:105F60002046FAF7F6FB194A2B781278317820464A
:105F7000FAF7EFFB02E02B78FF2B86D02878BDE8FC
:105F8000F88F00BFEC090020430A00209D63000841
:105F90002DC90108F55F000837C90108110A002062
:105FA000815B000841C90108130A00204BC90108A0
:105FB00057C9010865C90108100A002063090020BB
:105FC000140A0020F1090020620900206009002065
:105FD0006409002070B50D460446FEF7E9FD04494A
:105FE00022462B46BDE870400978FFF7E7BC00BFAA
:105FF000F1090020F7B55E4C2668A6B908200FF01D
:106000009DFE05460660012032466860042106F0C8
:10601000F7FD286018B91221564800F047FD564890
:1060200025600AF099FA554D554F296855480131B8
:10603000296004F001FA0AF079FA3B781BB90123D0
:106040003B700AF09FFA0023019323684E4A01A98E
:10605000186806F053FF012807D04C4804F0ECF90B
:106060004FF4C7714A4800F021FD019E731C51D1C5
:10607000484804F0E1F92B68042B0FD90EF0E6FE36
:1060800003785BB1444804F0D7F94FF47A7008F014
:1060900011F840F299113E4800F008FD00233B70D2
:1060A0002B681E22013BDBB21E2B28BF1E2302FAE7
:1060B00003F33A4A934226D8B3F5616F1E464FF078
:1060C000000722D2B3F5167F77F1000320DA3C2EC9
:1060D00077F10003ACBF1E210A21002004F0EAFA88
:1060E000341847EBE0752946204604F03BF9014699
:1060F0002B4804F0A1F920462946FFF76BFF294BF6
:10610000187803B0F0BD0027244E4FF41671E4E771
:106110003C21E2E74EB13146234804F08DF9019865
:106120000021FFF757FF214BEAE721482E6004F0DA
:1061300083F90AF0B5F9FEF73BFDFFF777FC03683A
:106140001B6898471B4BC3E9000123686BB13046BD
:106150000AF002FA256835B1286807F03FF90821EE
:1061600028460FF00BFE00232360134BC8E700BF47
:10617000F80900209CC40108455C00083C0A002086
:10618000380A002018C50108A08601002BC50108A7
:1061900045C5010891C50108A8C5010800A3020072
:1061A000F5C50108620900200BC60108140A002089
:1061B00020C601082000002064090020054B18704B
:1061C000054B1A700022054B1960054B1A705A7066
:1061D000704700BF0F0A00200E0A0020080A0020A6
:1061E0000C0A002082B0ADF80430064B1870064B44
:1061F0001A70064BBDF804201960054B1A8002B0D6
:10620000704700BF0F0A00200E0A0020080A002075
:106210000C0A002008B50AF0BFFAC0B2DE2828BF79
:10622000DE2008BD4FF47A7337B5002403FB00F27B
:106230000749B2FBF3F20D6801A92868019406F042
:106240005DFE012814BF2046019803B030BD00BF99
:10625000F4090020022818BF00200AF01FBC00002B
:10626000F8B53B4B05461E78002E6FD101271F70F5
:1062700009F018FE374928460EF06EFCC31F052BA7
:10628000354C42D820710E233449284663710EF0F4
:106290006CFC3349074612F063FF00283AD1E060F6
:1062A000304928460EF03EFC2F49607028460EF01B
:1062B00053FCB0F57A7F3AD8E0802C4928460EF09E
:1062C0004BFC42F21073984236D820812849284668
:1062D0000EF028FC2749A07028460EF03DFCB0F5D2
:1062E0007A7F2ED26081244928460EF01BFCE07094
:1062F00036B1224804F0A0F87121214800F0D6FB05
:10630000E068BDE8F840FFF7A5BF1E4804F094F828
:106310003E46B8E71C49384612F022FF10B9022366
:10632000E360BDE7194804F087F80126B8E718488C
:1063300004F082F80126C0E7164804F07DF8012633
:10634000C4E7154804F078F80126CCE7F8BD00BF93
:10635000420A00205CC80108180A002075C801081C
:1063600018C9010898C801089CC80108C3C80108D9
:10637000B4EF0108EBC8010815C901081AC90108E2
:1063800045C501085FC80108FFE001087CC8010895
:10639000A5C80108CCC80108F6C8010870B5234B90
:1063A000C0B21B78984206D10EF050FD0EF0E6FB0D
:1063B0001F4B187870BD1F4D0EF048FDFFF750FFC2
:1063C00095F905000BF0AAFE0AF08CFA28790BF07B
:1063D00073FE0AF07BFA68780AF05AFB164B1A68CB
:1063E0001C4612F0010213D10421144E08463260FB
:1063F000716006F005FC306018B91221104800F0F9
:1064000055FB01230F4A10490C48236010F0EEFAA7
:106410000E4B1A680AB9094A1A600D480AF044FB83
:10642000EB780BB10B4BC4E70B4BC2E7130A002010
:1064300064090020180A0020E8090020300A002022
:106440009CC4010800000020755A0008F4090020CF
:10645000FD650008100A002063090020034B93F833
:106460003230022B0CBF022000207047B000002009
:1064700008B5FFF7F3FF30B90AF036F818B9BDE8F0
:1064800008400AF00DB8FFF7E9FF022806D10AF02C
:106490002BF818B1BDE808400AF048B808BD000064
:1064A000F8B51D4600234171BDF81810044603607D
:1064B000C180174602B115B923712046F8BD0749BE
:1064C00028460FF057FC064610B920712660F4E705
:1064D0002A46394611F0A8FE2571F7E7E0F90108D0
:1064E00010B50446006808B10FF046FC204610BD08
:1064F00070B5364E86B03268044622B94FF4E67164
:10650000334800F0D3FA002C5DD00022314B1A80C2
:10651000D4E91C2313431FD02F4B1D6807F072FCD6
:1065200001462E48A847D4E91C0103F005FF226F5D
:1065300001462B4803F080FFD4E91C2303A803F095
:1065400093FED4E91C23274903A8C1E90023264967
:10655000C1E9002301F06AFAFEF72AFBFFF766FAA9
:1065600003681B689847214B214AC3E90001237A3D
:10657000C3F3C0031370637F2BB3237F1BB31D4989
:1065800008200FF0EDFB054630B163890093237FAF
:10659000A26E617FFFF784FF0395A5B100233068E9
:1065A0001A4603A9006806F04FFB01280BD01248D9
:1065B00003F042FF039C34B12046FFF791FF08210E
:1065C00020460FF0DBFB06B070BD00BFF4090020D1
:1065D00045C501082A0A0020B00000204FC7010865
:1065E0005CC70108280000203000002020000020A7
:1065F0002E0A0020E0F9010889C7010810B50446F9
:10660000FFF776FF24B12046BDE810400CF0F2B849
:1066100010BD000038B542F2107009F0A3FF044627
:10662000124803F009FFECB12578022D16D16068FD
:106630000021FFF7CFFCD4F89800FFF759FF237A29
:106640002BB10B4803F0F8FE00220A4B1A702046CB
:106650000AF072FE032D06D1284638BD032DEAD17B
:106660000020E5E70125FFF703FFF5E7D6C601089F
:10667000F4C60108150A0020002310B5144C84F854
:10668000363009F031FF08B109F050FFFFF7C2FFC3
:10669000032815D8DFE800F005020A080D4803F0CA
:1066A000CBFE0D4B187810BD0C4BFBE7FFF7D6FE69
:1066B000022809BF01230A4B84F83630094BF1E761
:1066C000094840F2BB2100F0F1F94FF0FF30EAE752
:1066D000B000002007C701086409002063090020FA
:1066E000140A0020F009002045C50108FF230021FD
:1066F0000D4A13700D4A13700D4A13700D4A137032
:106700000D4A13700D4A13700D4A13700D4A137021
:106710000D4A13700D4A13700D4A13700D4AC2E9E9
:1067200000111372704700BF120A0020110A0020E6
:10673000130A0020290A0020280A00202D0A002020
:106740002C0A0020100A0020140A0020F009002062
:10675000F1090020FC090020034AC0E900210022C1
:1067600002818272704700BF4849F8F9437A10B538
:1067700004461BB92121094800F098F9207A08B98C
:10678000002010BDA37A002BFBD0606803681B6853
:1067900098470028F4D00023A372F2E774C90108D7
:1067A00030B5044685B08DF80F10FFF7DFFF9DF878
:1067B0000F30606803F00F038DF80F3003685B68DB
:1067C000984768B1002260680DF10F0103680092DC
:1067D000DD6801222378A847606803689B689847B2
:1067E00005B030BD30B50446002585B0FFF7BEFFCB
:1067F00060688DF80F5003685B68984760B1606807
:106800000122036800951D690DF10F016378A84707
:10681000606803689B6898479DF80F0000F00F00C0
:1068200005B030BD7FB504460E46FFF79FFF606898
:1068300003685B689847054620B302226378606866
:106840008DF80C30E37803A98DF80D3003680092C1
:10685000DD680122A378A8470546606815B90123C1
:10686000A3720CE04FF40042036800921D690322FA
:10687000A3783146A84705466068002DEFD003682D
:106880009B689847284604B070BD13B501A904461B
:10689000FFF7C8FF70B19DF80530082B07D19DF8B0
:1068A00004209DF80630134301D101232372207A7E
:1068B00002B010BD2072FAE7002310B50381837285
:1068C0000446406803681B68984730B1012320469E
:1068D0006372BDE81040FFF7D8BF10BD70B5164613
:1068E00005460C46FFF77EFF3EB140EA040128460C
:1068F000BDE87040C9B2FFF753BF20EA0401F6E7D4
:106900002DE9F04742488AB003F096FD07F088FA77
:106910002425079007993F4803F08EFD07986843A8
:1069200003F026FE04463C4803F086FD94B1079927
:106930000DEB0502204607F0E7FD0023DFF8F4A089
:10694000364F07900893089A079B9A421DD320461A
:1069500003F0F8FD06F080F8044606F083F82146BF
:1069600002462F4803F068FD2E4B2F4819889A885D
:106970008B1A03F061FD2D4B1B6803B198472C481F
:1069800003F05AFD0AB0BDE8F087089B05FB0343FE
:106990001B7B013BDBB2032B98BF1AF80320099B3A
:1069A00088BF3F22642B83BF6420B3FBF0F30899B8
:1069B000002382BF05FB01418969B1FBF3F308990C
:1069C0000898DDF820C0DDF820E0DDF82080DDF853
:1069D000209005FB004005FB0949D9F81C6005FB28
:1069E0000141CDE9033605FB08439B69029305FB92
:1069F0000E439B68019305FB0C431B8C00930369BA
:106A00004968384603F018FD089B013308939AE75C
:106A1000B9C90108C5C90108D0C9010805CA0108DA
:106A200049B40108A253002037CA0108BC0A00205B
:106A300032B60108B5C90108014B1860704700BFA4
:106A4000D80A002073B5134C064623780D46124A27
:106A50001BB913780BB172B6FEE701230021137046
:106A60000E48642211F008FC2B4600960C4A642163
:106A70000A4812F0A5FA0B4B1B6803B19847012591
:106A8000064E304603F01CFD72B6074B2570013BE5
:106A9000FDD1F6E7B40A0020480A00204A0A002087
:106AA0006ECA0108D80A0020FFFF0F00F7B5184C86
:106AB000064623780D46174A1BB913780BB172B6F8
:106AC000FEE70123002113701348642211F0D4FB68
:106AD0002B460096114A64210F4812F071FA104BB0
:106AE0001B680BB10C4898470E4B1B6803B19847C5
:106AF0000125094E0C4F304603F0E2FC384603F006
:106B0000DFFC72B64FF0FF332570013BFDD1F2E799
:106B1000B50A0020490A00204A0A002096CA010846
:106B2000440A0020D80A0020A5CA01080368DFF83B
:106B300088C080B5CCF80030164F4368164E3B60D5
:106B40008368164D3360C36815492B600369154A85
:106B50000B604369144C13608369C0692360134B55
:106B60001860DCF800003868306828680968104848
:106B700012680021226864221B6811F07DFB2368E3
:106B80000C4A64210A4812F01BFA094803F098FCE9
:106B9000FEE700BFC80A0020D00A0020D40A002067
:106BA000CC0A0020B00A0020B80A0020C00A002049
:106BB0004A0A00205BCA0108C40A0020074B1B6870
:106BC00003B198471EF0040F0CBFEFF30880EFF3FA
:106BD00009808169004A10472D6B0008D80A0020FF
:106BE000002103E00A4B5B584350043109480A4B2B
:106BF00042189A42F6D3094A02E0002342F8043BC5
:106C0000074B9A42F9D300F00DF8FAF7F5FB7047FD
:106C1000E4FC010800000020E8020020E802002057
:106C200084540020314B82B01A6842F480721A609A
:106C300099682F4A0A409A601A6822F0885222F016
:106C400001121A601A6822F480221A609A6822F4EB
:106C50007D029A600022DA6001921B6813F40073CF
:106C600018BF01230193019B012B37D14FF48051B1
:106C7000204B1A68A3F5806322F00102C3F80024B8
:106C8000D3F8002422F00202C3F80024D3F8002431
:106C900022F00402C3F800245A6A42F080525A6279
:106CA000154A11605168C906FCD49A689A609A68BE
:106CB0009A609A689A605A6822F460425A605A68E8
:106CC00042F440425A609A6822F003029A609A683D
:106CD0009A60064A936813F00C0FFBD14FF00062E4
:106CE000064B9A60064ADA6002B0704700380240EC
:106CF0000CC0FF88003C02400070004000ED00E046
:106D00000003FA0570B5064688B02D4801F00CFC6A
:106D10002C4B1A680092009A91073AD501214FF442
:106D2000007001F05BFE012001F04CFC264A536824
:106D300043F400335360A2F5374253681B07FCD578
:106D40000024012502A801F029FC02A91C48069490
:106D50008DF81C50ADF80C4001F0FAFB2A460623D2
:106D60003146174801F03AFC2946154801F021FC4C
:106D70000221134801F0C4FC114801F0B3FC134D8B
:106D800001940F4C0221204601F0B4FC58B108B028
:106D900070BD1A6842F001021A60009A9207BDD4D1
:106DA0001A680092F9E7019B01330193019BB3F547
:106DB000805FE7DB38212846FFF778FEE2E700BF77
:106DC000002401400038024000270140C1CA0108E8
:106DD00008B5002001F0F6FB0021074801F0E9FBAF
:106DE00000214FF4007001F0F9FD044A136823F00C
:106DF0000103136008BD00BF0024014000380240B9
:106E000013B5072301220146114801F0E7FB0221D7
:106E10000F4801F075FC0E4801F064FC00230D4C96
:106E2000019302210A4801F065FC28B1084802B02C
:106E3000BDE8104001F05BBC019B01330193019B55
:106E4000B3F5805FEDDB4C212046FFF72FFEE8E72E
:106E500000240140C1CA010870B506460825FFF7A5
:106E600051FF00243046FFF7CBFF013D0444F9D128
:106E7000FFF7AEFFC4F3CF0070BD000000000000BC
:106E800008B51120FFF7E8FF10F082FC0146084822
:106E900010F08AFD10F064F803A3D3E9002310F08A
:106EA000B7F810F06FFB08BD2FDD24068195F33F86
:106EB00000F07F450F4A536A43F0805353620E4BF4
:106EC0001A465968C906FCD41B68022823F4C0532B
:106ED00006D143F4C05313605368DB06FCD47047FB
:106EE000012802D143F48053F5E70028F3D143F49D
:106EF0000063F0E7003802400070004010B50C4B12
:106F00005A68D206FCD41C6814F4C05F0BD114F488
:106F100080500AD114F4006404D106482A21FFF7F6
:106F2000C5FD204610BD0220FCE70120FAE700BFA6
:106F30000070004007CB010838B50546012001F07C
:106F4000EFFB022D01BF144A136843F001031360E5
:106F5000124B1A6842F480721A601A689205FCD5C6
:106F60005A6822F4604242F440425A6000229A6019
:106F70000A4B9C6814F00C04FBD14FF480721A6029
:106F8000074B084A28461A60FFF794FF2046BDE8E1
:106F9000384001F0B9BB00BF003C0240003802405D
:106FA00038000020D0FE3F000C4B5A6B900513D4E4
:106FB0005A6A42F080525A62094A116841F480715B
:106FC0001160596B41F480715963596B8905FCD587
:106FD000136823F480731360704700BF00380240C9
:106FE00000700040054B5A6B910706D45A6B42F073
:106FF00001025A635A6B9207FCD570470038024071
:10700000094B5A6A42F020025A629A6942F0200201
:107010009A619A6922F020029A610022A3F509334D
:107020001A801A855A6270470038024015210022E2
:1070300002384143064B1A85D962012199825A626E
:107040001A8219801A8AD207FCD500221A8070474A
:1070500000140040002349F6FE7282B00193019BA8
:10706000934201DD02B07047019B01330193F6E7C3
:10707000002340F6FE7282B00193019B934201DD32
:1070800002B07047019B01330193F6E7002382B001
:107090000193019BB3F5CC7F01DD02B07047019BEA
:1070A0000133F5E7D0B1012801D1FFF7EFBF0C4B59
:1070B00000211A684FF47A73B2FBF3F2094B013ADC
:1070C00092B21A8501220138D8629A8259621982D5
:1070D0001A801A8AD207FCD500221A80704700BF96
:1070E000380000200014004000F1774303F57803D6
:1070F000B3F5804F2DE9F04106460C4617462DD2D8
:1071000002F1F73303F608030344B3F5804F25D2A9
:10711000FFF7F4FE804610B10020FFF7CBFE01F030
:1071200017FB01252744361BA7420AD101F020FB9B
:10713000B8F1000F02D04046FFF7BCFE2846BDE87C
:10714000F08141F6027001F01BFB301914F8011BAD
:1071500001F072FB042818BF0025E5E70025EDE7E4
:1071600010B50C4600F1774101F57801B1F5804F7B
:107170000DD202F1F73303F608030344B3F5804F51
:1071800005D20146204611F04FF8012010BD002025
:10719000FCE7000008B5114B984215D003F5806359
:1071A000984213D003F58063984211D003F58063B1
:1071B00098420FD003F5006398420DD0084B094A5E
:1071C0001421094810F002FF002008BD0120FCE74F
:1071D0000220FAE70320F8E70520F6E70000024066
:1071E00096CB010850CB0108AFCB01080F2808B59A
:1071F00005D9094B094A3B21094810F0E7FE012354
:1072000003FA00F0C043074A516801405160136817
:107210001840106008BD00BFF8CB01085ACB010828
:10722000AFCB0108000401400F292DE9F84F824639
:107230000D4693461F4605D95A4B5B4A54215B487D
:1072400010F0C4FE4FF0010909FA05F900F0B8F892
:107250006FEA0903564E032D7268564C02EA030288
:107260007260326803EA0203534A3360136A43F0E0
:10727000010313622ED80F22A3684FEA850802FA91
:1072800008F223EA0203A3605046FFF783FFA368D6
:1072900000FA08F01843A0601BF0020F18BFB36893
:1072A000464A1CBF43EA0903B3601BF0040F1EBF2C
:1072B000F36843EA0903F360336843EA0903336080
:1072C0003B01DBB2002D45D182F806334023136029
:1072D000BDE8F88F072D13D80F22A5F10408E36845
:1072E0004FEA880802FA08F223EA0203E3605046F4
:1072F000FFF750FFE36800FA08F01843E060CBE7BF
:107300000B2D13D80F22A5F1080823694FEA88082E
:1073100002FA08F223EA020323615046FFF73AFF1C
:10732000236900FA08F018432061B5E70F22A5F1A0
:107330000C0863694FEA880802FA08F223EA02039C
:1073400063615046FFF726FF636900FA08F01843AF
:107350006061A1E7012D03D182F807338023B6E7EE
:10736000022D04D182F808334FF48073AFE7032D68
:1073700004D182F809334FF40073A8E7042D04D137
:1073800082F80A334FF48063A1E7092D04D882F80C
:1073900017334FF400039AE782F828334FF48073D1
:1073A000536095E704CC010875CB0108AFCB010809
:1073B00000040140000001400038024000E100E00C
:1073C000144B984205D1144AD36943F00103D361A9
:1073D0007047124B984204D10F4AD36943F002031D
:1073E000F5E70F4B984204D10B4AD36943F00403ED
:1073F000EDE70C4B984204D1074AD36943F00803E8
:10740000E5E7094B9842E3D1034AD36943F02003EF
:10741000DDE700BF000002400038024000040240E7
:1074200000080240000C02400014024003234900FF
:1074300010B584688B4024EA030484600124022A86
:1074400004FA01F407D0032A0DD0012A07D183687A
:107450002343836003E083688A401A438260836821
:107460001C43846010BD82681343F2E70F29F8B50E
:1074700004460F4615461E4603D94D211948FFF70D
:1074800015FB2046FFF79CFF03237A009340DB4364
:107490002168194021600121D4F800C001FA02F0EE
:1074A0004CEA000CB940C4F800C009B266B1A68825
:1074B000314389B2A180E168012D03EA0103E36051
:1074C00006D0022D08D0F8BDA68826EA0101F1E712
:1074D000E3680343E360F6E7E36805FA02F21A4360
:1074E000E260F0E754CC01080F2970B505460C4660
:1074F000164603D96D210E48FFF7D8FA2846FFF744
:107500005FFF032361008B40DB43EA68012E02EA40
:107510000302EA6005D0022E03D02A6813402B60D4
:1075200070BDEA6806FA01F11143E960F5E700BFB2
:1075300054CC01080F2910B505D9074B074A832100
:10754000074810F043FDFFF73BFF4B0003210268A3
:1075500099401143016010BDF8CB010810CC01081F
:1075600054CC01080F2938B50446154605D98921A0
:107570001B4B1C4A1C4810F029FD0F2A03D91B4B3A
:10758000184A8A21F6E7FFF71BFF07294FF00F0380
:1075900018D8006A8A00934020EA03032362236A12
:1075A00005FA02F21A4322620322236849008A4044
:1075B00023EA020323600223226803FA01F1114344
:1075C000216038BDA1F10802406A9200934020EA90
:1075D00003036362636A95401D436562E4E700BF8D
:1075E000F8CB010823CC010854CC010841CC010898
:1075F000012303FA01F189B201837047012303FAE1
:1076000001F189B241837047012303FA01F189B284
:107610000AB10183704741837047008A084100F036
:10762000010070470F2938B505460C4603D9B6212D
:107630000548FFF73BFA28686400E04000F00300CB
:10764000431E5842584138BD54CC0108808A084135
:10765000C04300F00100704710B5074C236853B9D0
:10766000012005F095FB206028B9BDE810403621C7
:107670000248FFF71BBA10BDDC0A00209BCC0108B2
:1076800010B50B4C22681AB93C210A48FFF70EFAD4
:10769000206842F2107105F0C3FC01280CBF0124E0
:1076A000002403D040210348FFF700FA204610BD14
:1076B000DC0A00209BCC010810B5074C22681AB9DF
:1076C00051210648FFF7F2F9002320681A46BDE869
:1076D0001040194605F0B8BADC0A00209BCC01081E
:1076E00010B50446FFF7B8FFFFF7CAFF2146102286
:1076F000034801F077FE0446FFF7DEFF204610BD89
:107700000054004010B5FFF7A7FFFFF7B9FF01F0E5
:1077100021FE0446FFF7D0FF204610BD08B51346F2
:107720000A460146034801F043FA003018BF012021
:1077300008BD00BF0054004008B513460A46014684
:10774000034801F03BFB003018BF012008BD00BF1B
:107750000054004008B513460A460146034801F0AC
:107760000BFC003018BF012008BD00BF00540040D2
:1077700008B513460A460146034801F08FFC003065
:1077800018BF012008BD00BF0054004008B51346D3
:107790000A460146034801F0DBFC003018BF012017
:1077A00008BD00BF005400400123064A83405169D0
:1077B000194205D05361044B53F8203003B11847E8
:1077C000704700BF00040140E00A00200F2838B5D0
:1077D00004460D4603D926210348FFF767F9034BFA
:1077E00043F8245038BD00BFE1CC0108E00A002076
:1077F0000020FFF7D9BF0120FFF7D6BF0220FFF717
:10780000D3BF0320FFF7D0BF0420FFF7CDBF08B5DB
:107810000920FFF7C9FF0820FFF7C6FF0720FFF781
:10782000C3FF0620FFF7C0FFBDE808400520FFF7B3
:10783000BBBF08B50F20FFF7B7FF0E20FFF7B4FF5F
:107840000D20FFF7B1FF0C20FFF7AEFF0B20FFF775
:10785000ABFFBDE808400A20FFF7A6BFFEE7FEE742
:10786000FEE7FEE7FEE7FEE7FEE7FEE7FEE7FEE7F0
:10787000FEE7FEE7FEE7FEE7FEE7FEE7FEE7FEE7E0
:10788000FEE7FEE7FEE7FEE7FEE7FEE7FEE7FEE7D0
:10789000FEE7FEE7FEE7FEE7FEE7FEE7FEE7FEE7C0
:1078A000FEE7FEE7FEE7FEE7FEE7FEE70A23B0FBA2
:1078B000F3F203FB120040EA0210C0B2704700006E
:1078C000CA22024B5A6253225A6270470028004073
:1078D000014B1860704700BF200B00204FF40032AE
:1078E0000F4B10B50F4C5A61E368DB0503D4302110
:1078F0000D48FFF7DBF8FFF7E3FF4FF40072A368D2
:1079000023F48853A360094BC3F88420FF236362E8
:10791000074B1B6813B1BDE81040184710BD00BFEE
:10792000000401400028004027CD010800E100E0EC
:10793000200B00202DE9FF479A46364B80461B78E6
:1079400091469DF830709DF834602BB9324B334A24
:107950008C21334810F03AFB431E1E2B58D80C29BB
:1079600056D8A2F5FA63632B52D8BAF1170F4FD845
:107970003B2F4DD83B2E4BD802F13000C0B2FFF761
:1079800095FF05460846FFF791FF000240EA0545CE
:107990004046FFF78BFF05435046FFF787FF04463D
:1079A0003846FFF783FF000240EA04443046FFF701
:1079B0007DFF20431B4CFFF783FFE36845F4005530
:1079C00043F08003E360E3685B06FCD565602060FC
:1079D000E36823F08003E360124BDA689206FCD57B
:1079E000FF2201A85A628DF807808DF80810ADF8C3
:1079F00009908DF806A08DF805708DF8046002F0EE
:107A000058FC094BC3E90001012004B0BDE8F08730
:107A10000020FAE7240B0020A0CD010894CD010836
:107A200027CD010800280040280B002007B5037867
:107A30000193437800938378B0F805200179C078EA
:107A4000FFF778FF03B05DF804FB000038B52B4B5F
:107A500004461B781BB9E4212948FFF727F8294A77
:107A6000D36823F02003D360D3689B06FCD513684A
:107A70005268C2F30741080900EB800001F00F01D2
:107A800001EB4001C9B201F5FA61A4F80510C2F397
:107A90000721C1F300108500284401F00F0101EB1C
:107AA0004001D2B22171C2F3011101EB810102F058
:107AB0000F0202EB4102E270C3F30742C2F301116D
:107AC00001EB810102F00F0202EB4102A270C3F34D
:107AD0000722C2F3021101EB810102F00F0202EB57
:107AE0004102DBB26270C3F3021202EB820203F0C6
:107AF0000F0303EB4203237038BD00BF240B0020AB
:107B000027CD0108002800401FB501A8FFF79EFF00
:107B100001A802F0CEFB05B05DF804FB08B5FFF745
:107B200043FA1B4A136843F480731360FFF7C8FEDF
:107B3000184A536B23F4403343F482035363164BC8
:107B4000DA6842F08002DA60DA685106FCD5FF227A
:107B50001A611A6942F4FE021A619A6822F0400220
:107B60009A609A6822F44C529A60DA6822F0800295
:107B7000DA60094BDA689206FCD5FF225A620122CC
:107B8000064B1A70FFF7C0FF054BC3E9000108BDA3
:107B9000007000400038024000280040240B002004
:107BA000280B002008B5094B1B7823B940F21F11A0
:107BB0000748FEF77BFFFFF783FE064B9A6822F427
:107BC00080729A60FF225A6208BD00BF240B002019
:107BD00027CD01080028004008B5144B1B7833B9A5
:107BE000134B144A40F22711134810F0EFF9FFF736
:107BF00067FE124BDA6822F48072DA60104A9168EC
:107C000041F400319160116841F400311160F021BC
:107C10000C4A82F829134FF4007151609A6842F4BB
:107C200088529A60FF225A6208BD00BF240B0020D0
:107C3000A0CD01086DCD010827CD01080028004026
:107C40000004014000E100E0F8B51E46194B17465C
:107C50001B7833B9184B194A4FF4A571184810F026
:107C6000B5F9184CFFF72CFEA56825F48075A560C2
:107C7000E56825F48075E560FFF718FE05460846BF
:107C8000FFF714FE000440EA05613846FFF70EFED8
:107C900005463046FFF70AFE084340EA0520E36840
:107CA000DB07FCD5FF23E0616362BDE8F840FFF726
:107CB00093BF00BF240B0020A0CD010882CD010896
:107CC00027CD010800280040037842788178C078E9
:107CD000FFF7BABF38B50D46044604F0BBFC194A9D
:107CE000136823F00103136004F0D4FC25B1164A95
:107CF000536843F00603536072B6BFF34F8FBFF370
:107D00006F8F124A0120136823F0030343F40073BA
:107D100043F00103136000F00FFD0D4B1A6942F0B0
:107D200004021A6130BF1A69022022F004021A61AB
:107D3000FFF702F9034A136843F00103136004B12B
:107D400062B638BD10E000E0002004E000700040A2
:107D500000ED00E062B6704700220E4B10B51A70BD
:107D60000D4A0E4C1388204623F040031B041B0CC5
:107D700013800D210222FFF7B7FB204602220E21BD
:107D8000FFF7B2FB2046BDE8104002220F21FFF7AB
:107D9000ABBB00BF300B00200038004000040240A5
:107DA000294A38B5136A054643F480531362052205
:107DB00026480C461146FFF7D5FB0522062123482D
:107DC000FFF7D0FB052207212048FFF7CBFBC5B109
:107DD000022205211D48FFF729FB022206211B482C
:107DE000FFF724FB022207211848FFF71FFB012C95
:107DF0001BD144F451740122154B1C80154B1A7091
:107E000038BD2A4605211148FFF710FB2A460621F6
:107E10000E48FFF70BFB2A4607210C48FFF706FB2D
:107E2000012C09D144F45974E5E7022CE1D0032C6C
:107E30000CBF03240024DCE7022CF3D0032C14BF76
:107E400000240324EEE700BF003802400000024097
:107E500000300140310B002000220E4B10B51A708B
:107E60000D4A0E4C1388204623F040031B041B0CC4
:107E7000138005210222FFF737FB2046022206214C
:107E8000FFF732FB2046BDE8104002220721FFF732
:107E90002BBB00BF310B002000300140000002402E
:107EA000064B074A988111781A461889C00701D4F1
:107EB0000029FAD19089C0B2704700BF003001405C
:107EC000310B0020054AD36823F4E0631B041B0C2C
:107ED00043F0BF6343F40033D360704700ED00E02C
:107EE00020220021114B10B5C3F88420104B114CF7
:107EF0001A6A204642F480421A625A6942F4804269
:107F00005A615A6922F480425A610B4A91811A6A75
:107F1000092122F480421A620222FFF7E5FA204684
:107F2000BDE8104002220A21FFF7DEBA00E100E0BE
:107F300000380240000002400038014010B50B4CF0
:107F400040F22551204600F00CFE48B1204600F0DA
:107F5000E6FD074B1B683BB1BDE81040C0B21847B7
:107F6000A388044ADBB2137010BD00BF0038014083
:107F7000340B0020A053002010B50446802108488F
:107F800000F0E9FD0028F9D02146054800F0C3FDC6
:107F9000034C4021204600F0DEFD0028F9D010BD42
:107FA0000038014010B5441E14F8010F00B910BD8F
:107FB000FFF7E2FFF8E7000008B5024800F0AFFD68
:107FC000C0B208BD003801402DE9F0410F46012143
:107FD0004FF4C066804688B0084614461D4600F03F
:107FE000EFFC01214FF4804000F0F8FC3B4B02A96C
:107FF0003B48CDE9026300F045FC072209213848DF
:1080000000F082FC07220A21354800F07DFC452F54
:10801000CDF810803AD14FF48063ADF81830072CBA
:1080200040D10023ADF81430052D4CD14FF48053CE
:10803000ADF816300023ADF81C300C2304A92948F4
:10804000ADF81A3000F00CFD274B1A6802B101227E
:1080500040F22551234800F066FD0121214800F03F
:108060004FFDFFF7A9FF25238DF804309DF8383028
:108070008DF805304FF48073ADF80630FFF722FF1E
:1080800001A800F035FA08B0BDE8F0814F2F02D109
:10809000ADF81860C3E70023072CADF818300DD1F8
:1080A000592107E0082C02D14FF48053BAE7092C7C
:1080B000BAD154210D48FEF7F9FCB5E7082CB0D031
:1080C000092CB1D1F0E70F2D02D14FF44053AFE7A7
:1080D000022D0CBF4FF400530023A9E70202000158
:1080E0000000024000380140340B0020A9CD0108F7
:1080F0000E2307B5082200934E210123FFF764FFEA
:1081000003B05DF804FB0000402200210D4B0E4837
:10811000C3F884200D4B5A6A42F400325A629A69BD
:1081200042F400329A619A6922F400329A61084A54
:1081300091815A6A032122F400325A620222FFF727
:10814000D3B900BF00E100E0000002400038024067
:108150000044004008B5024800F0E1FCC0B208BD90
:10816000004400402DE9F0471F46262388B08DF8D3
:10817000043000239DF8408089461446ADF806304F
:1081800082469DF844509DF848608DF80580FFF7C1
:1081900099FE01A800F0ACF90121084600F010FC9E
:1081A00001214FF4003000F027FC65B10821504B4D
:1081B0005048CDE9021302A900F064FB0722032115
:1081C0004C4800F0A1FB66B10422494B02A9494882
:1081D000CDE9022300F056FB07220221454800F0BA
:1081E00093FBB9F1450FCDF810A041D14FF4806356
:1081F000072CADF8183049D10023ADF81430052F05
:1082000055D14FF480530024ADF81630ADF81C4022
:10821000002E57D1ADF81A6075B1BDF81A3043F091
:108220000403ADF81A30344B1A6802B1012240F24F
:108230002551324800F077FC04A9304800F010FCCA
:1082400001212E4800F05CFC0DB1FFF783FF2623CF
:108250008DF804304FF480738DF80580ADF806304A
:10826000FFF730FE01A800F043F908B0BDE8F08741
:10827000B9F14F0F02D14FF4C063B9E70023072CC7
:10828000ADF818300ED14FF4827107E0082C02D1FE
:108290004FF48053B1E7092CB1D1FF211848FEF704
:1082A00005FCACE7082CA7D0092CA8D1F0E70F2FCC
:1082B00002D14FF44053A6E7022F0CBF4FF40053F6
:1082C0000023A0E70823224640F227710B48ADF8AF
:1082D0001A3000F028FC40F22661084800F060FCEB
:1082E000224640F22661054800F01DFC94E700BFDD
:1082F0000203000100000240380B0020004400404F
:10830000A9CD0108F8B505460024134E134F80216E
:10831000134800F020FC68B12946114800F0FBFB2F
:1083200000240F4D0C4E0D4F4021284600F013FC49
:1083300048B1F8BD0134B442E9D94FF4A4713846CC
:10834000FEF7B4FBE3E70134B442EDD940F251113A
:108350003846FEF7ABFBE7E7FFFF0F00A9CD0108AA
:108360000044004008B5064B0246186000B10122E7
:1083700040F22551034800F0D6FB012008BD00BFA4
:10838000380B00200044004070B5134C40F22551DA
:10839000204600F0E6FBC0B1104B1D6825B1204619
:1083A00000F0BDFBC0B2A84740F226610A4800F0C9
:1083B000D8FB78B140F22661074800F0F1FB084B8A
:1083C0001B683BB1BDE870401847A388054ADBB283
:1083D0001370E9E770BD00BF00440040380B002077
:1083E0003C0B0020A0530020BFF34F8F0449054BE6
:1083F000CA6802F4E0621343CB60BFF34F8FFEE71D
:1084000000ED00E00400FA0510B5441EE3B2052BB0
:1084100003D90E211148FEF749FBFEF7E3FD45F2B3
:1084200055520F4B1A60DA68D207FCD4052C06D8D7
:10843000DFE804F0030A0C0E101201225A604CF619
:10844000CC42074B1A6010BD0222F7E70322F5E782
:108450000422F3E70522F1E70622EFE77ACE0108CE
:108460000030004010B5194C23683BB95F2000F084
:10847000DFFA28B1164B236000F0EAFA206810BD3D
:108480005E2000F0D5FA08B1124BF4E75D2000F051
:10849000CFFA08B1104BEEE75C2000F0C9FA08B142
:1084A0000E4BE8E75B2000F0C3FA08B10C4BE2E7A3
:1084B0005A2000F0BDFA08B10A4BDCE7592000F061
:1084C000B7FA08B1084BD6E7084BD4E7400B0020B9
:1084D000F0CD010800CE010816CE010831CE01080A
:1084E00040CE01084FCE010868CE010872CE0108C7
:1084F00030B5012403780A4D03F01F029440C2787E
:10850000590952B1074A2B44D26842781201D2B2BB
:1085100083F8002345F8214030BD2031FAE700BF41
:1085200000E100E000ED00E008B5084B98420BD1F7
:1085300001214FF4007000F06DFABDE80840002101
:108540004FF4007000F066BA08BD00BF002401407F
:1085500043680A7923F0407323F4807343EA0223CB
:108560000A6810B513434360D1E9032313438A68B3
:1085700084681343084A224013434A7943EA42037A
:1085800083600A7D036B013A23F0F873D2B243EAA9
:108590000253036310BD00BFFDF7FFC000234FF07F
:1085A0004072036083808360C0E903230123037565
:1085B0007047836819B143F001038360704723F06B
:1085C0000103FAE7044B5A6818B142F400025A60FA
:1085D000704722F40002FAE7002701401D2970B518
:1085E0001BD90725A1F11E06C46D06EB4606B54052
:1085F00024EA050403FA06F62643C665062A38D897
:108600001F24013A036C02EB8202944023EA040324
:1086100001FA02F21A43026470BD13290DD907262C
:10862000A1F11405C46805EB4505AE4024EA060433
:1086300003FA05F52543C560E0E709290DD90726AA
:10864000A1F10A04056904EB4404A64025EA0605E5
:1086500003FA04F42C430461D0E70726446901EBD4
:108660004105AE4024EA060403FA05F626434661B6
:10867000C4E70C2A0CD81F24073AC36B02EB820212
:10868000944023EA040301FA02F21A43C263C3E7E7
:10869000122A0CD81F240D3A836B02EB82029440FD
:1086A00023EA040301FA02F21A438263B4E7182AA8
:1086B0000CD81F24133A436B02EB8202944023EA46
:1086C000040301FA02F21A434263A5E71F24193A90
:1086D000036B02EB8202944023EA040391401943A6
:1086E000016399E7836843F0804383607047806D3E
:1086F00080B270470368194214BF01200020704700
:10870000C943016070470000044B1A6818B142F079
:1087100002021A60704722F00202FAE7003C0240AF
:10872000044B1A6818B142F004021A60704722F034
:108730000402FAE7003C0240044B1A6818B142F008
:1087400008021A60704722F00802FAE7003C024073
:10875000044B5A68D20741BF034ADA60034ADA6021
:10876000704700BF003C0240EFCDAB890504030217
:10877000024A536843F0010353607047003C0240D3
:10878000014B9861704700BF003C0240084B9A695A
:10879000D10709D49A69D20508D49B6913F4F05F14
:1087A00014BF032004207047012070470220704747
:1087B000003C0240042313B504468DF80730FFF750
:1087C000E5FF8DF807009DF80730012B0AD11CB991
:1087D00005238DF8073007E0FFF7D8FF013C8DF83F
:1087E0000700F0E7002CF3D09DF8070002B010BDA1
:1087F00010B504464FF40040FFF7DCFF042804BF27
:108800000023236010BD000038B504464FF400403B
:108810000D46FFF7CFFF04280BD1064A4FF4004066
:10882000536823F4807353602560BDE83840FFF738
:10883000C1BF38BD003C024038B504464FF400408B
:108840000D46FFF7B7FF04281BD135B125704FF453
:108850000040BDE83840FFF7ADBFFF2324F003051B
:1088600004F003042968E40003FA04F421EA040490
:108870002846FFF7BDFF21462846BDE83840FFF7F0
:10888000C3BF38BD2DE9F0430022012703250E6840
:1088900007FA02F333EA060431D14FEA420C05FA33
:1088A0000CF4E44391F804E0D0F800900EFA0CF8D0
:1088B00004EA09090EF1FF3E48EA0908BEF1010F7A
:1088C000C0F8008011D8D0F808E004EA0E0E4C7908
:1088D00004FA0CF444EA0E048460848824EA030455
:1088E0008B7993409BB223438380C36805FA0CF4D1
:1088F00023EA0404CB7903FA0CF32343C360013267
:10890000102AC5D1BDE8F08310B50F2401F007038C
:10891000C90800EB8100016A9B009C4021EA040128
:108920000162016A9A400A43026210BD204B10B5F1
:108930009A6802F00C020C2A30D8DFE802F02F2FE0
:108940002F2F072F2F2F072F2F2F2000194B184ABB
:10895000036093681849C3F30313CC5C0368E340D6
:1089600043609468C4F302240C5D23FA04F4846029
:108970009268C2F3C2228A5CD340C36010BD99687A
:108980000E4CC1F383419A68615C9B68094BC2F34A
:1089900081524B430132B3FBF2F3D8E74FF400426C
:1089A0005B68C3F34233013302FA03F3CFE700BF3E
:1089B000003802400024F4003C0000204C0000205D
:1089C000054B19B1D9690143D9617047DA6922EAC7
:1089D0000002DA61704700BF00380240054B19B150
:1089E000196A0143196270471A6A22EA00021A6280
:1089F000704700BF00380240054B19B1596A014366
:108A0000596270475A6A22EA00025A62704700BFF0
:108A100000380240054B19B159690143596170474B
:108A20005A6922EA00025A61704700BF00380240CA
:108A30004309012B054B00F01F000CBF1B685B6B4B
:108A400023FA00F000F00100704700BF0038024038
:108A5000024A536B43F080735363704700380240FF
:108A600030B50D460446028AEB8892B222F4405299
:108A70001A43898902828389288923F4B052AB88FA
:108A800022F00C020343688985B003431343A3819A
:108A9000A38A68469BB223F440730B43A382FFF77B
:108AA00045FFDDE90213154A944208BF1946192310
:108AB000A2894B43296810044CBF49008900B3FBCD
:108AC000F1F16425B1FBF5F3A2891801120405FB4D
:108AD00013130BD5DA003232B2FBF5F202F00702C3
:108AE00042EA00039BB2238105B030BD1B01323343
:108AF000B3FBF5F303F00F030343F3E70038014042
:108B0000838919B143F400538381704723F40053E0
:108B10001B041B0CF8E7C1F30801818070478088B3
:108B2000C0F30800704701F01F0310B5C1F34214F1
:108B30000121012C01FA03F105D10C3003683AB18F
:108B40001943016010BD022C0CBF10301430F5E742
:108B500023EA0101F5E70388194214BF0120002030
:108B600070470123C1F3421210B5012A01F01F041E
:108B700003FA04F30DD182891340028892B26BB1DB
:108B80000123090A03FA01F10A4214BF1846002022
:108B900010BD022A0CBF028A828AEDE71846F7E769
:108BA0000123090A8B40DB439BB20380704700001E
:108BB0002DE9F3411F46002304460E460193154656
:108BC0001AB9012002B0BDE8F08140F6FF730193AD
:108BD0004FF40031204600F05EFD002852D1012103
:108BE000204600F028FD4FF2FF71204600F03CFDCA
:108BF0000121204600F009FD40F6FF73DFF8B8813F
:108C000001934146204600F03BFD002841D0394603
:108C10000122204600F01AFD40F6FF73614F0193D8
:108C20003946204600F037FD002838D0012D42D1CA
:108C30000021204600F0FFFC03F00CFD29462046F1
:108C4000238B00F0EDFC03F025FD40F6FF73564D3D
:108C500001932946204600F01EFD30B3204600F067
:108C600000FD307040F6FF73504D019329462046B9
:108C700000F011FD0028A4D0019B5A1E0192002B88
:108C8000F4D104E0019B5A1E0192002BA0D10020D8
:108C900098E7019B5A1E0192002BB2D1F7E7019B86
:108CA0005A1E0192002BBBD1F1E7019B5A1E019283
:108CB000002BCED1EBE7022D25D103F0CBFC4FF4F6
:108CC0000061204600F0D0FC0021204600F0B3FCFB
:108CD000238B03F0DFFC40F6FF73354D01932946EB
:108CE000204600F0D8FC40B10121204600F098FC5D
:108CF000238A3370238A7370B4E7019B5A1E019252
:108D0000002BECD1C3E740F6FF77033D238BDFF860
:108D1000A0803544AE4201972CD1254E31462046E5
:108D200000F0B9FC90B30021204600F084FC03F071
:108D300091FC204600F095FC01212870204600F0AF
:108D40006FFC03F0A7FC204600F08BFC40F6FF739D
:108D5000184E687001933146204600F091FCD8B15E
:108D6000204600F07EFCA8707CE7019B5A1E019211
:108D7000002B8CD04146204600F08DFC0028F4D01A
:108D8000204600F06EFC06F8010BC3E7019B5A1E5B
:108D90000192002BC2D17AE7019B5A1E0192002B4F
:108DA000D9D174E70200001040000010100000103C
:108DB0000400001040000300010003002DE9F3410E
:108DC0001D460023019340F6FF7304460E461746E6
:108DD0000193002A00F082804FF40031204600F019
:108DE0005AFC002843D10121204600F00EFC40F639
:108DF000FF73DFF8808101934146204600F040FC7C
:108E000000283DD029460022204600F01FFC40F6F5
:108E1000FF73544D01932946204600F031FC002891
:108E200034D03546204615F8011B3E4400F017FCAF
:108E300040F6FF77DFF83081B542019731D14A4DD6
:108E40002946204600F027FC002836D02046012184
:108E500000F0E6FB40F6FF73444D454C0193294674
:108E6000204600F018FC00282DD1012005E0019BD0
:108E70005A1E0192002BAFD1002002B0BDE8F08154
:108E8000019B5A1E0192002BB6D1F5E7019B5A1E99
:108E90000192002BBFD1EFE7019B5A1E0192002BDC
:108EA000EAD04146204600F0F6FB0028F4D015F841
:108EB000011B204600F0D3FBBEE7019B5A1E019226
:108EC000002BBDD1D8E7019B5A1E0192002BC6D1C1
:108ED000D2E7019B5A1E0192002BCDD04FF40031F6
:108EE000204600F0D8FB0028F3D10121204600F0F5
:108EF0008CFB40F6FF731F4E01933146204600F075
:108F0000BFFB10B329460022204600F09FFB40F62D
:108F1000FF73144D01932946204600F0B1FBD0B1F8
:108F20002046012100F07CFB40F6FF730F4D104CF2
:108F300001932946204600F0AEFB002895D0019B06
:108F40005A1E0192002BF4D196E7019B5A1E019202
:108F5000002BD2D190E7019B5A1E0192002BDAD14F
:108F60008AE700BF82000700040000101000001014
:108F700000540040010003002DE9F3411D46002389
:108F800004460E46019317461AB9012002B0BDE807
:108F9000F08140F6FF7301934FF40031204600F05A
:108FA0007AFB002838D10121204600F02EFB40F644
:108FB000FF73DFF8E48001934146204600F060FB38
:108FC000002843D029460022204600F03FFB40F60F
:108FD000FF732D4D01932946204600F051FB0028D8
:108FE0003AD03546204615F8011B3E4400F037FBC9
:108FF00040F6FF77DFF89480B542019737D1234DD3
:109000002946204600F047FB0028BED1019B5A1E8E
:109010000192002BF4D104E0019B5A1E0192002B17
:10902000BAD12046012100F0FBFA40F6FF73184D3B
:10903000184C01932946204600F02DFB20B1019BDE
:109040005A1E0192002BF5D100209FE7019B5A1E6A
:109050000192002BB0D1E4E7019B5A1E0192002B34
:10906000B9D1DEE7019B5A1E0192002BD9D04146AF
:10907000204600F010FB0028F4D015F8011B204614
:1090800000F0EDFAB8E700BF82000700040000100E
:1090900010000010005400400100030000232DE9DF
:1090A000F3410E464FF4003104461746019300F099
:1090B000F2FA18B9002002B0BDE8F0810FB9012022
:1090C000F9E73546204615F8011B3E4400F0C7FA83
:1090D00040F6FF77DFF86C80B54201971FD1194D3C
:1090E0002946204600F0D7FA28B32046012100F097
:1090F00097FA40F6FF73144D144C0193294620460D
:1091000000F0C9FA0028DAD0019B5A1E0192002B08
:10911000F4D1CFE7019B5A1E0192002BCAD04146E1
:10912000204600F0B8FA0028F4D015F8011B2046BC
:1091300000F095FAD0E7019B5A1E0192002BCFD187
:10914000B8E700BF040000101000001000540040F9
:109150002DE9F3411F46002304460E4601931546B0
:109160001AB9012002B0BDE8F0814FF4003100F0DF
:1091700092FA08B90020F5E70121204600F05BFAD9
:109180004FF2FF71204600F06FFA0121204600F0F7
:109190003CFA40F6FF73DFF8B88101934146204660
:1091A00000F06EFA00283AD039460122204600F03D
:1091B0004DFA40F6FF73614F01933946204600F0A7
:1091C0006AFA002831D0012D3BD10021204600F061
:1091D00032FA03F03FFA29462046238B00F020FAAA
:1091E00003F058FA40F6FF73554D01932946204687
:1091F00000F051FAF8B1204600F033FA307040F632
:10920000FF73504D01932946204600F044FA002890
:10921000A7D0019B5A1E0192002BF4D1AAE7019B13
:109220005A1E0192002BB9D1A4E7019B5A1E01924C
:10923000002BC2D19EE7019B5A1E0192002BD5D173
:1092400098E7022D29D14FF40061204600F00CFA76
:1092500003F000FA00212046238B00F0ECF903F024
:1092600019FA40F6FF73384D01932946204600F065
:1092700012FA60B103F0EEF90121204600F0D0F9B6
:10928000238A3370238A737003F004FAB7E7019BD3
:109290005A1E0192002BE8D16CE740F6FF77033DA0
:1092A000238BDFF8A4803544AE4201972DD1264EA2
:1092B0003146204600F0EFF998B30021204600F037
:1092C000BAF903F0C7F9204600F0CBF90121287064
:1092D000204600F0A5F903F0DDF9204600F0C1F9C1
:1092E00040F6FF73194E687001933146204600F036
:1092F000C7F9E0B1204600F0B4F9A8707FE7019B00
:109300005A1E0192002B3FF435AF4146204600F033
:10931000C2F90028F3D0204600F0A3F906F8010BAB
:10932000C2E7019B5A1E0192002BC1D122E7019B8B
:109330005A1E0192002BD8D11CE700BF020000107A
:109340004000001010000010040000104000030056
:109350000100030038B5204B08219A691F4842F4E8
:1093600000129A619A6922F400129A615A6A22F4F0
:1093700000125A62FEF73CF9012308211A461748E9
:10938000FEF774F8092115480122FEF7ADF809210E
:109390001248FEF742F9D8B1012038BD082128460D
:1093A000FEF726F9FDF772FE08212846FEF726F99A
:1093B000FDF76CFE013CF1D109210848FEF72DF9BB
:1093C00020B94FF4BD710648FDF770FB2046E4E775
:1093D0003324024DEEE700BF003802400004024093
:1093E000C5CE01082DE9FF41444B054698420E4683
:1093F00017467CD103F5F2335A6A082142F4001271
:109400005A629A693E4842F400129A619A6922F4BB
:1094100000129A61FEF7ECF8012308211A46384839
:10942000FEF724F8092136480122FEF75DF80921EC
:109430003348FEF7F2F8002855D0012308211A46D8
:109440002F48FEF713F8042208212D48FEF78AF86A
:10945000012309211A462A48FEF708F804220921A7
:109460002748FEF77FF8274B9A6942F400129A6169
:109470009A6922F400129A61684600F0ADF8224B16
:10948000694601934FF48063ADF80A304FF480438E
:109490002846ADF80C30ADF80870009600F038F8AA
:1094A0002846012100F0A6F8012019E008214046D5
:1094B000FEF79EF8FDF7EAFD08214046FEF79EF80C
:1094C000FDF7E4FD013CF1D109210D48FEF7A5F8B7
:1094D0000028B2D10D484FF4D171FDF7E7FA2046CC
:1094E00004B0BDE8F0813324DFF81480EAE740F2ED
:1094F000B1110648FDF7DAFABEE700BF005400409C
:1095000000040240003802400000FFBFC5CE010841
:109510007FB50446868868460D46FFF707FA029A2B
:109520002B4926F03F06B2FBF1F13604360C88B227
:109530000643A6802388274E23F001031B041B0C3F
:1095400023802B68B3421ED85B00B2FBF3F39BB2BF
:10955000042B38BF0423013080B22084A3832388E6
:10956000AA8843F0010323802388698923F4816357
:109570000A4323F00203134323802A89AB89134350
:10958000238104B070BD4BF6FF70EE8886421BBF8E
:109590001920434303EB4303B2FBF3F30BBFB2FBCE
:1095A000F3F39BB29BB243F48043C3F30B020AB9BB
:1095B00043F001034FF496724A434FF47A71B2FBC1
:1095C000F1F2013292B243F400432284C6E700BFB5
:1095D00040420F00A086010041F28832044BC0E9EE
:1095E0000023002383604FF480438381704700BFD2
:1095F0000000FFBF038819B143F0010303807047E7
:1096000023F001031B041B0CF8E7038819B143F492
:1096100080730380704723F480731B041B0CF8E7EE
:10962000038819B143F400730380704723F4007377
:109630001B041B0CF8E7038819B143F48063038013
:10964000704723F480631B041B0CF8E722B141F040
:10965000010189B20182704701F0FE01F9E7018240
:109660007047008AC0B270470388B1F5006F1BBF16
:1096700023F400631B0443F400631B0C0380704756
:10968000838A008B43EA00430B4023F07F435B1A3D
:10969000584258417047002382B0009301930B0F4A
:1096A00001900093009B21F07F4153B1019B143343
:1096B0000193019B1B680B4214BF0120002002B0E4
:1096C0007047019B090C1833F2E7F8B50E460546C2
:1096D00080B14F1C384600F04BFF044640B13A467B
:1096E00000210EF0C9FD3246294620460EF09CFDB1
:1096F0002046F8BD0446FBE738B50D46044628B1C0
:109700000FF040FD23462044834201D1002038BDA4
:1097100013F8012BAA42F7D10120F8E773B50546EB
:109720000E4600240EF07EFC2246046001A9284665
:109730000FF03CFE05460EF075FC0368222B0BD0A3
:10974000019B1B7843B9A542ADBF284620460123A3
:109750002346336002B070BD01232046F9E70000C4
:109760002DE9F04F05464FF0010B002687B0CDE9FB
:10977000031206F10903122B8CBF0320022000F014
:10978000F7FE0090E8B1324636490FF04DFC039BDE
:1097900053F82690EDB90024009800F0D3FEBBF1F9
:1097A000000F02D1284600F0CDFE84B1049B0136A3
:1097B000B34225464FF0000BDBD1204607B0BDE891
:1097C000F08FBBF1000F02D1284600F0BBFE002451
:1097D000F3E7254B4FF00008B9F1000F08BF994699
:1097E00048460FF0CFFC019000980FF0CBFC0290A0
:1097F000284649460FF0F3FCB8B928460FF0C2FCE2
:10980000DDE9012301309B1A08FB030000F0B0FEE4
:1098100004460028BFD003462F4618F1FF3809D26E
:10982000394618460FF0A6FCB6E7019B08F101087F
:109830001844DEE74946384605930FF0D0FC059BF7
:10984000A0EB070A5246394618460FF0B5FC0099BE
:1098500050440FF08FFC019A029B9244C318574466
:10986000DBE700BF82AF0108B4F0010830B580B17A
:109870000346021F00F1180452F8045F8D4208D01D
:10988000A242F9D11C301A4614680433013401D1C4
:10989000116030BD8342F6D1FBE7000068B1084992
:1098A000431E13F8010F00B970470A5C02F003026F
:1098B000022A08BF20381870F3E70120704700BF64
:1098C0001EFA010870B5044680B1064600EB81051A
:1098D000AE4204D12046BDE8704000F033BE56F8D9
:1098E000040B0028F4D000F02DFEF1E770BD00005D
:1098F0002DE9F74F8B460092002839D00027C35D31
:1099000093BB1D46064600EB070A024638485245FF
:1099100038D103B10135002D63D00137384600F04E
:1099200027FE804600285AD03A4600210EF0A4FCBB
:10993000A80000F01DFE0446002854D04FF0000996
:109940000021B2452CD131B14046FFF7BEFE0028C0
:1099500049D044F82900404600F0F4FD009B1D600A
:10996000204603B0BDE8F08F0137B7F5807FC6D140
:1099700000242546204600242946FFF7A3FF009B2C
:109980001C60EDE712F8011B594504D1002BBED035
:1099900001350023BBE7095C090758BF0133B6E76F
:1099A00016F8013B5B4512D10029CAD04046FFF7AB
:1099B0008CFEC0B109F1010344F829003A460021A8
:1099C000404601930EF058FC019B9946B8E7084ABF
:1099D000985C02075CBF08F801300131B1E704462A
:1099E000C8E72C46BCE7404600F0ACFDC2E700BF2C
:1099F0001EFA01082DE9F74300250646082088468F
:109A000091461F46009500F0B3FD0446002865D03E
:109A1000C0E9005530460FF0B5FB01280FD133786F
:109A20002A2B0CD109F1FF33C4F80080636022684F
:109A30004A4502D263684B4540D3294B0DE02D21A6
:109A40003046FFF759FE0546B8B9019001A93046E6
:109A5000FFF764FE019B63B1224B3B6000992846EF
:109A6000FFF730FF002C35D0204600F06BFD0024BE
:109A700030E0C4E900001D46D9E76A462D21304692
:109A8000FFF736FF009B0546013B012B01D9164B22
:109A9000E3E7002301A900680193FFF73FFE206080
:109AA000019B0BB1114BD8E701A96868FFF736FE9F
:109AB0006060019B002BBAD00D4BCEE7424501D32D
:109AC000434501D20B4BC8E700992846FFF7FAFE41
:109AD00000233B60204603B0BDE8F0830546BDE7A8
:109AE000E8CF010862CF010881CF0108AACF0108A1
:109AF000C9CF010808D0010808B520B34A1C22D0FC
:109B0000062920D8DFE801F0040D101316191C00F7
:109B1000002303600EF092FC0840431C5842584159
:109B200008BD00234360F5E700238360F2E70023CC
:109B30008361EFE70123C360ECE700230361E9E7FA
:109B400000234361E6E70120EAE770B506460D1FF2
:109B500001F1180455F8041F4B1C03D1A542F9D19B
:109B6000002070BD3046FFF7C7FF0028F6D0F8E7A9
:109B700000290B46B8BFCB1D4A4202F0070201F094
:109B8000070158BF51420122C3F3C703C9B202FA09
:109B900001F1C25C1143C154704700290B46B8BFA4
:109BA000CB1D4A4202F0070201F0070158BF5142A3
:109BB0000122C3F3C703C9B28A40C15C21EA020192
:109BC000C15470470B460029B8BFCB1DC3F3C70370
:109BD000C05C4B4203F0070301F0070158BF594234
:109BE000C9B2084100F0010070472DE9F047089E16
:109BF0008A4690461D46DDF82890074610B1144667
:109C0000A24507D875B9012200240B9B1A60204693
:109C1000BDE8F08721463846FFF7D4FF00285ED123
:109C20000134EDE7099B023B042B04D8DFE803F085
:109C3000282C2C3034006B6801336B6028460EF002
:109C4000FDFB013108BFB0F1FF3FDCD031462846B3
:109C5000FFF752FF0028D6D117B3044621463846F5
:109C6000FFF7B0FF00283FD10134A245F6D10446EA
:109C7000013E042E16D8DFE806F0282A2C2E3000EC
:109C8000AB680133AB60D9E7EB680133EB60D5E734
:109C90002B6901332B61D1E76B6901336B61CDE730
:109CA0003C46E5E72C6028460EF0C8FB013108BFB2
:109CB000B0F1FF3FA7D0B9F1000FA4D04946284624
:109CC000FFF743FF0028A2D09DE76C60EBE7AC6094
:109CD000E9E7AC61E7E7EC60E5E72C61E3E7A04585
:109CE00095D0002DC4D18EE7A045C1D18FE72DE9D5
:109CF000F04F4FF000098BB006461C200C469046F2
:109D0000CDF8249000F034FC0546002800F0E080F7
:109D10001C2000F02DFC0746002800F0D9804B469F
:109D20004FF0FF3245F8232047F823200133072B5B
:109D3000F8D100230121D4F800A00DF12409CDE9C8
:109D40000031CDE902793C21234652463046FFF7E7
:109D50004CFF0999002940F08E80824502D12846A7
:109D6000FFF784FD02234FF0010AD4F804B0CDE9D7
:109D700000A3CDE9025923465A463C2106F10800CA
:109D8000FFF733FF099B002B75D183456BD15146FB
:109D90002846FFF76BFD03234FF0020AD4F808B002
:109DA000CDE900A3CDE9025923465A46182106F110
:109DB0001000FFF71AFF099B002B5CD1834565D18A
:109DC00051462846FFF752FD40F26F1BA3690593E9
:109DD000E368049306F114030693DDF810A006F17E
:109DE0001303079351460698FFF7ECFE20B105993F
:109DF0000798FFF7E7FE88B9BBF1010B0ED0E368C7
:109E000020460133E3600EF019FB013108BFB0F1C9
:109E1000FF3F44D101234FF0000A0993099B53BB34
:109E2000049B534544D104212846FFF71FFD052319
:109E30000622D4F810A0CDE90032CDE9025923461C
:109E400052460C2106F11800FFF7CFFE099B93B98B
:109E5000824510D06369A3EB0803042B31D94FF07E
:109E6000FF33099307E0424621463046FFF73FFFA4
:109E7000099000288FD0284600F064FB17B13846BF
:109E800000F060FB09980BB0BDE8F08F4246214618
:109E90003046FFF72CFF0990002895D0EBE7A36927
:109EA00029462046D4F80CA00593FFF74EFE99E70B
:109EB000424621463046FFF71AFF09900028B6D0E7
:109EC000D9E7424621463046FFF711FF0990D2E715
:109ED0004FF0FF330993002DD4D00027CBE70000CB
:109EE0002DE9F04F002487B0894692462C2103AA21
:109EF0009846109D0394FFF7FBFC074688B93E4B3C
:109F00002B6003993846FFF7DDFC07B0BDE8F08F02
:109F1000D0F800B072685A451CD2304600F012FBEF
:109F20000134039BA342ECD957F824602F2130461B
:109F3000FFF7E2FBA8B92B46304642465146FFF7F1
:109F400059FD2B680646002BE2D00028D9D000F03E
:109F5000F9FAD6E759464846FFF70AFE0BF1010B1E
:109F6000D8E700232F21304604AA0493FFF7C0FC52
:109F7000049906464B1E012B04D9204B2B60FFF79A
:109F8000A1FCBEE742462B4651460068FFF732FD72
:109F90002A6883462AB108B100F0D4FA0499304601
:109FA000EDE72D213068FFF7A7FB18B908F1FF3264
:109FB000CBF80420002305A970680593FFF7AEFBDA
:109FC000059A00901AB10E4A58462A60E4E7DBF879
:109FD0000020DBF80410914205D230460499FFF7C7
:109FE00071FC58469AE7114648460192FFF7C0FDBA
:109FF000DDE900321A44ECE72DD001083FD001081A
:10A0000064D001082DE9FF4100230E460393144656
:10A0100002B902AC236048B90546564B2360039948
:10A020002846FFF74FFC04B0BDE8F08103AA2021C9
:10A03000FFF75EFC039B0546062B02D04E4B2360C8
:10A04000EDE71A22002130460EF016F900940022A6
:10A050003C2331462868FFF743FF2268002ADED1FF
:10A0600000943C2306F108016868FFF739FF226875
:10A07000002AD4D10094182306F11001A868FFF734
:10A080002FFF2368002BCAD16869FFF707FC07225E
:10A090003A496869FFF764FB80460FF073F80128BE
:10A0A00006F1130706D198F800303F2B04BF2A238E
:10A0B00088F8003000220823394640460094FFF714
:10A0C0000FFF404600F03EFA2268002AA7D1072180
:10A0D0003846FFF777FD30B111463846FFF748FDA7
:10A0E0000721FFF75AFDEF6806F1140838460FF014
:10A0F00049F8012804D13B783F2B04BF2A233B7049
:10A1000020230022414638460094FFF7E9FE002153
:10A110004046FFF742FD2368002B80D12F69384667
:10A12000FFF7BCFB00287FF47AAF38460D221449B4
:10A13000FFF716FB074600283FF471AF183600946E
:10A140000D2301223146FFF7CBFE384600F0FAF925
:10A15000012421463046FFF735FD30B1611E3046FF
:10A16000FFF706FD2146FFF718FD01340D2CF0D155
:10A1700055E700BF0CCF010824CF0108580000208C
:10A1800074000020F0B58DB0CDE90023054628B954
:10A190004FF0FF304FF0FF310DB0F0BD2422002111
:10A1A00003A80EF069F803A968460DF065FF0446A0
:10A1B0000028EDD00EF042F94A1C08BFB0F1FF3F75
:10A1C00006460F46E4D0626921462846FFF78FFD18
:10A1D0000028DDD120460EF031F94B1C08BFB0F14C
:10A1E000FF3FD5D08F4208BF864203D020460EF0F5
:10A1F00025F9D1E723682046013323600EF01EF9CC
:10A20000013108BFB0F1FF3FC2D062692146284644
:10A21000FFF76DFD0028E9D0BAE770B53C258AB09C
:10A22000DDE90E64019496FBF5F405FB14640294D9
:10A23000182493FBF4F505FB1433CDE903300C200F
:10A24000013991FBF0F300FB131305930023CDE9D3
:10A2500007339DF84030A2F26C7201A80692099370
:10A260000EF0ECF80AB070BDF7B504466846CDE9CB
:10A2700000230DF0EFFE0269037A551C426990F845
:10A2800004C0077B02F26C71067EC2690068A3708D
:10A290000033207018BF01232046013284F801C02A
:10A2A000E7702571A4F80510E6712272637203B09D
:10A2B000F0BD1FB5437A029303780193437800936E
:10A2C0008378B0F805200179C078FFF7A6FF05B0C4
:10A2D0005DF804FB904271EB0303B4BF0120002042
:10A2E00070470000032210B5104986B00B78013387
:10A2F000B3FBF2F202EB42029B1A0D4A0B7052F8CA
:10A30000234003780B4A049343781A2103938378FC
:10A310000293C378019303790093B0F80530204687
:10A320000EF04EFE204606B010BD00BF920B00207E
:10A3300010D10108D3D00108B1F1004F08BF0028A7
:10A340001FB502460B4608D001A8FFF78DFF01A8F4
:10A35000FFF7C8FF05B05DF804FB0148FAE700BF4E
:10A3600005D101082DE9FF4703220D462B4900289E
:10A370000B78044603F10103B3FBF2F202EB420255
:10A38000A3EB0203264A0B7052F8236075F1000319
:10A390003EDA4FF0010A444265EB4505214A0023AD
:10A3A000204629460DF058FC1E4A07460023204649
:10A3B00029460DF051FC104619464FF46162002306
:10A3C0000DF04AFC4FF46162804600232046294686
:10A3D0000DF042FC104619463C2200230DF03CFCD7
:10A3E0003C2281460023204629460DF035FCCDF85D
:10A3F0000080CDE901923B46BAF1000F0BD00A4A2A
:10A400001A2130460EF0DCFD304604B0BDE8F0877E
:10A410004FF0000AC2E7054AF2E700BF920B0020A6
:10A4200010D1010880510100F1D00108F2D00108DB
:10A430000FB404B0704700000FB437B51B4C25684B
:10A4400055B903222946012002F0DAFB2B462A46A1
:10A450002946206002F0F8FB154D2A68013A0332C4
:10A460001ED86421206802F0DBFD80220021114803
:10A470000DF002FF07AB069A80210E4801930FF002
:10A4800003FA7F2803DD0C490C480EF073FE2B689D
:10A4900008489847002320681A46194602F0D4FB62
:10A4A00003B0BDE8304004B0704700BF1C0C002072
:10A4B000940B00209C0B002088B40108170C00208E
:10A4C0000FB410B50D4CA2B02268013A033210D877
:10A4D00025AB249A802102A801930FF0D5F97F289B
:10A4E00004DD07490DF183000EF044FE236802A845
:10A4F000984722B0BDE8104004B07047980B002088
:10A5000088B4010870B50446054E4518AC4200D128
:10A5100070BD14F8011B3046FFF78EFFF6E700BF51
:10A520001CD1010838B50C461546FFF785FF2046BB
:10A530002946FFF7E7FFBDE838400148FFF77CBF39
:10A54000B3F0010810B5044670B102F0A9F9204635
:10A5500002F048FA02F07EF8BDE81040034A938802
:10A560000133938002F096B810BD00BFA2530020C3
:10A5700070B5214C8AB0226806460132632A2260F7
:10A580001E4D0BDD04F020F80523002201A903F085
:10A590004FFF03F037FC00232860236003F032FCF8
:10A5A0002B6803F57A73984204D903F02BFC00233F
:10A5B00028602360124A134C13781BB92360636030
:10A5C0000123137002F06CF9304602F07FF9054662
:10A5D00068B1324600210DF04FFE02F03BF82388AF
:10A5E0000133238002F056F828460AB070BD638814
:10A5F00001336380F8E700BF240C0020280C002002
:10A60000200C0020A2530020006800BA7047008888
:10A6100040BA80B2704700687047837842781B0464
:10A62000007843EA02231843704700887047FFF719
:10A63000F2BF0B0E03700B0C43700B0A8370C170DA
:10A64000042070470B0A03704170022070470B0A08
:10A65000017043700B0C090E8370C17004207047A9
:10A66000A0F14103052B02D83738C0B27047A0F1E2
:10A670006103052B01D85738F7E73038C0B20A28F4
:10A6800028BFFF207047002210B5441E21B114F8E6
:10A69000010F08B1002A01DA104610BDFFF7E0FFF4
:10A6A00001390F28C9B202D840EA0212EEE74FF092
:10A6B000FF32F1E738B505460C460EF035FC611B5C
:10A6C000013190FBF1F303FB1100284438BD007801
:10A6D000013070470FB404B0704700002DE9FF4708
:10A6E0000F460021254D03AE80469246286832462B
:10A6F0009946039102F0D6FD0128039B31D13BB16D
:10A700004FF080521E4B1A60BFF34F8FBFF36F8F15
:10A71000B7F5C87F88BF4FF4C87741463A46194815
:10A720000DF082FD184C174B31462868A780236036
:10A73000A4F806A084F8089002F096FB039B3BB1B6
:10A740004FF080520E4B1A60BFF34F8FBFF36F8FE5
:10A750000E480096002301220421006804F0F6F858
:10A76000039B3BB14FF08052054B1A60BFF34F8FF4
:10A77000BFF36F8F04B0BDE8F08700BF300E00203C
:10A7800004ED00E0940C0020880C0020380E00201E
:10A790000348002301220221006804F06DB800BFC5
:10A7A000380E00201FB500230B4A4021107003AA69
:10A7B0000A48009200680122039304F0C7F8039B43
:10A7C0003BB14FF08052064B1A60BFF34F8FBFF37F
:10A7D0006F8F05B05DF804FB780C0020380E002068
:10A7E00004ED00E01FB5002303AA0A48009280216F
:10A7F00001220068039304F0A9F8039B3BB14FF0DA
:10A800008052054B1A60BFF34F8FBFF36F8F05B0B7
:10A810005DF804FB380E002004ED00E01FB50F4B7F
:10A820001C680346A0B1002303AA0092082101225C
:10A830002046039304F08AF8039B3BB14FF080520B
:10A84000074B1A60BFF34F8FBFF36F8F04B010BD7B
:10A8500001220821204604F00FF8F7E7380E002007
:10A8600004ED00E01FB503AA00920122002309486D
:10A8700011460068039304F069F8039B3BB14FF065
:10A880008052054B1A60BFF34F8FBFF36F8F05B037
:10A890005DF804FB380E002004ED00E01FB5002336
:10A8A00003AA0A480092102101220068039304F0D1
:10A8B0004DF8039B3BB14FF08052054B1A60BFF33C
:10A8C0004F8FBFF36F8F05B05DF804FB380E00208B
:10A8D00004ED00E000487047700C0020114810B5EE
:10A8E000002303224FF48071006803F0C5FF4FF08E
:10A8F00080520D4B1A60BFF34F8FBFF36F8F0B4C1D
:10A90000206802F01BFD40B1BDE81040002308485C
:10A910001A461946006802F097B9012003F0CAFBF5
:10A92000EEE700BF380E002004ED00E0340E0020FA
:10A930002C0E0020F8B5104B0146186802F070FB91
:10A940000446B8B14FF080560C4F0D4D0023032242
:10A950004FF40071386803F08FFF2E60BFF34F8F04
:10A96000BFF36F8F386803F0C3F92E60BFF34F8FCA
:10A97000BFF36F8F2046F8BD2C0E0020380E00204C
:10A9800004ED00E0014B1860704700BF240E00206A
:10A9900070B5044678B10378032B0CD1436853B1EA
:10A9A0000025054E1868F26990476068F3690560F4
:10A9B00098476560257070BD4C0C002010B50D489F
:10A9C0000D4C002305222146006802F03DF90128C4
:10A9D00005D10A4B1B6863B1BDE810401847084B0E
:10A9E000217808485B6998472046BDE81040FFF78A
:10A9F000CFBF10BD280E00207C0C0020240E0020AC
:10AA00004C0C002022D101087FB50024094E002201
:10AA100001A9306802F072FA651C30B9064BE1B248
:10AA20005B690648984704B070BD01A8FFF7B0FF06
:10AA30002C46ECE7280E00204C0C002049D10108E0
:10AA4000014B1868704700BF280E002010B504465F
:10AA5000064B010AA3F84A00202000F091FBE1B266
:10AA60002120BDE8104000F08BBB00BFAC5300209C
:10AA700008B5FFF7EBFF0122014B83F8522008BD18
:10AA8000AC530020002238B50B4B05461D2083F83F
:10AA90004E100C4683F84C2000F0CAFB20F0060054
:10AAA00040EA4401C9B21D2000F06AFB2946BDE816
:10AAB0003840232000F064BBAC53002013B5164C83
:10AAC0000120A3689847002341F6FE720093009B83
:10AAD000934218DDA36802209847002341F6FE72D6
:10AAE0000193019B934212DD0C4BB5211C6C40205D
:10AAF000A047A0214120A04700210120234602B009
:10AB0000BDE810401847009B01330093DFE7019B2D
:10AB100001330193E5E700BF4C0C002080D401080D
:10AB2000094B07B51B6CC2213B209847002341F617
:10AB3000FE720193019B934202DD03B05DF804FBBA
:10AB4000019B01330193F5E780D401089048914BB4
:10AB50002DE9F04F0360904B904F8360904B914CE8
:10AB60004360914B85B0C360904B914D0361914B15
:10AB7000DFF874A28361904BDFF87092C3613B6889
:10AB8000984763698D489847002328681A461946F4
:10AB900002F05AF8DFF858B29AF8040068B94FF09A
:10ABA000FF33194603AA03F023FE68B9666903F070
:10ABB000FBFC01468248B047EEE741F2883303AA26
:10ABC0004FF0FF310020EEE7039BDA0516D500F0C9
:10ABD00097FA002000F0E8FDFB6A9847FFF714FFA2
:10ABE0006369784898470023D9F800001A46194647
:10ABF00002F02AF8002003F0D5FACDE79B0510D526
:10AC000000F07EFAFFF78CFFFB6A9847FFF7FCFE27
:10AC100063696D4898476421D9F8000002F000FA92
:10AC2000BAE7D9F8000002F089FB012803D1636973
:10AC300066489847B0E7DBF8003023B940F23B1193
:10AC40006348FBF733FF039B1E0604D50722614BC5
:10AC50001A70FFF7B3FE039B580752D500212868EE
:10AC600002F0DEF901284CD1A3690C209847064672
:10AC700088B963690C2158489847334632463146B3
:10AC8000286801F0E1FF002886D14FF4A8715048F0
:10AC9000FBF70CFF80E7DFF85C81A369B8F80400DC
:10ACA00098470346A0B9B8F80410019062694B4870
:10ACB0009047E26930469047019B28681A4619463A
:10ACC00001F0C2FF00287FF467AF4FF4AC71DEE7FC
:10ACD00008F1040203CA33607060B1601846D8F806
:10ACE0000010B8F804200DF09FFA0322394B1A70B7
:10ACF0005E60FFF763FE002328681A46194601F0DC
:10AD0000A3FF039BD90709D50123324E33700023DB
:10AD1000736003F077F8B060FFF750FE039BDB062B
:10AD200006D505222B4B1A7000225A60FFF746FE0B
:10AD3000039B1E0706D50422264B1A7000225A6078
:10AD4000FFF73CFE039B980706D50222214B1A70A1
:10AD500000225A60FFF732FE039B990606D50622B1
:10AD60001C4B1A701E4A5A60FFF728FE039B5B06B5
:10AD70007FF512AF1B4B1B78002B14BF0822092252
:10AD8000144B1A7000225A60FFF718FE04E700BF48
:10AD90002C0C002065A80008DDA6000880D401085E
:10ADA00091A700084C0C00201DA800089DA80008D1
:10ADB000300E0020A5A70008E5A7000843D301082E
:10ADC00059D3010877D301089FD30108B6D30108EE
:10ADD000CCD301087C0C002010D4010846D4010813
:10ADE000790C0020780C0020700C0020340E00201C
:10ADF000280E0020880C0020044B10B55B69984792
:10AE00000446FFF75BFE204610BD00BF80D401085A
:10AE1000F0B56B4C064625460F460FCE0FC596E89B
:10AE20000F0085E80F0097E803006369654E013B5A
:10AE3000033388BF644B85B088BF6361636886E86D
:10AE40000300013B033307D96048636998474FF417
:10AE500023715F48FBF72AFE2368013B033307D9C0
:10AE60005C48636998474FF424715948FBF71EFE0C
:10AE7000A368013B033307D95748636998474FF4E8
:10AE800025715348FBF712FEE368013B033307D9F2
:10AE90005248636998474FF426714D48FBF706FE08
:10AEA0002369013B033307D94D48636998474FF441
:10AEB00027714748FBF7FAFDE369013B033304D9E7
:10AEC0004FF428714248FBF7F1FDA369013B0333BE
:10AED00004D94FF429713E48FBF7E8FD414B0FCBF5
:10AEE0008DE80F0094E80F0000F0E0F82368984721
:10AEF000FFF7E4FD3C4B42205B6C9847222801465B
:10AF0000636931D13948984703220021012001F0BB
:10AF100077FE374B1860012001F03AFF354B18607F
:10AF200020B940F2BF212A48FBF7C0FD012001F003
:10AF30002FFF314D286020B940F2C3212448FBF790
:10AF4000B5FD4FF0FF31286802F06AF800220C21AD
:10AF5000032001F055FE294B186078B96369284831
:10AF6000984740F2C92103E02648984740F2B621AD
:10AF70001748FBF79BFD002005B0F0BD224B234A8C
:10AF80001A6033680BB904233360214B1D680DB17F
:10AF90000120F1E701933368FA2200931D49012350
:10AFA0001D4802F00DFD0128F2D063691B48984747
:10AFB000074840F2DB21FBF779FD2846DCE700BFBC
:10AFC0004C0C0020700C0020D5A600087AD1010896
:10AFD000CCD30108BBD10108F2D101082AD2010863
:10AFE00063D201085C0C002080D401089FD20108C4
:10AFF000300E00202C0E0020340E0020280E0020E1
:10B00000D1D20108B6D201086C0C0020CFA60008EE
:10B01000380E002005D301084DAB00080DD3010800
:10B0200070B5084C054622680E4622B940F2EB2165
:10B030000548FBF73BFD236831462846BDE87040D4
:10B04000184700BF6C0C0020CCD3010800F048B8B2
:10B05000034B0344034883428CBF00200120704708
:10B060000071BDCCFF6789090120704708B5FFF763
:10B0700031FC4379002B0CBF8020002008BD00006C
:10B08000094B0022194610B51C68844202D89C68FE
:10B09000844205D80132152A03F10803F4D1FEE7F2
:10B0A00001EBC202107910BDF0D4010884B030B5B4
:10B0B00003AC84E80F00064C03AD0FCD0FC495E838
:10B0C0000F0084E80F00BDE8304004B0704700BFB7
:10B0D00068110020014B1878704700BFAC53002066
:10B0E000C82307B50093002304481A4603210068CB
:10B0F00003F058FD03B05DF804FB00BF400E0020D4
:10B1000013B5104C0120A368984700230093009BBF
:10B11000B3F5CC7F0FDDA36800209847002342F6EB
:10B12000FE720193019B934208DD0220A36802B0E6
:10B13000BDE810401847009B0133E7E7019B01334E
:10B140000193EFE7681100202DE9F04107460B4C11
:10B150000020E3680D4616469847236947F08000B3
:10B1600098472E44B54204D1E3680120BDE8F04180
:10B170001847236915F8010B9847F3E76811002079
:10B1800007B501228DF807100DF10701FFF7DCFF6D
:10B1900003B05DF804FB0000134A10B55060134A79
:10B1A000904219D00BF0BAFE0DA3D3E900230CF0A6
:10B1B00059F80CF0C7F90446C4F307410620FFF71D
:10B1C000DFFFC4F307210720FFF7DAFFE1B2082011
:10B1D000BDE81040FFF7D4BF054CEDE7AFF30080AA
:10B1E0000000000080844E40AC530020F01FCB33A1
:10B1F000CD3CD9002DE9F04107460C4C0020E36816
:10B200000D4616469847236907F07F0098472E445D
:10B21000B54204D1E3680120BDE8F0411847236935
:10B220000020984705F8010BF2E700BF68110020E5
:10B2300007B501220DF10701FFF7DCFF9DF80700BC
:10B2400003B05DF804FB000001282DE9F84F0D461E
:10B2500004D0022854D00020BDE8F88F6C4E27207F
:10B26000B48BFFF7E5FFA4B220F0F80001342044CE
:10B270000BF054FEB37F0022002B3CD1654B0BF04A
:10B2800011FD804630208946FFF7D2FF30F0F903E8
:10B290000CBF00235F4B0022404649460BF002FDE5
:10B2A0008046284689460BF049FE02460B4640463A
:10B2B00049460BF0F7FC96F820300022EBB900234A
:10B2C0000BF0F0FC0022544B0BF0A2FEB6690446D2
:10B2D00030460D460BF022FE02460B46204629461C
:10B2E0000BF0C0FF00224D4B0BF092FE0BF08CFCDC
:10B2F0000CF028F9B0E70023C1E74FF08043DFE707
:10B30000434C226C022A79D8454B03EBC203D3E9A4
:10B3100000670120636C98400BF010FE02460B465C
:10B32000304639460BF09EFF02460B460020394955
:10B330000BF098FF06460F46B4F84A000BF0FEFDEE
:10B340000022384B0BF0AEFC32463B460BF060FE61
:10B350008B46616C824694F84E0094F84C3089001C
:10B36000002BC1F11C0101EB001114BF14200020BF
:10B3700001EBC501081A0BF0D1FD8046606C94F812
:10B3800048308946002B14BF02230023C3EB800002
:10B390000BF0C4FD02460B46404649460BF062FFE7
:10B3A0000BF02AFB8046894694F8490004300BF0E4
:10B3B000C5FD42464B460BF02BFE002200230446FF
:10B3C0000D460CF0B5F8E0B10022134B204629469B
:10B3D0000BF068FC32463B460BF01AFE52465B46C9
:10B3E0000BF060FC00220D4B0BF012FE06A3D3E91C
:10B3F00000230BF057FC0BF083FB79E700260027B6
:10B4000087E700200449E5E72B8716D9CEF7EF3F01
:10B41000AC5300200000F03F0000204000408F406F
:10B42000D8D4010800001140012808B504D0022832
:10B430000AD04FF0FF3008BD1120FFF7F9FEC0F32E
:10B440004700404200B2F6E71B20FFF7F1FE8B38C1
:10B45000F8E700000B4B10B55B68044660B90220AA
:10B4600098470120FFF7E4FE00F0F8012143012096
:10B47000BDE81040FFF784BE03280CBF0120002068
:10B48000EEE700BF6811002013B5C82400230B4865
:10B4900000941A460321006803F084FB0023084847
:10B4A00000941A460321006803F07CFB0020FFF79C
:10B4B000D1FF0022034B1A7002B010BD400E0020D5
:10B4C00064110020AC53002013B5C82400230B489E
:10B4D00000941A460321006803F064FB0023084827
:10B4E00000941A460321006803F05CFB0120FFF77B
:10B4F000B1FF0022034B1A7002B010BD400E0020B5
:10B5000064110020AC53002073B55E4C064663788E
:10B51000DBB2012B2FD0022B67D000254FF4C8726D
:10B52000002159480CF0A8FE01232370574B1868DE
:10B530004FF0FF33002E00F097804FF47A7101FB3B
:10B5400006F20093B2FBF1F20023042103F02AFB80
:10B550006378012B40F08D800520FFF77BFF0D20E5
:10B56000FFF766FE40F020010D20C9B202B0BDE831
:10B570007040FFF705BE402094F82250FFF758FEB8
:10B580000C214020FFF7FCFD4120FFF751FE60F049
:10B590000E01C9B24120FFF7F3FD3520FFF748FE49
:10B5A00000F0C00141F012013520FFF7E9FD352020
:10B5B000FFF73EFE00F03F00112184F83A003F20E3
:10B5C000FFF7DEFD00230D2084F82C3084F82D30A9
:10B5D0002387E386FFF72CFE00F04001EDB241F037
:10B5E0002E010D20FFF7CCFD98E794F85130332061
:10B5F0001BB3FFF71DFE40F04101C9B23320FFF736
:10B60000BFFD19213B20FFF7BBFD94F8525094F881
:10B610004F30EDB2E3B11D211120FFF7B1FD402005
:10B62000FFF706FE00F033014020FFF7A9FD0021DF
:10B630000F20FFF7A5FD0021D3E7FFF7F9FD00F08C
:10B64000BE0141F001013320FFF79AFD1D21D9E72A
:10B650000F211120FFF794FD4020FFF7E9FD00F0D6
:10B660003C0141F00101DFE70093324633460321FC
:10B670006CE72DB1052002B0BDE87040FFF7EABECF
:10B680000620F8E7AC530020440E0020400E0020B6
:10B6900037B54FF47A72642350432B4DB0FBF2F26E
:10B6A000009304210023286803F07CFA0022274B32
:10B6B000274C1A706378DBB2012B14D0022B26D0F2
:10B6C000022323702C6802F09DFB052302460093A1
:10B6D00001210023204603F065FA032003B0BDE8F2
:10B6E0003040FFF7B7BE14214020FFF749FDB021DD
:10B6F0004120FFF745FD8F213520FFF741FD352023
:10B70000FFF796FD00F03F0084F83A00D8E794F880
:10B710004F3073B1F5211120FFF732FD4020FFF7C4
:10B7200087FD00F0330141F040014020FFF728FD84
:10B73000C6E7F7211120FFF723FD4020FFF778FD32
:10B7400000F03F01EFE700BF6411002088110020E6
:10B75000AC53002010B5124C6378DBB2012B04D03F
:10B76000022B09D040F2114101E040F2FA31BDE86C
:10B7700010400C48FBF79AB9FA211120FFF700FDA1
:10B780004020FFF755FD00F0FC014020FFF7F8FCDA
:10B79000032307202370BDE81040FFF75BBE00BF06
:10B7A000AC530020B4D5010808B51A4B5A78824230
:10B7B0002ED058705B780020022B13D0FFF74AFE82
:10B7C0000120FFF735FD00F07F010120FFF7D8FCD5
:10B7D00000214020FFF7D4FC30214120BDE8084083
:10B7E000FFF7CEBCFFF736FE0120FFF721FD60F02A
:10B7F0007F01C9B20120FFF7C3FC00214020FFF701
:10B80000BFFC00214120FFF7BBFC43213120E5E7CD
:10B8100008BD00BFAC5300201D4B13B518600023BA
:10B820001C4C1A4600944FF47A711B4803F098F9A7
:10B830001A4B186020B94FF486711948FBF736F996
:10B84000002300941A464FF47A71164803F088F9E1
:10B85000154B186020B94FF487711148FBF726F992
:10B86000FFF74EFC0020FFF79FFF0020FFF7F2FDDF
:10B870004FF4C87200210D480CF0FEFC002201219B
:10B880000B4B83F8282083F829101A7002B010BDE2
:10B890003C0E00203DBE0008A0D501086411002028
:10B8A000B4D50108A3D50108400E0020440E0020A5
:10B8B000AC53002073B50E4614460546FFF774FFDF
:10B8C0003046FFF769FC0520FFF7C4FD0023019314
:10B8D000019BB3F5CC7F0BDD2846FFF7A5FD0546A0
:10B8E000FFF7D2FDA542CCBF0020012002B070BD01
:10B8F000019B0133EBE773B500240220FFF754FFEF
:10B90000FF211120FFF73CFC0520FFF7A3FD254692
:10B9100026460196019BB3F5CC7F0DDD2C20FFF769
:10B9200087FC00F00100A0400134202C45EA00050E
:10B93000EFD1284602B070BD019B01330193E9E7C6
:10B940002DE9F04F824689B00193129B0D46029378
:10B95000BDF850309DF8601003939DF86430934615
:10B9600004939DF868209DF86C3006920593BDF80D
:10B970004C609DF854709DF858809DF85C9007913C
:10B98000FFF712FFDDE90532BAF1010F06D0BAF177
:10B99000020F079968D009B0BDE8F08F804C02997A
:10B9A00025615846C4F818B06161A77784F81F80F4
:10B9B00084F8209084F8212084F82230A6830BF0AC
:10B9C000ADFA02460B4674A1D1E900010BF04AFC26
:10B9D0000BF0B8FD1FFA80FB4FEA1B210220FFF796
:10B9E000CFFB5FFA8BF10320FFF7CAFB2846FFF776
:10B9F00047FB01461220FFF7C3FB0298FFF740FB0D
:10BA000001461320FFF7BCFB310A2520FFF7B8FBE6
:10BA1000F1B22620FFF7B4FBE27F2346DAB9A27F1A
:10BA2000CAB184F829A041463220FFF7A9FB302093
:10BA3000FFF7FEFB002F14BF0021802100F06F00F4
:10BA400040EA0919302041EA0901C9B209B0BDE84C
:10BA5000F04FFFF795BB00224FF4D271514883F8A5
:10BA60002920FBF723F8DEE74D48019C0564C0F868
:10BA700044B080F84940A0F84A6080F84C7080F8E3
:10BA80004D8080F84E9080F84F100499BBF10C0F58
:10BA900080F85010824680F8512080F8523074D8D7
:10BAA000BBF1050F62D925B9ABF10B03012B5FD8B0
:10BAB00004E0012D5CD1BBF10C0F59D101238AF8B0
:10BAC00048301D20FFF7B4FB019B9AF848101D2059
:10BAD00041EAC30141EA490141EA870141EA85118E
:10BAE000C9B2FFF74DFB1E20FFF7A2FB039B00F03E
:10BAF0000C00C3F30121014341EA0B11C9B21E201E
:10BB0000FFF73EFB9DF80C101F20FFF739FB310AB1
:10BB10002020FFF735FBF1B22120FFF731FB1FB1E9
:10BB200041462220FFF72CFB9AF84F306BB14B2097
:10BB3000FFF77EFB60F07F01C9B24B20FFF720FBCF
:10BB40009AF850102420FFF71BFBBBF1060F4FF0B3
:10BB500031000FD1FFF76CFB00F0F80141F0050157
:10BB60003120FFF70DFB0C2137206FE74FF0060B5C
:10BB70000023A4E7FFF75CFB00F0F80141F00301AC
:10BB80003120FFF7FDFA0A21EEE74FF00C0B012DF3
:10BB90008DE700BFAFF300800000000080847E418D
:10BBA000AC530020B4D501082DE9F04F89B01E46F2
:10BBB0009DF84C30079101939DF85C3000920493FE
:10BBC0009DF86030834605939DF86430129D029382
:10BBD0001A9BBDF8507003939DF854809DF85890BF
:10BBE000FFF7E2FD0920FFF723FB04465A20FFF789
:10BBF0001FFB04F07F03904C824660680693FFF7BA
:10BC000035FA069B07991843C0B210F0800F00F078
:10BC1000F00C2AD011291EDD14290B46A8BF1423CD
:10BC20004AF007025FFA82FA591F4CEA010C5FFAE8
:10BC30008CF109200693FFF7A3FA51465A20FFF72B
:10BC40009FFABBF1010F069B17D0BBF1020F68D022
:10BC500009B0BDE8F08F02290B46B8BF02230AF0F5
:10BC6000F80242F0040A991EDFE70E290B46A8BF2E
:10BC70000E2343EAE373591CD7E72372009B009815
:10BC8000E360029B2661A561A78384F81E8084F887
:10BC9000209084F82130039B63620BF03FF962A38C
:10BCA000D3E900230BF0DEFA0BF04CFC84B2210A3E
:10BCB0000420FFF765FAE1B20520FFF761FA284694
:10BCC0000BF02CF902460B4659A1D1E900010BF00B
:10BCD000C9FA0BF037FC84B2210A0220FFF750FAB0
:10BCE000E1B20320FFF74CFA390A2520FFF748FAA2
:10BCF000F9B22620FFF744FA3020FFF799FAB8F19D
:10BD0000000F14BF0021802100F06F0040EA0919E4
:10BD1000302041EA0901C9B209B0BDE8F04FFFF790
:10BD20002FBA84F83C30019B2664656484F849305E
:10BD3000049BA4F84A7084F84C8084F84F30059B2B
:10BD40000C2D84F85030029B84F84E9084F85130CA
:10BD5000039BDFF8E4A0636562D8052D52D926B9AC
:10BD6000A5F10B03012B4ED803E0012E4BD10C2D76
:10BD700049D101238AF848309AF84F306BB14B20F3
:10BD8000FFF756FA60F07F01C9B24B20FFF7F8F9D0
:10BD90009AF850102420FFF7F3F91D20FFF748FA16
:10BDA000019B94F848101D2041EAC30141EA490172
:10BDB00041EA880141EA8611C9B2FFF7E1F91E2084
:10BDC000FFF736FA00F00F0141EA0511C9B21E2053
:10BDD000FFF7D6F9390A2020FFF7D2F92120F9B26E
:10BDE000FFF7CEF9062D4FF031000ED1FFF720FA04
:10BDF00000F0F80141F005013120FFF7C1F90C21F5
:10BE0000372089E706250023B4E7FFF711FA00F091
:10BE1000F80141F003013120FFF7B2F90A21EFE701
:10BE20000C25012E9FE700BF0000000080844E40DB
:10BE30000000000080847E41AC53002010B5254CEA
:10BE40002378DBB2012B02D0022B34D010BD6378F3
:10BE5000012B29D100230B213E2084F82C3084F8BB
:10BE60002D302387E386FFF78BF910213F20FFF762
:10BE700087F994F8223003F0FF029BB10D20FFF701
:10BE8000D7F940F02001C9B20D20FFF779F9124B24
:10BE90001B68002BDAD0DB68002BD7D0BDE8104040
:10BEA000002018472270F2E794F85230002BEED0B1
:10BEB000FFF70AFBEBE7002301222370074B1A7000
:10BEC000054B1B68002BC1D05B68002BBED0BDE8C2
:10BED00010401847AC5300203C0E00208811002071
:10BEE00007B50022154B8DF8072083F82C2083F826
:10BEF0002D201A87DA8683F82E2093F8223023B972
:10BF000003B05DF804EBFFF7BFBA3F20FFF790F9ED
:10BF10008DF807009DF80730DB0603D510213F2080
:10BF2000FFF72EF90D20FFF783F940F040010D20B7
:10BF3000C9B203B05DF804EBFFF722B9AC5300209F
:10BF40002DE9F04107460C4C0020E3680D461646EB
:10BF50009847236907F07F0098472E44B54204D1E3
:10BF6000E3680120BDE8F0411847236900209847A5
:10BF7000C04305F8010BF1E7681100200A460146AD
:10BF80000020FFF7E1B80000F7B5564C064663788D
:10BF90000D46DBB2012B12D0022B36D000252846ED
:10BFA000FFF776FB6378012B40F09980002D00F0BD
:10BFB00096804D4E4D4D3378002B69D08FE0002395
:10BFC00023878BB2E386A37F13B13220FFF7D8F823
:10BFD0006B1E3F2B0FD884F83B500025304694F859
:10BFE0003B10FFF7CBFF94F83B30228F13449BB2FA
:10BFF0002387606AD4E72A4631463C480CF014F99E
:10C000003C23012584F83B30E8E794F85130332095
:10C010002BB3FFF70DF900F0BE013320FFF7B0F8A6
:10C0200019213B20FFF7ACF82946222084F85C5008
:10C03000FFF7A6F800210E20FFF7A2F800210D203F
:10C04000FFF79EF80120FFF7F3F830F0F80711D062
:10C0500029463046FFF792FF0025606DA0E7FFF705
:10C06000E7F800F0BE0141F001013320FFF788F846
:10C070001D21D6E7FFF728FA0197019BB3F5CC7F86
:10C08000E6DC019B01330193F7E7012002F012F88F
:10C090003F20FFF7CDF88306F7D4E38E218F94F885
:10C0A0003B205B1A9342208F0BDD94F83B10284411
:10C0B000FFF764FF94F83B30228F13449BB2238731
:10C0C00079E7E18E238F2844C91AC9B2FFF756FFDA
:10C0D000E18E228F238F0B449B1A9BB2238703B0E0
:10C0E000F0BD00BFAC53002088110020440E00209A
:10C0F0000A4601460020FFF77DB80A4601460020A7
:10C10000FFF71EBF38B505460C46FFF74DFB012D66
:10C1100002D0022D0AD038BD064B9B7F002BFAD1EE
:10C1200021463220BDE83840FFF72AB821462320B7
:10C13000F8E700BFAC5300207FB50022654D8DF8B5
:10C140000B202B780392DBB2012B2C4604D0022B60
:10C1500000F09E8004B070BD6B78DBB2012B34D050
:10C16000022BF7D140211220FFF70AF81220FFF727
:10C170005FF88DF80B009DF80B30574E13F0200F31
:10C1800029D020211220FEF7FBFF95F8523003F052
:10C19000FF0203B92A7000225048009203AB082125
:10C1A000006802F0FFFC039B3BB14FF080524C4B08
:10C1B0001A60BFF34F8FBFF36F8F3368002BC9D066
:10C1C0001B69002BC6D09847C4E740F21C51454874
:10C1D000FAF76CFCBEE71920FFF72AF840B285F8A1
:10C1E000580095F8583095F858501B0642BF6DB26C
:10C1F0006D42C5F385054FF01A004CBF6D42AD0886
:10C20000FFF716F8002D40F30B13B8BF40198B3819
:10C210009BB203441BB2A4F85A301320FFF708F86E
:10C2200084F85C001020FFF703F801460D20FEF7AC
:10C23000A7FF94F85C102C48FFF75AFF94F852308F
:10C2400003F0FF028BB925482270009203AB08214E
:10C25000006802F0A7FC039B3BB14FF08052204BDB
:10C260001A60BFF34F8FBFF36F8F3368002B3FF41B
:10C2700071AF9D68002D3FF46DAF94F85C10B4F879
:10C280005A2094F8583012B25BB21748A84761E7B9
:10C290001648009203AB0821006802F083FC039B60
:10C2A0003BB14FF080520E4B1A60BFF34F8FBFF37C
:10C2B0006F8F6378022B03D108211220FEF760FFF5
:10C2C00000232370044B1B68002B3FF443AF1B6813
:10C2D00077E700BFAC5300203C0E0020400E00204A
:10C2E00004ED00E0B4D50108440E002064110020E4
:10C2F0002DE9FF41002259498DF80B200B7803925C
:10C30000DBB2012B0C4605D0022B00F0A58004B057
:10C31000BDE8F0814B78DBB2012B22D0022BF6D1A5
:10C320004F48009203AB0821006802F03BFC039BDE
:10C330003BB14FF080524B4B1A60BFF34F8FBFF3AE
:10C340006F8F80211220FEF71BFF00232370464BC6
:10C350001B68002BDBD0DB68002BD8D0012098476E
:10C36000D5E73F20FEF764FF8DF80B009DF80B30FA
:10C370009A06CCD59DF80B30DB0605D53B48FEF779
:10C380009FF8FFF7ADFDC2E794F8293023B940F2DA
:10C39000C1513748FAF78AFB94F82830022B2DD187
:10C3A000238F344894F83A101844FFF7A6FE238FE1
:10C3B0009BB2002B3DD094F83A30228F13449BB2AD
:10C3C0002387238FE28E9A42A1D8E28E29492A48F8
:10C3D0000BF02AFF94F82E50E48EFFF781FD224BDC
:10C3E0006DB21B68A4B2002B91D09E68002E8ED037
:10C3F00000232A4621462048B04788E71F4D0020E9
:10C40000EB6898472B69002098470027DFF8648085
:10C4100094F83A30BB4203DCEB6801209847C6E74A
:10C420002B690020268F9847B6B24644F055013755
:10C43000EEE794F82D30002BA3D094F83A100D4875
:10C44000FEF7EEFDE086E38EB3F5C87F99D2E38E6A
:10C450009BB2002BAFD194E74B7858E7AC53002048
:10C46000400E002004ED00E03C0E0020A6D501089F
:10C47000B4D50108440E0020D40F0020681100201C
:10C4800010B51A4C2378DBB2012B02D0022B2AD034
:10C4900010BD6178C9B2012918D00229F8D194F8E9
:10C4A0004F30002BF4D01220FEF76AFE104B1B68B1
:10C4B000002BEDD05C69002CEAD01C20FEF7B8FE02
:10C4C0002346BDE8104000F03F001847002311202C
:10C4D000238784F82D10FEF7ABFE4008404240B29F
:10C4E00084F82E00D4E76178C9B2D6E7AC530020B7
:10C4F0003C0E00201F4B70B55A78022A05D11B78DC
:10C50000DBB2012B02D0032B13D070BD1220FEF73B
:10C510008FFEC306F9D510211220FEF731FE164B0F
:10C520001B68002BF1D0DB69002BEED0BDE870401A
:10C5300018471220FEF77CFE10F001050E4C0DD0BE
:10C5400005211220FEF71CFE2368002BDDD09B691D
:10C55000002BDAD00120BDE87040184704211220DA
:10C56000FEF70EFE2368002BCFD09B69002BCCD0AA
:10C570002846F0E7AC5300203C0E0020074A5378D1
:10C58000012B09D11378DBB2012B05D102213E200A
:10C5900082F82C30FEF7F4BD704700BFAC5300208A
:10C5A000014B5B78704700BFAC5300200648006821
:10C5B000006880F3088862B661B6BFF34F8FBFF39F
:10C5C0006F8F00DF00BF000008ED00E0002307B51B
:10C5D00001930B4B1B68013303D0CA210948FAF7BA
:10C5E00065FA4FF0500383F31188BFF36F8FBFF3E9
:10C5F0004F8F019B002BFCD003B05DF804FB00BF04
:10C60000A800002001D601084FF0807340F8043CD8
:10C61000054B21F0010140F8081C40F80C3C40F8A3
:10C62000202C4038704700BFCDC500080000000036
:10C63000074B19680868B0E8F00F80F30988BFF36A
:10C640006F8F4FF0000080F311884EF00D0E704791
:10C65000A84D00204FF0500383F31188BFF36F8F74
:10C66000BFF34F8F084A13680133012B136009D1C0
:10C67000064B1B6813F0FF0F04D040F275110448FD
:10C68000FAF714BA704700BFA800002004ED00E0DC
:10C6900001D6010810B5074C236823B94FF4BE71C9
:10C6A0000548FAF703FA2368013B23600BB983F3CB
:10C6B000118810BDA800002001D60108000000006C
:10C6C000EFF30980BFF36F8F0D4B1A6820E9F00F6D
:10C6D00010602DE908404FF0500080F3118801F000
:10C6E0000FFD4FF0000080F31188BDE80840196885
:10C6F0000868B0E8F00F80F30988BFF36F8F7047C8
:10C70000A84D002008B54FF0500383F31188BFF304
:10C710006F8FBFF34F8F01F089FB18B14FF080523C
:10C72000024B1A60002383F3118808BD04ED00E07A
:10C730000022054B05491A600A6041F26701044A6C
:10C74000116007221A60704710E000E018E000E076
:10C7500014E000E013B5254B254C1A78D2B20192B3
:10C76000FF221A701B78234ADBB28DF803309DF844
:10C77000033003F0500313700723002223609DF859
:10C780000310581E090628D412B1032B236004D0CD
:10C790004FF49B711848FAF789F92368134A1B0272
:10C7A00003F4E06323600024019BDBB21370134B9E
:10C7B0001A6842F470021A601A6842F070421A60F5
:10C7C000FFF7B6FF0E4B1C60FFF7F0FE01F098FC80
:10C7D000FFF7FCFE204602B010BD9DF80330012299
:10C7E0005B00DBB28DF803300346C8E700E400E0ED
:10C7F0008C1100208911002001D6010820ED00E0F5
:10C80000A800002008B5EFF305830F2B0AD90D4AC5
:10C810009B5C0D4A12789A4204D940F2A5210B483C
:10C82000FAF744F90A4B0B4A1B68126803F4E063F9
:10C83000934206D9BDE8084040F2B5210348FAF713
:10C8400035B908BDF0E300E08911002001D60108E8
:10C850000CED00E08C11002010B50F4B1A688242DD
:10C8600018D35C681919884201BF41681846091934
:10C870005960446801198A4207D1084909688A4207
:10C880001FBF51681268091941609842026018BFC1
:10C89000186010BD1346E1E7A04D00209011002064
:10C8A00038B5064B064D1C68246804B938BD6307CB
:10C8B000FAD079212846FAF7F9F8F5E7A04D0020DB
:10C8C00059D6010800487047941100202DE9F8431B
:10C8D000074601F08FFA3B493B4D0B68D3B93B4B00
:10C8E0003B4A58074FF000001CBF073323F00703F3
:10C8F00013605060374A22F00702C2E90000D01AE4
:10C90000C3E90020344B0A601860344B18604FF0C4
:10C9100000432B602B681F4252D1002F41D007F1FA
:10C92000080462071CBF24F007040834002C47D019
:10C930002A4B1A689846A24242D3254B1E68726859
:10C94000A24202D23068002837D10968B14237D0FC
:10C950001F683168121B102A07F10807196010D9E7
:10C9600006EB040919F0070F03D0D7211C48FAF78A
:10C970009DF8736848461B1BC9F804307460FFF7C4
:10C980006BFF15497268D8F8003008689B1A83421B
:10C99000C8F8003038BF0B602B6813437360002366
:10C9A000336001F0D3FA7B0704D040F217110C4832
:10C9B000FAF77CF83846BDE8F88333460646BEE70A
:10C9C0000027EEE790110020944D002094110020E4
:10C9D000A04D00208C4D00209C4D0020984D002043
:10C9E00059D6010838B5044670B3184D50F8041CE8
:10C9F0002A68114204D140F22B111548FAF756F873
:10CA000054F8083C23B14FF496711148FAF74EF8E8
:10CA100054F8043C2A68134216D054F8081C99B9FB
:10CA200023EA020344F8043C01F0E4F9094A54F80B
:10CA3000043C1168A4F108000B441360FFF70CFFDD
:10CA4000BDE8384001F082BA38BD00BF944D0020E7
:10CA500059D60108984D0020014B1868704700BF57
:10CA6000984D0020014B1868704700BF9C4D002076
:10CA700010B50446FFF7EEFDA46BFFF70BFEB4FA0A
:10CA800084F0400910BD70B51546026C0446866BF3
:10CA900042B905689DB9806801F0FEFDA5600136C8
:10CAA000A66370BD6DB940680BF0BEFB6368226C75
:10CAB0001344A2686360934201D32368636000203B
:10CAC000EDE7C0680BF0B0FB236CE2685B422168C5
:10CAD0001A448A42E2603EBFA2689B18E360022DBE
:10CAE000EDD10EB1013EEAE73046D8E703461A6CB5
:10CAF00010B4084662B1D9689C681144A142D9605B
:10CB000028BF196810BC28BFD960D9680BF08CBB4E
:10CB100010BC704770B50446FFF79CFD94F8455073
:10CB200004F124066DB2002D14DCFF2384F8453097
:10CB3000FFF7B0FDFFF78EFD94F8445004F11006A6
:10CB40006DB2002D12DCFF2384F84430BDE8704044
:10CB5000FFF7A0BD636A002BE7D0304601F0C6FBAB
:10CB600008B101F05FFC013D6DB2DCE72369002BE9
:10CB7000E9D0304601F0BAFB08B101F053FC013DA9
:10CB80006DB2DEE738B50D46044620B940F2031118
:10CB90001948F9F78BFFFFF75DFDD4E90F314B43DF
:10CBA0002268D0185B1A1344A060E3600020FF23C2
:10CBB000A063626084F8443084F8453095B92369F5
:10CBC00063B104F1100001F091FB38B14FF08052D5
:10CBD0000A4B1A60BFF34F8FBFF36F8FFFF75AFDF9
:10CBE000012038BD04F1100002F01CF904F124000A
:10CBF00002F018F9F2E700BFAFD6010804ED00E03B
:10CC0000F8B50D461746064620B94FF4BB710D48DE
:10CC1000F9F74CFF05FB06F05030FFF757FE0446CE
:10CC200058B165B100F150032360C4E90F650121DB
:10CC30002046FFF7A7FF84F84C702046F8BD034656
:10CC4000F2E700BFAFD601082DE9FF478846019201
:10CC50001E46044620B940F2F1214B48F9F726FF61
:10CC6000B8F1000F06D1236C23B140F2F2214648FF
:10CC7000F9F71CFF022E07D1E36B012B04D040F221
:10CC8000F3214148F9F712FF01F0A4FC30B9019BF0
:10CC900023B140F2F6213C48F9F708FF0027B946D6
:10CCA000DFF8E8A0FFF7D6FCA26BE36B9A4201D352
:10CCB000022E19D1324641462046FFF7E4FE636A50
:10CCC0001BB104F1240001F011FB38B14FF0805288
:10CCD0002E4B1A60BFF34F8FBFF36F8FFFF7DAFC55
:10CCE000012004B0BDE8F087019D1DB9FFF7D2FC1B
:10CCF0000020F6E717B902A801F052FBFFF7CAFCC3
:10CD000001F078F8FFF7A6FC94F84430FF2B08BF39
:10CD100084F8449094F84530FF2B08BF84F8459080
:10CD2000FFF7B8FC01A902A801F046FB28BBFFF7FA
:10CD300091FCA26BE36B9A420ED1FFF7ABFC019919
:10CD400004F1100001F098FA2046FFF7E3FE01F02D
:10CD5000FDF848B10127A5E7FFF79CFC2046FFF747
:10CD6000D9FE01F0F3F8F5E74FF08053CAF8003030
:10CD7000BFF34F8FBFF36F8FECE72046FFF7CAFE7C
:10CD800001F0E4F8B4E700BFAFD6010804ED00E01D
:10CD900010B5024600210120FFF732FF044638B1EA
:10CDA000002383600360C3601A461946FFF74CFFF7
:10CDB000204610BD2DE9F843894690461F4604469B
:10CDC00020B940F2C3312748F9F770FEB9F1000FDE
:10CDD00006D1236C23B14FF471712248F9F766FE36
:10CDE000022F07D1E36B012B04D040F2C5311D485F
:10CDF000F9F75CFEFFF706FDEFF311864FF05003E5
:10CE000083F31188BFF36F8FBFF34F8FA26BE36B78
:10CE10009A4201D3022F22D194F845503A466DB27E
:10CE200049462046FFF72FFE6B1C13D1636A0BB9EE
:10CE300001200BE004F1240001F058FA0028F7D09B
:10CE4000B8F1000FF4D00120C8F8000086F3118873
:10CE5000BDE8F88301356DB284F84550E8E700205D
:10CE6000F4E700BFAFD6010870B50D46044620B9FF
:10CE70004FF48C612048F9F719FE236C23B140F27E
:10CE800064411D48F9F712FE236833B9A36823B142
:10CE900040F269411848F9F709FEFFF7B3FCEFF3D8
:10CEA00011864FF0500383F31188BFF36F8FBFF3E8
:10CEB0004F8FA26BE36B93421CD994F8453001323B
:10CEC0005BB2A2635A1C10D1636A0BB9012009E05E
:10CED00004F1240001F00AFA0028F7D0002DF5D063
:10CEE0000120286086F3118870BD01335BB284F89D
:10CEF0004530EBE70020F5E7AFD601082DE9F04318
:10CF000085B00F460192044620B94FF4A061424813
:10CF1000F9F7CCFD37B9236C23B140F204513E48F8
:10CF2000F9F7C4FD01F056FB30B9019B23B140F283
:10CF300009513948F9F7BAFD0026B046DFF8DC9010
:10CF4000FFF788FBA56BD5B139462046013DFFF7B9
:10CF5000CDFDA563236963B104F1100001F0C6F9AA
:10CF600038B14FF080522D4B1A60BFF34F8FBFF393
:10CF70006F8FFFF78FFB012005B0BDE8F083019DA7
:10CF80001DB9FFF787FB0020F6E716B902A801F0EC
:10CF900007FAFFF77FFB00F02DFFFFF75BFB94F82C
:10CFA0004430FF2B08BF84F8448094F84530FF2BB1
:10CFB00008BF84F84580FFF76DFB01A902A801F0C6
:10CFC000FBF9F0B92046FFF753FDA0B1019904F138
:10CFD000240001F051F92046FFF79CFD00F0B6FF58
:10CFE00038B94FF08053C9F80030BFF34F8FBFF30B
:10CFF0006F8F0126A4E72046FFF78CFD00F0A6FF07
:10D00000F7E72046FFF786FD00F0A0FF2046FFF778
:10D010002FFD0028EDD0B6E7AFD6010804ED00E003
:10D020002DE9FF410446019120B940F29151524847
:10D03000F9F73CFD236C23B140F295514E48F9F7C6
:10D0400035FD01F0C7FA30B9019B23B140F29A5186
:10D050004948F9F72BFD00252F462E46DFF81C81A5
:10D06000FFF7F8FAA36BE3B1013BA363236813B99D
:10D0700001F0B2FBA060236963B104F1100001F07C
:10D0800035F938B14FF080523C4B1A60BFF34F8FE7
:10D09000BFF36F8FFFF7FEFA0125284604B0BDE805
:10D0A000F081019B4BB925B140F2E1513248F9F7CB
:10D0B000FDFCFFF7EFFA0025EFE717B902A801F032
:10D0C0006FF9FFF7E7FA00F095FEFFF7C3FA94F85F
:10D0D0004430FF2B08BF84F8446094F84530FF2BA0
:10D0E00008BF84F84560FFF7D5FA01A902A801F04E
:10D0F00063F940BB2046FFF7BBFCF0B123683BB9A6
:10D10000FFF7A8FAA06801F075FA0546FFF7C2FA22
:10D11000019904F1240001F0AFF82046FFF7FAFC72
:10D1200000F014FF38B94FF08053C8F80030BFF357
:10D130004F8FBFF36F8F012792E72046FFF7EAFC7E
:10D1400000F004FFF7E72046FFF7E4FC00F0FEFEE6
:10D150002046FFF78DFC0028EDD0002D9DD0FFF775
:10D1600079FA616A19B1236B1968C1F10501A068E8
:10D1700001F0DEFA9DE700BFAFD6010804ED00E044
:10D180002DE9F04385B00F460192044620B94FF4D3
:10D19000CD614248F9F78AFC37B9236C23B140F2DC
:10D1A0006C613E48F9F782FC01F014FA30B9019B3A
:10D1B00023B140F271613948F9F778FC0026B04696
:10D1C000DFF8DC90FFF746FAA36BD3B1394620466F
:10D1D000E568FFF78BFC636AE56063B104F1240046
:10D1E00001F084F838B14FF080522D4B1A60BFF334
:10D1F0004F8FBFF36F8FFFF74DFA012005B0BDE8E9
:10D20000F083019D1DB9FFF745FA0020F6E716B936
:10D2100002A801F0C5F8FFF73DFA00F0EBFDFFF7BB
:10D2200019FA94F84430FF2B08BF84F8448094F82E
:10D230004530FF2B08BF84F84580FFF72BFA01A982
:10D2400002A801F0B9F8F0B92046FFF711FCA0B12F
:10D25000019904F1240001F00FF82046FFF75AFC71
:10D2600000F074FE38B94FF08053C9F80030BFF3B6
:10D270004F8FBFF36F8F0126A4E72046FFF74AFCCC
:10D2800000F064FEF7E72046FFF744FC00F05EFE86
:10D290002046FFF7EDFB0028EDD0B6E7AFD601083A
:10D2A00004ED00E02DE9F84389469046054620B993
:10D2B00040F2FB612048F9F7F9FBB9F1000F06D104
:10D2C0002B6C23B140F2FC611B48F9F7EFFBFFF731
:10D2D00099FAEFF311874FF0500383F31188BFF3EE
:10D2E0006F8FBFF34F8FAC6B1CB395F8446049460A
:10D2F00076B22846FFF7FAFB013C731CAC6313D1EE
:10D300002B690BB901200BE005F1100000F0EEFFD6
:10D310000028F7D0B8F1000FF4D00120C8F80000C1
:10D3200087F31188BDE8F883013676B285F844604A
:10D33000E8E72046F4E700BFAFD6010810B5044681
:10D3400020B940F28A710548F9F7B0FBFFF782F97E
:10D35000A46BFFF79FF9204610BD00BFAFD60108B0
:10D3600038B5054620B940F2A4710648F9F79EFB8E
:10D37000FFF770F9A86BEC6B241AFFF78BF92046C6
:10D3800038BD00BFAFD60108002330B5064A52F8B9
:10D39000335002EBC3041DB942F83310606030BD56
:10D3A0000133052BF3D1FAE70C540020002310B50C
:10D3B000084951F83320DC00824206D10021064A98
:10D3C00042F833102244516010BD0133052BF0D1D7
:10D3D000FAE700BF105400200C54002010B504469A
:10D3E00020B94FF4F8610548F9F760FB2046FFF7D4
:10D3F000DDFFBDE81040FFF7F5BA00BFAFD601086A
:10D4000070B504460D461646FFF724F994F84430EB
:10D41000FF2B04BF002384F8443094F84530FF2BE1
:10D4200004BF002384F84530FFF734F9A36B2BB910
:10D430003246294604F1240000F038FF2046BDE8BA
:10D440007040FFF767BB8268436800681344181A8E
:10D45000824298BF801A70472DE9F84305468846F6
:10D46000174622B940F244411848F9F71FFB6C688F
:10D47000AB681E1BBE4228BF3E46A219934204D28F
:10D4800040F24E411148F9F711FBA8693246414676
:10D4900020440AF0C9FEB7420FD9AB68A7EB0609D2
:10D4A000994504D940F256410848F9F7FFFA4A462F
:10D4B00008EB0601A8690AF0B7FEAB683C44A3423A
:10D4C00098BFE41A6C603846BDE8F883F3D60108CB
:10D4D0009A422DE9F843164628BF1E46074689465C
:10D4E000904686B305688468641BB44228BF3446FE
:10D4F000A24204D24FF490611448F9F7D7FABA68FF
:10D500002B19934204D940F281411048F9F7CEFA21
:10D51000B9692246294448460AF086FEA6420CD93B
:10D52000B04504D240F289410848F9F7BFFA321BEE
:10D53000B96909EB04000AF077FEBB683544AB42D9
:10D5400098BFED1A3D603046BDE8F883F3D6010878
:10D55000012A2DE9F04104460F46164630D1042831
:10D5600003D8E8211A48F9F7A1FABC4203D2F02106
:10D570001748F9F79BFA002F04F1250008BF01278F
:10D58000FFF7A4F90546C0B100F124080134224692
:10D59000552140460AF070FE804504D04FF4996151
:10D5A0000B48F9F783FA2422002128460AF064FE8A
:10D5B000C5E90247C5F818802E772846BDE8F081F6
:10D5C00018B9EE210248F9F771FA0026CDE700BF3D
:10D5D000F3D601082DE9F843044620B940F2911131
:10D5E0001748F9F763FA276AFFF734F8206918BB80
:10D5F00063691BBBD4E90269A569324655212846F7
:10D6000094F81C800AF038FE854204D04FF49961EA
:10D610000B48F9F74BFA2046202200210AF02CFE95
:10D62000A561C4E9026984F81C8027620124FFF720
:10D6300031F82046BDE8F8830024F8E70446F6E711
:10D64000F3D6010810B5044620B940F2DB110648B4
:10D65000F9F72CFAA3682068626818440138801A28
:10D66000834298BFC01A10BDF3D601082DE9F047D8
:10D6700086B0044616460193884621B94FF40171DD
:10D680004048F9F713FA24B940F205213D48F9F76B
:10D690000DFA237FDA0715D5371DBE4204D34FF4A8
:10D6A00004713848F9F702FA019B6BB92046FFF77D
:10D6B000C9FF05460396002D38D10025284606B03F
:10D6C000BDE8F0873746EFE704A800F04FFE4FF0C3
:10D6D0000009DFF8B0A0FEF7BDFF2046FFF7B2FF5C
:10D6E000874205461FD9002001F0B4F9636923B1D0
:10D6F00040F229215046F9F7D9F900F065FF606141
:10D70000FEF7C8FF0022019B1146104601F070F899
:10D71000C4F8149001A904A800F04EFE0028DAD045
:10D72000002DC3D0C6E7FEF7B5FFF9E7237FDB077F
:10D7300020D4B54294BF03950396039A41462046F0
:10D74000FFF78AFE05460028B8D02046FFF77BFE8B
:10D75000E3689842B2D300F04DFB23693BB100234C
:10D7600020691A46194601F087F80023236100F06A
:10D77000EDFBA3E7BD42A0D3042203A92046FFF797
:10D780006BFEDAE7F3D601082DE9F74304461746A6
:10D790009946884621B940F2D1213348F9F786F9F4
:10D7A00024B940F2D2213048F9F780F9237F13F0F1
:10D7B000010F14BF04260026B9F1000F20D0FEF798
:10D7C00049FF2046FFF73FFE864205460CD3002066
:10D7D00001F040F9236923B140F2F5212248F9F71D
:10D7E00065F900F0F1FE2061FEF754FFAE4212D35E
:10D7F00000224B461146104600F0FAFF0023236139
:10D800002046FFF720FEB042054604D800252846F2
:10D8100003B0BDE8F0837EB12B46324601A9204615
:10D82000D4F80090FFF754FE019BAD1B9F4236BF1A
:10D8300000271F46C4F800902B463A464146204632
:10D84000FFF746FE05460028E0D000F0D3FA6369F2
:10D850003BB1002360691A46194601F00DF8002318
:10D86000636100F073FBD2E7F3D60108064A136840
:10D870001968064B19B94FF0FF321A6070471268E9
:10D88000D268D2685268F8E7AC4D00205C4E0020A8
:10D8900010B5044620B940F2F2610848F9F706F9DC
:10D8A0006269074B9A4207D1A06A064B984203D09F
:10D8B000B0FA80F0400910BD0020FCE73FD7010816
:10D8C0007C4E0020644E0020F8B51B4B1B4E1C689C
:10D8D000054630680F46043001F0D5FA334640B9AA
:10D8E00001203168164EC96A3268884022EA000277
:10D8F00032606A1C07D137B1196812480431BDE89B
:10D90000F84001F09DBA1A686419546007D30E4AB2
:10D9100010681968BDE8F840043101F09DBA0B4A5F
:10D9200010681968043101F097FA094B1A68A2428D
:10D9300088BF1C60F8BD00BFA44E0020A84D002089
:10D940002C4E00207C4E0020B04D0020AC4D00201D
:10D950005C4E002080B5DFF86480144F144C154EE7
:10D96000236863B9144B1B68012BF8D94FF080531F
:10D97000C8F80030BFF34F8FBFF36F8FEEE7FEF7AD
:10D9800069FEFB68DD68281D01F07DFA3368013B04
:10D9900033602368013B2360FEF77CFE286BFFF7B2
:10D9A00021F82846FFF71EF8DAE700BF904E002066
:10D9B0001C4E0020184E0020B44D002004ED00E065
:10D9C0002DE9F84F4FEA820A804650460D469946A7
:10D9D0000B9EFEF77BFF0746002800F0AA805C2024
:10D9E000FEF774FF0446002800F0A080076325B905
:10D9F0004FF458715648F9F759F85246A521206B53
:10DA00000AF03AFC236BAAF1040A9A442AF0070AA6
:10DA10006B1E04F134020F3513F8011F02F8011BCD
:10DA200009B19D42F8D10A9D4FF0000B042D28BF8B
:10DA30000425271DE562C4E9135B384684F843B02A
:10DA400001F0FBF9C5F1050504F1180001F0F5F945
:10DA5000C4F854B02461A561646284F858B04A46A1
:10DA600041465046FEF7D0FD206006B13460FEF717
:10DA7000F1FD384B384E1A68DFF8188101321A6010
:10DA80003268002A58D134601B68012B25D13348F5
:10DA900001F0C8F9324801F0C5F9324801F0C2F985
:10DAA000DFF8F490304801F0BDF9304D304801F016
:10DAB000B9F9484601F0B6F9284601F0B3F92D4806
:10DAC00001F0B0F92C4801F0ADF92C4801F0AAF9A9
:10DAD0002B4BC3F800902B4B1D6001252A4A2B4984
:10DAE0001368086801331360E26A636405FA02F39D
:10DAF000034314200B60194B394600FB023001F040
:10DB00009FF9FEF7C7FDD8F8003063B13368DA6AD1
:10DB1000E36A9A4207D24FF080521D4B1A60BFF35E
:10DB20004F8FBFF36F8F2846BDE8F88F3846FEF75A
:10DB300059FF4FF0FF35F6E7D8F80030002BCCD175
:10DB40003368DA6AE36A9A4298BF3460C5E700BF77
:10DB50003FD70108184E0020A84D0020B44D0020EA
:10DB6000C84D0020DC4D0020F04D0020444E002028
:10DB7000044E0020644E0020904E00207C4E002079
:10DB8000AC4D0020B04D0020284E00202C4E00202F
:10DB900004ED00E0784E0020304E002070B50446C1
:10DBA000284DFEF757FD04B92C68261D304601F0BC
:10DBB0006AF960B91421E06A234B41435B5833B9D9
:10DBC0000122224982400B6823EA02030B60A36A08
:10DBD0001BB104F1180001F056F91D4A1368013316
:10DBE00013602B68A34220D131461A4801F028F96E
:10DBF000194A136801331360FEF74CFD174B1B687D
:10DC000093B12B68A3420FD1154B1B6823B140F28F
:10DC1000B6411448F8F74AFF4FF08052124B1A6091
:10DC2000BFF34F8FBFF36F8F70BD104A206B136827
:10DC3000013B1360FEF7D6FE2046FEF7D3FEFFF74A
:10DC400015FED9E7A84D0020B44D00202C4E002031
:10DC5000284E0020904E00201C4E0020784E0020C0
:10DC6000244E00203FD7010804ED00E0184E0020AC
:10DC7000F8B5054620B940F24C511748F8F716FFA1
:10DC8000164B1B68AB4220D0FEF7E4FC144B6C69CA
:10DC90001F68144B1E68FEF7FDFCBC4217D0B4424F
:10DCA00015D0114B9C4208D1AB6A83B995F8583016
:10DCB000012B0CBF02200320F8BD0C4B9C4208D066
:10DCC000002C0CBF04200120F6E70020F4E702201E
:10DCD000F2E70420F0E700BF3FD70108A84D00207D
:10DCE000AC4D0020B04D00207C4E0020904E002016
:10DCF00070B5044620B940F21C711948F8F7D6FEF9
:10DD0000184D2B68A34229D044B3FEF7A3FC20464C
:10DD1000FFF7BEFDF0B1261D304601F0B4F8012337
:10DD20001149E26A08689340034314200B600F4BCB
:10DD3000314600FB023001F083F82B68E26ADB6AAF
:10DD40009A4207D34FF08052094B1A60BFF34F8FAE
:10DD5000BFF36F8FBDE87040FEF79CBC70BD00BF85
:10DD60003FD70108A84D00202C4E0020B44D0020C4
:10DD700004ED00E013B50024174B009401935022EA
:10DD8000234616491648FFF71BFE012818D100F05C
:10DD9000C1FE012814D14FF0500383F31188BFF363
:10DDA0006F8FBFF34F8F4FF0FF320E4B1A600E4B49
:10DDB00018600E4B1C6002B0BDE81040FEF7CABCF4
:10DDC000013007D140F60401094802B0BDE8104017
:10DDD000F8F76CBE02B010BD584E002083D7010882
:10DDE00055D900085C4E0020784E0020A44E00203B
:10DDF0003FD70108024A136801331360704700BF20
:10DE0000244E0020014B1868704700BFA44E00202C
:10DE100008B5FEF7F7FC014B186808BDA44E0020BA
:10DE2000014B1868704700BF184E00202DE9F84FCD
:10DE30003A4B1B68002B6AD1394B1C6801341C60BB
:10DE40009CB9384D2B681B6823B140F662213648D7
:10DE5000F8F72CFE354B2A68196829601A60344A95
:10DE6000136801331360FFF701FD324D4FF0000BD3
:10DE70002B68314FA34211D93A68304BD16A142232
:10DE80004A439A58022A28BF4FF0010B2C4A1268C5
:10DE9000002A0CBF58460120BDE8F88FDFF884A0A7
:10DEA000DFF8A490DAF8002012681AB94FF0FF32B8
:10DEB0002A60E1E7DAF80020D268D66871688C42FF
:10DEC00001D22960D8E706F10408404600F0DBFFE4
:10DED000B16A19B106F1180000F0D5FF01224FF028
:10DEE000140CF06AD9F8003002FA00F11943134B10
:10DEF000C9F800100CFB0030414600F0A1FF386863
:10DF0000F16AC26A914228BF4FF0010BCAE70D4A7D
:10DF10004FF0000B136801331360B7E7244E002065
:10DF2000A44E0020AC4D00203FD70108B04D00208A
:10DF3000604E00205C4E0020A84D0020B44D002013
:10DF4000A84E0020204E00202C4E00202DE9F84342
:10DF50002E4C236823B940F668012D48F8F7A6FD3A
:10DF6000FEF778FB2368013B236024682CB1002472
:10DF7000FEF790FB2046BDE8F883264B1B68002B7C
:10DF8000F5D0254D254EDFF8A8801FE0EB6801276E
:10DF9000DC6804F1040904F1180000F074FF48463D
:10DFA00000F071FF1420E26A316807FA02F30B43B4
:10DFB00000FB02804946336000F042FF184BE26AE2
:10DFC0001B68DB6A9A4201D3164B1F602B68002B3B
:10DFD000DCD10CB1FFF74AFC134D2C6844B101278A
:10DFE000104EFFF723FF00B13760013CF9D12C60E0
:10DFF0000C4B1B68002BBAD04FF080520B4B1A60B1
:10E00000BFF34F8FBFF36F8F0124B1E7244E002081
:10E010003FD70108184E0020644E00202C4E0020EF
:10E02000A84D0020A84E0020204E002004ED00E066
:10E03000B44D002038B50C46054620B940F2CA411F
:10E040001848F8F733FD24B940F2CB411548F8F7EA
:10E050002DFD154B1B6823B140F2CC411148F8F758
:10E0600025FDFFF7C7FE114B2A68186814192CBF4D
:10E070000121002182422C600CD961B9FFF766FFB3
:10E0800038B94FF080520A4B1A60BFF34F8FBFF37D
:10E090006F8F38BD09B9A042F0D20021201AFFF7D6
:10E0A00013FCEBE73FD70108244E0020A44E0020CC
:10E0B00004ED00E010B5044640B94FF080520D4B1E
:10E0C0001A60BFF34F8FBFF36F8F10BD0A4B1B68F1
:10E0D00023B14FF4A4610948F8F7E8FCFFF78AFE82
:10E0E00000212046FFF7F0FBFFF730FF0028E4D0C7
:10E0F000EBE700BF04ED00E0244E00203FD701080D
:10E10000224B70B51A68224B12B101221A6070BD01
:10E11000204E1A6033681B6B1A68B2F1A53F0BD111
:10E120005A68B2F1A53F07D19A68B2F1A53F03D171
:10E13000DB68B3F1A53F04D0306831683431F8F7BB
:10E1400081FC154B1C68B4FA84F41423E4B2C4F1C6
:10E150001F046343114DEB5823B940F68831104832
:10E16000F8F7A4FC142202FB04F3E918486808330A
:10E1700040682B44984202FB045408BF436848603F
:10E1800008BF4B606368DB683360C0E7244E002043
:10E19000A84E0020A84D00202C4E0020B44D002099
:10E1A0003FD7010870B504462A4EFEF753FA04B96A
:10E1B0003468251D284600F066FE60B91421E06A27
:10E1C000254B41435B5833B90122244982400B68F7
:10E1D00023EA02030B60A36A1BB104F1180000F0EC
:10E1E00052FE29461E4800F02BFE94F858301D4D73
:10E1F000012B04BF002384F85830FEF74BFA2A683D
:10E200002AB1FEF727FAFFF731FBFEF743FA33682E
:10E21000A34211D12B6883B1134B1B6823B14FF478
:10E22000D9611248F8F742FC4FF08052104B1A6047
:10E23000BFF34F8FBFF36F8F70BD094A11680D4A4E
:10E240001268914201D13360F6E7BDE87040FFF7F4
:10E2500057BF00BFA84D0020B44D00202C4E002019
:10E260007C4E0020784E0020244E00203FD701082D
:10E2700004ED00E0184E002038B50D46044620B9E4
:10E2800040F69F310748F8F711FC074B2046196804
:10E29000183100F0E1FD2846BDE838400121FFF7C4
:10E2A00013BB00BF3FD70108A84D002070B50E4634
:10E2B0001446054620B940F6CA310A48F8F7F6FB7D
:10E2C000094B28461968183100F0BAFD002C214688
:10E2D00008BF3046BDE8704018BF4FF0FF30FFF771
:10E2E000F3BA00BF3FD70108A84D002038B5C36876
:10E2F000DC6824B940F6FA311548F8F7D7FB04F189
:10E300001805284600F0BFFD124B1B68E3B9251D18
:10E31000284600F0B8FD01230F49E26A08689340DF
:10E32000034314200B6029460C4B00FB023000F025
:10E3300087FD0B4BE26A1B68DB6A9A4285BF0120AE
:10E34000084B0020186038BD29460748EFE700BF9A
:10E350003FD70108244E00202C4E0020B44D002051
:10E36000A84D0020A84E0020644E002010B50446A1
:10E3700020B940F64F410748F8F798FBFEF76AF9D5
:10E38000054B1B682360054B1B686360BDE81040AC
:10E39000FEF780B93FD70108604E0020A44E002050
:10E3A000034B1B680360034B1B684360704700BF4F
:10E3B000604E0020A44E002070B50C46054620B9E2
:10E3C00040F665411448F8F771FB24B940F6664100
:10E3D0001148F8F76BFBFEF73DF9104B19682368FD
:10E3E0005A1C10D00E482E6800686A68864201D018
:10E3F0008A420FD9881A83420AD95B1A13442360D0
:10E400002846FFF7CDFF0024FEF744F9204670BDF3
:10E41000002323600124F7E73FD70108A44E002022
:10E42000604E00200122014B1A607047A84E002068
:10E4300070B50C461646054608B91B4A156805F125
:10E4400034026260EA6A052B22612A6B2560E26170
:10E450006A6CA260EA6C62614FF00002A26119D09E
:10E4600011490968A94209D12273D6B10023296B49
:10E47000CA5CA52A13D09B08238470BD032B237389
:10E48000F3D1FFF7B7FCAB6A0BB102232373FFF79D
:10E490005DFDEAE72846FFF7EBFB2073E5E7013374
:10E4A000E6E72684E9E700BFA84D00202DE9F84FF4
:10E4B0000D6881460C4692461DB300254FF0240B93
:10E4C0004B6801F108065B68B3424B6004BFCB6840
:10E4D0004B604B68D3F80C8063680BFB05915B685D
:10E4E00001229E42636008BF736805F1010508BF01
:10E4F00063606368DF6853463846FFF799FFB845A5
:10E50000EAD12846BDE8F88F2DE9F04706461746C0
:10E51000FFF770FC1E4B1B688B4237D80525002483
:10E520004FF0140A4FF02408DFF87890013D08FB03
:10E53000046001220AFB0591FFF7B8FF0444002D97
:10E54000F4D1144B0222196808FB0460FFF7AEFFF8
:10E55000114B04441968022208FB0460FFF7A6FF70
:10E56000044404220D4908FB0460FFF79FFF0444A4
:10E5700008FB046003220A49FFF798FF044407B12F
:10E580003D60FFF7E3FC2046BDE8F0870024F8E794
:10E59000184E0020AC4D0020B04D0020904E0020C1
:10E5A0007C4E0020B44D002008B9064B1868026B61
:10E5B0000020135CA52B02D0C0F38F007047013000
:10E5C000F7E700BFA84D0020014B1868704700BF57
:10E5D000A84D0020054B1B6833B1054B1B68002B71
:10E5E0000CBF02200020704701207047784E0020A9
:10E5F000244E00202DE9F0410446002836D0234A5D
:10E60000C36A11681746C96A8B4237D214268269D9
:10E610001F4D002AA8BF3A6806FB0353A2BFD26A67
:10E62000C2F10502826142699A4221D100F10408D7
:10E63000404600F028FC174B48B9E06A4643AA5907
:10E640002AB901211A68814022EA01021A603A6857
:10E650001968D26AE262012404FA02F008431860E1
:10E660001420414600FB025000F0EAFB204603E084
:10E670003B68DB6AC3620120BDE8F0811368C06CAF
:10E68000DC6AA0422CBF00200120F5E7A84D002045
:10E69000B44D00202C4E0020F8B5044608B90020E7
:10E6A000F8BD1F4B1B68834204D040F67A711D48A9
:10E6B000F8F7FCF9236D23B940F67B711948F8F798
:10E6C000F5F9236DE16AE26C013B91422365E6D0E6
:10E6D000002BE4D1251D284600F0D5FB124E134A2D
:10E6E00050B91421E76A794373582BB90120136894
:10E6F000B84023EA00031360E36CC3F10501A16194
:10E70000E3620124116804FA03F008431060142046
:10E71000294600FB036000F093FB2046C0E700BFE2
:10E72000A84D00203FD70108B44D00202C4E0020FA
:10E73000F8B50D460446002845D0036D23B940F6D0
:10E74000C9712148F8F7B2F9E36C9D4238BF1D4604
:10E75000E36AAB4237D0236D012B34D11B4B1B68CE
:10E76000A34204D140F6E4711748F8F79FF9142644
:10E77000A269E36A002AE562A4BFC5F10505A561A7
:10E78000134D626906FB03539A421CD1271D38467C
:10E7900000F079FBE26A0F4C40B95643AB592BB9F4
:10E7A00001212368914023EA0103236001231420FF
:10E7B000216893400B432360394600FB0250BDE8BB
:10E7C000F84000F03DBBF8BD3FD70108A84D002040
:10E7D000B44D00202C4E0020044B1A681AB1196861
:10E7E0000A6D01320A651868704700BFA84D002005
:10E7F0002DE9F0411E4C1E4680460F461546FDF79A
:10E8000029FF236893F85830022B14D00121236884
:10E810005A6D22EA08025A65236883F8581056B1E7
:10E820003046FFF751F84FF08052124B1A60BFF399
:10E830004F8FBFF36F8FFDF72DFFFDF70BFF15B166
:10E8400023685B6D2B602368002293F85830022BFD
:10E8500009BF012500252368596D04BFB9435965D7
:10E86000236883F85820FDF715FF2846BDE8F0819E
:10E87000A84D002004ED00E0F8B50E4617461D46F1
:10E88000044620B941F219212B48F8F70FF9FDF79A
:10E89000E1FE0DB1636D2B60022394F8585084F8AB
:10E8A0005830EDB2042F16D8DFE807F00A03070549
:10E8B0001100636D1E43666502E0636D013363659D
:10E8C000012D11D00124FDF7E5FE2046F8BD022DF3
:10E8D000F1D10024F7E7636D0133F1D041F24A2111
:10E8E0001548F8F7E3F8EBE7261D304600F0CBFAC1
:10E8F0001420124AE36A11689D400D431560104AC6
:10E90000314600FB032000F09BFAA36A23B141F2D9
:10E9100059210948F8F7CAF80A4BE26A1B68DB6A12
:10E920009A42CFD94FF08052074B1A60BFF34F8FF6
:10E93000BFF36F8FC6E700BF3FD701082C4E002002
:10E94000B44D0020A84D002004ED00E02DE9F8436F
:10E95000DDF820800E4691461D46044620B941F25E
:10E960008C213548F8F7A2F8FDF74CFFEFF311873B
:10E970004FF0500383F31188BFF36F8FBFF34F8FB6
:10E980000DB1636D2B60022394F8585084F8583011
:10E99000EDB2B9F1040F16D8DFE809F00A03070554
:10E9A0001100636D1E43666502E0636D01336365AC
:10E9B000012D11D0012087F31188BDE8F883022DC5
:10E9C000F1D10020F7E7636D0133F1D041F2CF219F
:10E9D0001948F8F76BF8EBE7A36A23B141F2DA21A3
:10E9E0001548F8F763F8154B1B6803BB251D28462F
:10E9F00000F049FA01231249E26A08689340034390
:10EA000014200B6029460F4B00FB023000F018FA6F
:10EA10000D4BE26A1B68DB6A9A42CBD90123B8F13D
:10EA2000000F01D0C8F80030084A1360C2E704F1B3
:10EA300018010748EAE700BF3FD70108244E00202D
:10EA40002C4E0020B44D0020A84D0020A84E0020E0
:10EA5000644E002038B5054608B9084B1D680024EF
:10EA6000FDF7F8FD95F85830022B04BF85F85840A3
:10EA70000124FDF70FFE204638BD00BFA84D002041
:10EA8000F8B50F4CFDF7E6FD2568ADB90D4F0E4EFC
:10EA9000384600F0C7F9304600F0C4F90B4B2A465F
:10EAA0001F600B4B0C210A201E60FEF7A9F82060A6
:10EAB00010B10849FEF768FCBDE8F840FDF7EABD73
:10EAC000E04E0020B44E0020C84E0020AC4E002086
:10EAD000B04E002088D70108914208B5416000611E
:10EAE0000AD8D21A83699A420DD2084B011D1868C0
:10EAF00000F0B2F9002008BD9A4201D2994202D238
:10EB0000011D034BF3E70120F5E700BFB04E0020E5
:10EB1000AC4E002007B5FFF7B3FF0C4B1B6843B9A1
:10EB20000B484FF48971F7F7C1FF002003B05DF87F
:10EB300004FB084BC82201930123074900930748AF
:10EB40000023FEF73DFF0028EAD0EFE7E04E00206B
:10EB50008DD70108E44E0020D2D7010879EC0008D7
:10EB60002DE9F04180462C200D4617461E46FDF744
:10EB7000ADFE044688B125B94FF4B6710848F7F7E1
:10EB800095FFFFF77DFF069BC4F80080C4E9065798
:10EB900026626362201D00F050F92046BDE8F08136
:10EBA0008DD701082DE9FF410D4690461F460646C8
:10EBB00020B94FF4C3710F48F7F778FF0E4C206867
:10EBC00078B1052DCDE9015803960DDCFFF702FD64
:10EBD000002302280CBF0A9A1A4601A92068FEF7F2
:10EBE00033F804B0BDE8F08100233A4601A9FEF7EE
:10EBF000E1F8F6E78DD70108E04E00202DE9F74354
:10EC000000271A4DDFF86C802B681A6832B9184A51
:10EC100011681360296003B0BDE8F083DB68DC682D
:10EC20001E6804F10409484600F02DF9636A204685
:10EC30009847E369012BE7D1A36933449E4206D28A
:10EC4000636024614946286800F006F9DCE7002388
:10EC50000097324619462046FFF7A4FF0028D3D17B
:10EC600040F272314046F7F721FFCDE7AC4E00206D
:10EC7000B04E00208DD701082DE9F04F4FF001086C
:10EC8000624D87B0DFF898B1DBF80020136843B31A
:10EC90000024D368D3F80090FFF7ACF8FFF7B2F880
:10ECA0005B4B82461A681F4690425A4E1CD318602E
:10ECB000002C4BD0584B1B681A68B2FA82F25209EA
:10ECC000A9EB0A013068FEF79BFBFFF73FF990B90B
:10ECD0004FF08052514B1A60BFF34F8FBFF36F8FCD
:10ECE00009E001249946D7E7FFF788FF484BC3F8AE
:10ECF00000A0FFF72BF9002203A93068FEF7FEF809
:10ED00000028BFD0039B002BF5DB059C636913B182
:10ED1000201D00F0B8F8FFF775F83B68814698426F
:10ED200001D2FFF76BFF039BC7F80090092BE2D8D5
:10ED300008FA03F313F4047A57D113F0C70F33D151
:10ED40009B06D8D52046FDF74DFED4E7814529D84E
:10ED5000FFF7FCF8DBF80030DB68D3F80CB00BF100
:10ED6000040000F090F8DBF81C30012B15D1DBF823
:10ED700018104B46524649445846FFF7ADFE60B165
:10ED8000009423464A4621465846FFF70BFF20B918
:10ED90004FF4F4712846F7F789FEDBF82430584623
:10EDA0009847A8E722468BE7A169049B4A46194485
:10EDB0002046FFF791FE00289DD0636A20469847C1
:10EDC000E369012B97D1A2690499CDF800A00A4408
:10EDD000534651462046FFF7E5FE00288BD140F20E
:10EDE00001312846F7F762FE85E7049BA36123B94A
:10EDF0004FF446712846F7F759FEA1694B464A463B
:10EE000049442046FFF768FE75E700BF8DD701082B
:10EE1000DC4E0020E04E0020B04E002004ED00E06B
:10EE2000AC4E00204FF0FF3200F108034360C0E910
:10EE300002230361002303607047002303617047CE
:10EE400043689A684B608A609A6851609960036869
:10EE500008610133036070470A6830B5531C0AD15A
:10EE600003695A684A6091608B6059600368086161
:10EE70000133036030BD00F108035C6825689542EA
:10EE8000EFD82346F9E70369D0E901128A6051609F
:10EE90005968814208BF5A60002202611A68013A2B
:10EEA0001A60186870470000021C18BF0122002178
:10EEB0000148F8F7A9BB00BF00040240F8F7F0BF13
:10EEC00038B505460C460020FFF7EEFF45F0800000
:10EED000FFF7F4FF2046FFF7F1FFBDE838400120BF
:10EEE000FFF7E2BF08B50120F8F780F90A20F8F72C
:10EEF0007DF90B20F8F77AF90720F8F777F9052064
:10EF0000F8F774F9BDE808400420F8F76FB900007D
:10EF1000204B70B59D780446EDB958B902211E48C2
:10EF2000F8F76CFB23461A460221BDE870401A48E8
:10EF3000F8F79CBA012805D102211748F8F758FBC9
:10EF40002B46F0E7022823D102460146BDE8704077
:10EF50001148F8F7C9BA012D14D138B904210E4867
:10EF6000F8F74CFB002304211A46DEE7012804D100
:10EF700004210948F8F73CFBF4E7022808D10246CF
:10EF80000421E3E76A21BDE870400448F7F78EBD2D
:10EF900070BD00BFE84E002000000240DAD7010833
:10EFA00008B50020FFF7B4FFF8F762F80120FFF77B
:10EFB000AFFFF8F75DF80220FFF7AAFFBDE80840B1
:10EFC000F8F756B808B500210120F8F7E9FE01204E
:10EFD000FFF76AFF0023094819461A46F8F746FA70
:10EFE000B5214020FFF76CFFA0214120FFF768FF0B
:10EFF000BDE8084000210120FFF762BF0004024085
:10F0000010B5FFF76FFF0120FFF74EFF00233A48CE
:10F010001A461946394CF8F729FA00210120F8F769
:10F02000BFFE22787AB1002306211A463248F8F74B
:10F030001DFA06213048F8F7DBFAF8F719F819211C
:10F040005820FFF73DFFFFF7ABFFFFF7BBFF6378EB
:10F050005BB1002304211A462948F8F707FA002378
:10F060000D211A462748F8F701FA0022012122480B
:10F07000F8F73AFA00220A211F48F8F735FA002279
:10F080000B211D48F8F730FA002207211A48F8F73B
:10F090002BFA002205211848F8F726FA002204214D
:10F0A0001548F8F721FA0523022201211248F8F742
:10F0B000BBF8052302220A210F48F8F7B5F805230B
:10F0C00002220B210C48F8F7AFF805230222072192
:10F0D0000948F8F7A9F80523022219460648F8F767
:10F0E000A3F8094B1B782BB9BDE81040BE21074897
:10F0F000F7F7DCBC10BD00BF00040240E84E002062
:10F100000000024000080240EB4E0020DAD7010860
:10F1100082B00190064B9DF80620BDF804109A704D
:10F1200001221980034B1A7002B0FFF769BF00BFBC
:10F13000E84E0020EB4E00201A4B10B55B78D3B19F
:10F140000128194C18D104211848F8F751FA0D215B
:10F150001748F8F753FA23786BB1002304211A46B5
:10F160001248F8F783F900230D211A461048F8F7E2
:10F170007DF90023237010BD40B904210B48F8F736
:10F180003DFA0D210A48F8F733FAE4E70222042198
:10F190000648F8F7A9F902220D210548F8F7A4F965
:10F1A0000123E7E7E84E0020AC0000200000024009
:10F1B0000008024008B5FFF795FEFFF7F1FEFFF7E4
:10F1C00001FFF8F749FE012200211F48F8F78CF9EA
:10F1D0000220FFF7B1FF0220FFF79AFE0222012171
:10F1E0001948F8F781F902220A211748F8F77CF943
:10F1F00002220B211448F8F777F90222072112485E
:10F20000F8F772F9022205210F48F8F76DF902228A
:10F2100004210D48F8F768F90C4B1B781BB9E22163
:10F220000B48F7F743FC0B4B1B785BB1002306211F
:10F230001A460548F8F71AF9BDE8084006210248C1
:10F24000F8F7DCB908BD00BF00040240EB4E002017
:10F25000DAD70108E84E002010B5064C02222046FD
:10F260000021F8F741F92046BDE8104002220121B3
:10F27000F8F73AB900140240014BDB68184700BFA9
:10F28000EC4E00200120704701B1096818B1806A76
:10F29000431A58425841704710B5044618B9D22154
:10F2A0000748F7F703FC074B5B689847D4E9062348
:10F2B000904271EB0304B4BF101A002010BD00BFD0
:10F2C00059DC0108EC4E00202DE9F0418846044647
:10F2D00010B10369012B03D1E7211648F7F7E6FBCC
:10F2E000D4E9062352EA030122D0D4E90867901B2F
:10F2F00063EB070108F066FA05462069013808F05B
:10F3000047FA0146284608F04FFB0546404608F0FC
:10F310003FFA294608F094FA294608F087F908F0E0
:10F320007BFC321847F1000310461946C4E9060178
:10F33000BDE8F08159DC010838B50C4B054618686A
:10F3400000F0E3FB10B90023184638BD4FF47A747F
:10F3500003686C431A68A242F6D000F0CDFB002887
:10F36000F1D003681A689442F6E700BFEC4E002023
:10F3700041F65832A0F55223A3F61833934224D80D
:10F38000A0F55423A3F1F902622A1ED96FF4547236
:10F390009A18C62A19D9A3F21353302B15D9104B3A
:10F3A000984214D903F6B833984212D903F516736C
:10F3B000984210D903F5167398420ED903F5E173FC
:10F3C00098428CBF0620052070470020704701201E
:10F3D000704702207047032070470420704700BF29
:10F3E000E8320D00F8B5054618B9F3212148F7F7C2
:10F3F0005DFB214F386800F088FB002838D0002DD5
:10F4000036D003681A79AA422ED11E7B00F074FB15
:10F4100008BB6EB3062D03D940211648F7F746FB0B
:10F42000164B53F835400CBBFE211248F7F73EFB54
:10F430003868744300F069FB0646C8B107683B7939
:10F44000AB4204D121463846FFF73EFF3C613046CF
:10F4500000F052FBF0E703681A79AA42D6D11B7B71
:10F46000002BD3D00136D1E70026CFE7012CDFD126
:10F47000F8BD00BF59DC0108EC4E002020D801087F
:10F480002DE9F04F044687B058B3254B00681D693D
:10F4900008F07EF907F064FD1FA3D3E9002307F00D
:10F4A000E1FE227B06460F462379D4F82890D4F853
:10F4B0001080D4F808A0BAB1062B98BF194A20468C
:10F4C00094BF52F823B0DFF868B0FFF7E5FE32468C
:10F4D0003B46CDE90198CDE903A01348CDF800B033
:10F4E000A84707B0BDE8F08F062B98BF0D4A20460D
:10F4F00094BF52F823B0DFF838B0FFF7CDFECDE966
:10F500000189CDE903A0CDF800B032463B4607485B
:10F51000E6E700BFAFF300800000000080842E41CA
:10F52000EC4E002058D8010840DB010895DB0108AB
:10F5300032DB010810B5104C206820B923690F4850
:10F54000BDE81040184700F0E9FA2369014660B1B0
:10F550000B489847206800F0D8FA044638B920468E
:10F5600000F0CAFA044610B910BD0648E8E7206862
:10F57000FFF786FFF3E700BFEC4E0020B4DA010886
:10F58000D2DA01080CDB0108F8B5134D06462B7ED4
:10F590000F4623B94FF4B1711048F7F787FA2C687A
:10F5A00024B96B690E4898472046F8BD0D4B20469C
:10F5B000002E08BF1E4600F0A8FA054608B9002430
:10F5C000F2E7046839462046B0470028ECD12846C7
:10F5D00000F092FAF1E700BFEC4E002059DC010880
:10F5E00075DA010885F200082DE9F04F3E4D91B023
:10F5F0002B7E83468946924623B94FF4C9713B4816
:10F60000F7F754FA2C6834B96B69394898472046A3
:10F6100011B0BDE8F08F374B2046B9F1000F08BF9D
:10F62000994600F072FA064620B96B69324898474D
:10F630003446ECE70468237BF3B94FF0FF3700242E
:10F640004FF00008304600F057FA064608BBBAF102
:10F65000000F01D0CAF80070002FD8D1B8F1010F07
:10F66000D5D908F1FF313846FBF724F810AB03EB8E
:10F67000800050F8404CCAE7A3685B45DDDB002101
:10F680002046C8470028D8D02046FFF705FE074689
:10F69000D6E735682B7B002BD4D0AB685B45D1DB3C
:10F6A00000212846C8470028CCD02846FFF7F4FDA3
:10F6B00048B9B8F10F0F9FBF10AB03EB880343F8B5
:10F6C000405C08F101086CB187420AD8BAD1D4E98C
:10F6D0000823D5E90801FAF7FDFD002818BF2C46DC
:10F6E000B0E707462C46ADE7EC4E002059DC010898
:10F6F00075DA010885F2000899DA010800000000B7
:10F700002DE9FF478946044620B940F2E111284817
:10F71000F7F7CCF9236923B94FF4F1712448F7F7CF
:10F72000C5F9DFF894A00027DAF804309847C4E957
:10F73000080105462069884608F02AF8494608F07D
:10F740007FF8494607F072FF07F00AFC16A3D3E9D9
:10F75000002307F087FD07F04FF907F0F3FE2D189F
:10F7600048EB0703C4E906530646206808F010F882
:10F7700007F0F6FB0CA3D3E9002307F073FD044662
:10F7800048460D46CDE9026707F0EAFB2246CDE97F
:10F7900000012B46DAF810100648884704B0BDE88F
:10F7A000F047FFF7C7BE00BF0000000080842E4175
:10F7B00059DC010874D80108EC4E002008B5FFF7A9
:10F7C000D7FD003018BF012008BD000038B50D4D31
:10F7D00004462A7E22B94FF407710B48F7F766F901
:10F7E00074B1237B63B1002320792373FFF7FAFD03
:10F7F0002B69064898472046BDE83840FFF740BED1
:10F8000038BD00BFEC4E002059DC010844DA010885
:10F8100038B50D4D04462A7E22B94FF40A710B48C3
:10F82000F7F744F974B1237B63B90123207923737B
:10F83000FFF7D8FD2B69064898472046BDE83840B9
:10F84000FFF71EBE38BD00BFEC4E002059DC01089A
:10F850005DDA0108F8B5194D06462B7E23B94FF441
:10F860000D711748F7F722F92C6824B96B69154810
:10F870009847204601E00EB90020F8BD204600F070
:10F8800044F904460028F7D023689E420CD137790A
:10F890003046FFF7F1FC2146286800F04DF9384664
:10F8A000FFF7A0FD0120E8E7204600F025F9044617
:10F8B0000028E9D16B690448DAE700BFEC4E00206C
:10F8C00059DC010811DC010833DC01082DE9F8439B
:10F8D000384D06462B7E8846914623B940F2F911F1
:10F8E0003548F7F7E3F83046FFF768FF044630B9CC
:10F8F0006B693146314898472046BDE8F883304669
:10F90000FFF71AFD044630B12D482B693146984760
:10F910002046FFF79FFF2B7E1BB976212648F7F77D
:10F92000C5F8AB6830209847044640B96B69254854
:10F9300098476B693146244898470024DCE7302219
:10F94000002108F099FC3046FFF712FD07462071B0
:10F9500038B9EB68204698476B6931461B48984791
:10F96000E7E7062803D940211348F7F79FF8184B1B
:10F97000214603EBC70253F83730526823614FF436
:10F980007A73A2605E4300220023C4E906230123A8
:10F9900026602373C4E90A89286800F097F8207963
:10F9A000FFF720FD2B690B4898472046FFF768FDBD
:10F9B000A2E700BFEC4E002059DC01082CD9010859
:10F9C00063D9010898D9010809DA0108C6D90108E4
:10F9D00020D80108F1D9010870B50F4C0546237EE7
:10F9E00023B94FF41C710D48F7F760F823685BB139
:10F9F0000B4E29463046FFF7C7FD50B9236929460B
:10FA0000BDE870400748184763690748BDE8704083
:10FA10001847FFF731FCECE7EC4E002059DC0108F9
:10FA200089F20008EBDB010811DC0108014B187EAC
:10FA3000704700BFEC4E002084B070B504AC84E881
:10FA40000F00154B1A7E1C462AB1BDE870405B6959
:10FA5000124804B018471D1D04AE0FCE0FC5336801
:10FA60002B600BB90E4B636123690BB90C4B2361FF
:10FA7000E3680BB1A36833B923690A4898470A4B76
:10FA8000E3600A4BA36000F013F8012320602376A3
:10FA9000BDE8704004B07047EC4E0020B8D80108B3
:10FAA00031A40008F1D80108E1810108D1810108E1
:10FAB00010B50820FAF75CFD0446FEF79BF9002319
:10FAC000C4E90034FEF742FA204610BD70B5054681
:10FAD0000C200E46FAF74CFD044660B10660FEF7B6
:10FAE00089F9002363606B68A3601C6004346C6058
:10FAF000FEF72CFA012070BD10B50446FEF77AF926
:10FB00006468FEF723FA204610BD10B50446FEF7E0
:10FB100071F92468FEF71AFA204610BD10B50446A4
:10FB2000FEF768F9236800241BB9FEF70FFA204698
:10FB300010BD01345B68F7E738B50C460546FEF7A3
:10FB400059F9D4E901324BB19A60A2681360FEF70B
:10FB5000FDF92046BDE83840FAF7F4BC6A60F4E7E6
:10FB600070B50446044E451814F8011B3046FAF7E8
:10FB700063FCAC42F8D170BDE9AF010870B5154621
:10FB80000022C0E901150270C0E90332C0E9052274
:10FB9000C0E907224262DDE90412044600F11C06B6
:10FBA00004F0DEF838B929460748FAF745FC2B215E
:10FBB0000648F6F77BFFDDE904233146204604F0D2
:10FBC000BCF8204670BD00BFFCAE010827AF01089D
:10FBD0002DE9F04100259DF81860C0E9011205707B
:10FBE000C0E90335C0E90555C0E90755456231460E
:10FBF0000446174600F11C0803F0B4FE38B9394634
:10FC00000748FAF719FC20210648F6F74FFF32465D
:10FC10004146204603F094FE2046BDE8F08100BF37
:10FC2000FCAE010827AF0108F8B50025C0E90112B4
:10FC30000570C0E90335C0E90555C0E907554562BF
:10FC400006990446164600F11C0703F08FFF38B9E9
:10FC500031460748FAF7F0FB20210648F6F726FF61
:10FC6000069A3946204603F06AFF2046F8BD00BFD9
:10FC7000FCAE010827AF010810B50446006810B1BA
:10FC8000012106F07BF8204610BD0000F0B50126EA
:10FC9000044608270D468DB0694B6A4A31460096E6
:10FCA00002A8FFF795FF02A9204605F061F902A816
:10FCB000F0F7E2FB644BCDE900571A4604210DEB47
:10FCC0000700FFF75BFF0DEB0701204605F050F939
:10FCD0000DEB0700F0F7D0FBEB195C4A019700939E
:10FCE00004215B4B0DEB0700FFF748FF0DEB07010D
:10FCF000204605F03DF90DEB07001027F0F7BCFB9F
:10FD0000EB190093534B04211A46019702A8FFF701
:10FD100035FF02A9204605F02BF9203502A8F0F79F
:10FD2000ABFB4D4B4D4A00950421019702A8FFF70C
:10FD300025FF02A9204605F01BF902A8F0F79CFB5D
:10FD40000C23474A00930221464B02A8FFF76CFFA1
:10FD500002A9204605F00CF902A8F0F78DFB424BF2
:10FD6000424A3146009602A8FFF732FF02A9204618
:10FD700005F0FEF802A8F0F77FFB032200230392B0
:10FD80003B4D3C4A3C4902A88DF808300495CDE92A
:10FD90000523CDE90733CDE909330B9303F0C8FF01
:10FDA00038B929463548FAF747FB20213448F6F799
:10FDB0007DFE0025304A09A902A803F081FF02A9AF
:10FDC000204605F0D5F802A8F0F756FB2D4B2E4A39
:10FDD0000095022102A8FFF727FF02A9204605F09F
:10FDE000C7F802A8F0F748FB284B294A00950221E2
:10FDF00002A8FFF719FF02A9204605F0B9F802A8EA
:10FE0000F0F73AFB0121234B234A009102A8FFF7A8
:10FE1000DFFE02A9204605F0ABF802A8F0F72CFBA4
:10FE20001E4B1F4A0095022102A8FFF7FDFE02A902
:10FE3000204605F09DF802A8F0F71EFB0DB0F0BDBE
:10FE40002FDD010815C9010842DD0108B3E00108F2
:10FE50009AE0010850DD0108BBE00108E5E0010877
:10FE60005CC8010857DD0108B0DD010898C8010829
:10FE700075C80108ECE0010818C90108FCAE0108CA
:10FE800027AF010801E101089CC801083FE1010812
:10FE9000C3C801087AE10108B4EF010896E101083E
:10FEA000EBC8010830B504468DB001467A4A684671
:10FEB00004F041FE794A214603A804F03CFE784A4A
:10FEC000214606A804F037FE7649204604F02AFEB3
:10FED00005467548FAF7B0FA0123039A02F11001BA
:10FEE000914205D011F8010D002818BF0023F7E753
:10FEF000002B53D06D48FAF79FFA5DB36C48FAF7C0
:10FF00009BFA6C4A214609A804F015FE6A48FAF7E4
:10FF100093FA08210098FFF723FE6848FAF78CFA55
:10FF200008210998FFF71CFE6548FAF785FA1021A9
:10FF30000698FFF715FE6348FAF77EFA0998069AC5
:10FF4000009900F059FE09A8FFF796FE5E48FAF7FF
:10FF500073FA61E05D48FAF76FFA5D48FAF76CFAF8
:10FF60000699009800F0A6FD5A48FAF765FA0421B0
:10FF700000980844FFF7F4FD5748FAF75DFA10219E
:10FF80005648FFF7EDFD5648FAF756FA1021554846
:10FF9000FFF7E6FD4B48FAF74FFAD7E7102206982D
:10FFA00008F034F95049514B002818BF1946504801
:10FFB000FAF742FA002D3DD03D48FAF73DFA3D4AA6
:10FFC000214609A804F0B7FD4A48FAF735FA082196
:10FFD0000098FFF7C5FD4848FAF72EFA082109985E
:10FFE000FFF7BEFD4548FAF727FA10210398FFF7FF
:10FFF000B7FD4348FAF720FA10210698FFF7B0FD45
:020000040801F1
:100000003048FAF719FA0998039B069A009900F00C
:1000100007FE09A8FFF730FE2A48FAF70DFA06A8EE
:10002000FFF72AFE03A8FFF727FE6846FFF724FE26
:100030000DB030BD2548FAF7FFF93248FAF7FCF960
:10004000039A0699009800F079FD2248FAF7F4F92E
:10005000042100980844FFF783FD2B48FAF7ECF9D8
:1000600010211E48FFF77CFD2848FAF7E5F910211A
:100070002748FFF775FD2748FAF7DEF910212648D3
:10008000FFF76EFD2548FAF7D7F916481021FFF75C
:1000900067FD0C485BE700BF42DD0108E5E00108B1
:1000A00050DD010815C90108E2DD0108F9DD01088C
:1000B00014DE0108B3E001081ADE01082BDE010896
:1000C0003DDE0108B3F00108E5DE01085DDE010850
:1000D00062DE010894DE0108A6DE01085801002056
:1000E000D2DE010888010020CBDD0108B4F0010850
:1000F00004DF010821DF010833DF010846DF0108C2
:1001000066DF0108AFDF0108E9DF010855E00108FB
:10011000680100206CE001087801002083E00108FC
:1001200010B5084CD4F82C211AB964210648F6F70A
:10013000BDFCD4F82C010023BDE81040032220218F
:10014000FEF79ABBB0000020F6E20108F0B51F46AA
:100150001446C7B005460E46F122002109A808F052
:100160008BF809AA1021384602F0D6F8204609F08B
:1001700009F807461022002101A808F07DF8102F89
:100180003A46214628BF102201A808F04DF809AAD6
:1001900005A901A802F03AF9324605A9284608F057
:1001A00043F847B0F0BD000038B50C4C0C4D94F846
:1001B0003230022B0ED1082394F8FF20D4F800111E
:1001C000012002F05FF86B6B00209847042384F84D
:1001D000303038BDEB6A98470123F8E7B0000020C3
:1001E00080D4010810B5044601F068F820B9204613
:1001F000BDE8104001F03AB810BD0000054B93F87F
:10020000212022B993F8350080F0010070470020CA
:10021000704700BFB0000020F0B570279DB00646C3
:100220000D463A460021684608F026F808212B467C
:100230000DEB010004AC0B4AFFF788FF2B4620466C
:10024000094A102108ADFFF781FF94E80F0085E807
:100250000F003A466946304607F0E6FF30461DB0CB
:10026000F0BD00BFE7E20108EFE2010808B505486C
:10027000FAF7E2F8044A92F80431013382F80431C3
:1002800008BD00BF8BE20108B00000200022024B35
:1002900083F80421704700BFB000002084B070B51F
:1002A0008AB00EAC84E80F00744C4FF49C72254663
:1002B000002120460EAE07F0DFFF0FCE0FC596E8F7
:1002C000030014AE85E803000FCE04F118050FC536
:1002D00033682B600E9B0BB9694B23600F9B0BB9E6
:1002E000674B2360109B23B940F26D116548F6F708
:1002F000DDFB129B23B940F271116248F6F7D6FB81
:10030000119B23B940F275115E48F6F7CFFB139BA2
:1003100023B940F279115B48F6F7C8FBA3690BB922
:100320000323A361E3690BB90A23E36194F8233043
:1003300013B9012384F8233001F03EFD94F82430F2
:1003400013B9012384F8243001F02EFDA36A0BB900
:100350004D4BA36201F01CFDFAF772FBC4F82801B3
:100360000138033004D963684848984700207CE08E
:10037000032200210120FCF743FCC4F8300120B91E
:100380004FF4D1713F48F6F791FB00220421E06958
:10039000FCF736FC606420B94FF4D3713948F6F7A6
:1003A00085FB00220421E069FCF72AFCA06420B947
:1003B00040F2A9113348F6F779FB0022042101200D
:1003C000FCF71EFCE06420B94FF4D6712D48F6F717
:1003D0006DFB4FF48163A4F80A31002384F83630B2
:1003E000012384F80E31FFF721FB05AD68B9A3683E
:1003F00022690593236807920893E268636806926E
:10040000009395E80F00FFF717FB01F0FBFC236852
:100410001F4E079363680496089323690693E36865
:10042000059306F1A003039303AB93E803008DE863
:100430000300DC3695E80F0002F074F90196A36919
:100440004FF4CD720093134901231348FDF7B8FA16
:10045000012805460ED1002303220421D4F82C01E3
:10046000FEF70AFA284684F834500AB0BDE8704016
:1004700004B070476368094877E700BFB000002008
:1004800031A40008F6E2010808E6D333E5E10108EB
:100490000001002018E20108F905010820E2010826
:1004A00010B50F4CD4F82C3123B940F2D9110D48B6
:1004B000F6F7FCFA002303220421D4F82C01FEF7FE
:1004C000DBF942F21071D4F83001FCF7A9FD0023EA
:1004D000D4F830011A46BDE810401946FCF7B4BB09
:1004E000B0000020F6E2010838B50E4DD5F83031E5
:1004F00023B94FF4F5710C48F6F7D8FA0021D5F876
:100500003001FCF78DFD0128044608D10023D5F801
:1005100030011A461946FCF797FB204638BD0020EB
:10052000FCE700BFB0000020F6E2010810B5FFF7BD
:10053000DBFF68B1074C0023D4F82C01032208210B
:10054000FEF79AF9D4F82C01BDE81040FDF7D0BBB6
:1005500010BD00BFB0000020014BD863704700BF42
:10056000B0000020002307B50193054B024601A906
:10057000D86CFCF7C3FC019803B05DF804FB00BF26
:10058000B000002038B5FFF7AFFF184D044620B18A
:100590006B6817489847002038BD686CFCF7CEFEA2
:1005A000EB698342F7D32146204602F0EBF805467B
:1005B0000028F0D0047000F047FE044618B9284621
:1005C00002F018F9E7E70B4A1368013313605BB9CF
:1005D000136801331360636040F2031320462380E5
:1005E000FFF700FE6068D7E71368F4E7B00000206B
:1005F00050E20108084F002001232DE9F0415F4C33
:10060000DFF880815E4E84F830300A235D4A4FF077
:10061000FF310020FEF7ECF8012867D1D8F8000080
:1006200043071AD5337833B1FAF758F90020FAF7AF
:10063000A9F900233370FCF70DF8FCF72BF802231F
:1006400084F830300023D4F830011A461946FCF7FC
:10065000FBFA0020FDF7A6FDD7E710F0080521D032
:1006600033787BB941F28830FAF764F918B9A021E0
:100670004548F6F71BFA4548FAF784F90123337029
:10068000FFF792FD0020FEF7E5F94FF4FA61D4F888
:100690003001FCF7C5FC0028B7D1A7213A48F6F78E
:1006A00005FAB2E710F020003FD03378DBB194F8C0
:1006B0003030042B17D1364F2A463946D4F828015A
:1006C000FCF75EFD01280ED13B78072B21D128468F
:1006D00000F0BAFD38B140F20512C0E901550561DC
:1006E0000280FFF77FFD0020FEF7B4F93378002B7E
:1006F0008BD000F0FBFD0546002886D0032384F84C
:1007000030300378052B35D8DFE803F01219192AA9
:100710002A312A463946D4F82801FCF7EFFB012894
:10072000E1D13846FAF734F9DDE7FEF793F96CE7E3
:10073000D6211548F6F7BAF9FFF736FD65E7FFF75A
:100740005DFD38B9284600F08BFA60B1284600F00C
:100750008DFDF1E72846FFF745FDFFF713FFEBE7B7
:1007600001F058F9F1E72846FFF73CFDE4E700F017
:100770003BFDEBE7636807489847E7E7B0000020D8
:100780000C4F00201C4F0020F6E201082101010857
:10079000104F0020C5E10108024B93F8FC0001F066
:1007A000E7BC00BFB0000020F0B585B007460C469E
:1007B0001546ADF80430FFF797FE404E28B1736838
:1007C0003F489847002005B0F0BD706CFCF7B6FDBF
:1007D000F3698342F6D3FFF7DFFF8442F2D8002D9E
:1007E00047D1002CEED12146384601F0CBFF04461C
:1007F0000028E7D09DF80530002B3DD0042303707E
:10080000FFF734FD9DF804303BB10D23012203A90D
:1008100020468DF80C3000F0A5FE96F8312096F8B1
:100820003230934203D196F83330934217D02023CD
:10083000022A18BF00228DF80C3094F8783003A9F2
:100840000BBF43F0040343F001038DF80D208DF836
:100850000D20204684F87830022200F083FE657770
:10086000204600F0F1FC054648B9204601F0C2FFE1
:10087000A8E7DF2DA6D8B6E702230370C2E700235E
:10088000104A836013680133136093B9136801330E
:1008900013606B600A9B28462B6140F201132B808A
:1008A00000F0F6FC38B9284600F0E0FC7368064812
:1008B00087E71368EDE7686885E700BFB0000020B0
:1008C00050E20108084F0020BFE20108082808BFD5
:1008D0000120034B83F8230083F8FC00704700BF1E
:1008E000B0000020024B83F8240083F8FD0070471D
:1008F000B000002008B5F9F787FE014B586508BD28
:10090000B0000020034630B5054C00F1100522462A
:1009100018685968083303C2AB421446F7D130BD9A
:1009200078010020034630B5054C00F11005224641
:1009300018685968083303C2AB421446F7D130BD7A
:1009400068010020034630B5054C00F11005224631
:1009500018685968083303C2AB421446F7D130BD5A
:1009600058010020034630B5054C00F11005224621
:1009700018685968083303C2AB421446F7D130BD3A
:100980008801002010B50446FFF7BCFF2046FFF7A2
:10099000C9FF2046BDE81040FFF7D4BF30B5102591
:1009A000C3B0224CF122002105A807F065FC2A46BD
:1009B000002101A807F060FC94F8673005AA8DF8C3
:1009C000053094F8663029468DF8063094F8653085
:1009D00004F178008DF8073094F864308DF8083011
:1009E00094F863308DF8093094F862308DF80A304D
:1009F00094F861308DF80B3094F860308DF80C303D
:100A000001F08AFC052305AA04F1980101A88DF8DC
:100A1000043001F0FBFC062305AA04F1880101A8BB
:100A20008DF8043001F0F2FC43B030BDB00000207E
:100A30000246024B0068516803C37047080100205A
:100A40000246024B0068516803C370471001002042
:100A5000034630B5054C00F1100522461868596868
:100A6000083303C2AB421446F7D130BD1801002051
:100A7000034630B5054C00F1100522461868596848
:100A8000083303C2AB421446F7D130BD2801002021
:100A9000014B83F822007047B0000020014B83F81F
:100AA00031007047B0000020014B1864704700BF50
:100AB000B000002010B50430C6B00C46FFF71AFF96
:100AC0001C4B0DF1050203F10C0153F8040B8B4292
:100AD00042F8040BF9D11B881021138000238DF8F4
:100AE0001330022309AA20468DF8043001F014FCCB
:100AF00009AA05A901A801F089FC05A8FFF732FFA2
:100B0000012309AA102120468DF8043001F004FCCD
:100B100009AA05A901A801F079FC05A8FFF732FF91
:100B20004FF48872044B1A84102283F8502046B088
:100B300010BD00BF7CE20108B000002030B50430D9
:100B4000C7B00C461546FFF7D5FE294B0DF105023F
:100B500003F10C0153F8040B8B4242F8040BF9D15A
:100B60001B882046138000238DF8133002230124B4
:100B700009AA10218DF8043001F0CEFB09AA05A9BD
:100B800001A801F043FC05A8FFF7ECFE09AA10211B
:100B900028468DF8044001F0BFFB09AA05A901A869
:100BA00001F034FC05A8FFF7ADFE032309AA05A94F
:100BB00001A88DF8043001F029FC05A8FFF7B2FE6A
:100BC000042309AA0DEB030005A98DF8043001F0F8
:100BD0001DFC05A8FFF7B6FE40F21112054B1A8462
:100BE000112283F8084183F8502047B030BD00BF80
:100BF0007CE20108B000002038B50D461446FFF72E
:100C000017FF2846FFF71CFF2046FFF721FF20466D
:100C1000FFF72EFF1022014B1A8438BDB0000020D0
:100C200070B50E4615461C46FFF702FF3046FFF72B
:100C300007FF2846FFF70CFF2046FFF719FF112298
:100C4000024B1A84BDE87040FFF7A8BEB000002038
:100C500028B1836A012B01D1007B704700207047C7
:100C60002DE9F047044686B010B10378012B03D07C
:100C70001C217A48F5F71AFF63691BB91D217748D3
:100C8000F5F714FF63691B78042B05D0022B03D002
:100C90001E217248F5F70AFF0026714D03AA71491B
:100CA00095F8FD00D5E93F9A0396FEF79DFC0746AF
:100CB00040B9204600F07CFB4FF00108404606B0EA
:100CC000BDE8F087039B93B1FEF734FC0399042938
:100CD00005D9204600F0A4FB4FF00008EEE74FF4E2
:100CE0007A7361484843B0FBF3F0FDF7E3F9A3687A
:100CF0000133012BA3600FD1D5F8F03060690133C7
:100D0000C5F8F03095F80931013385F8093100F064
:100D1000E3FB606900F046FC6B6D66697360D5F8B3
:100D2000F030738195F80531002B65D0002385F8EC
:100D30000531337A43F00403337295F8FC303846BA
:100D400086F87C3001F0A0F886F87D00012160690A
:100D500000F0DAFB95F80E214FF47A7312F00F02CF
:100D600008BF012200265A4305AB019304AB009350
:100D7000394602F57A736069049600F051F98046AD
:100D8000002896D0FDF73EF8E060049870B1314637
:100D900000F0BAFBFFF77AFA049B1B78052B04BF1F
:100DA000012385F80531002385F80731049800F008
:100DB0006FFBDDE9040100F0DDFD049F77B13F7AB0
:100DC00017F0040703D0474695F80C31A360636918
:100DD0001B78022B02D195F80C31A36000F09CFA2D
:100DE0000646F0B98E211D48F5F760FE1F4B204ADC
:100DF0008F211A4807F0EAF8A6F87A309DE73146C5
:100E0000606898476420FDF755F9304600F094FA81
:100E100095F80C31A2689A42BFF450AF03233370A7
:100E20005AE780226169183007F0FEF90023049A1E
:100E3000C6F88030C6F8982022787372337095F81F
:100E40003530C6E9039A3375236972703772002B07
:100E5000D5D1304600F08AFADAE700BF44E3010852
:100E6000B0000020510C010840420F0081E301084E
:100E700036E301082DE9F04385B006460C468DF8AF
:100E80000F202BB101220DF10F010020FAF75CF9C0
:100E9000FCF7B8FF1C4B1D4DDFF878809DF80F1054
:100EA00007469B6A2046984741F288322946D8F87F
:100EB0002801FCF723F828B32B78012B1DD12846F5
:100EC000AC68F9F765FD4FF47A70A4EB070909FBEC
:100ED000000006F05DFC01463046FEF711FCCDE94E
:100EE0000049D8F800503B4632689DF80F1008487A
:100EF000A847204605B0BDE8F0832846F9F748FD2D
:100F00000024F6E70446F4E780D40108204F0020CF
:100F100025E40108B00000202DE9F84F394E98462D
:100F2000736B0546894614464FF47A7A9847DFF882
:100F3000DCB0354F0AFB05F202F59C328032B2FB81
:100F4000FAF23249D7F82801FBF7D8FF20B9336B02
:100F500098474FF0FF302FE09BF80030072B07D168
:100F60005846F9F715FD4FF47A65FAF76FF8E1E79F
:100F7000032B366B22D1DBF8045028792968844290
:100F800028BF04464846224607F04EF93F6895F9C7
:100F90000830B5F90620A9881D48B847B8F1000FF8
:100FA00005D0EB88A8F800302B7A88F80230174873
:100FB000F9F7EEFCB0472046BDE8F88F042B0BD1C3
:100FC0001248F9F7E5FCB0473C68FCF71BFF014607
:100FD0001048A0470020EFE7052B0AD10B48F9F78E
:100FE000D7FCB0473C68FCF70DFF01460A48A04714
:100FF000AFE7D3210948F5F759FD0448F9F7C8FCD4
:10100000B047A6E780D40108B00000202C4F002094
:1010100092E30108BCE30108D4E30108EAE3010814
:101020002DE9F04FC9B08946174608A9FF22029062
:101030001E46DDF84C8101F0F7FB824618B900200E
:1010400049B0BDE8F08F634CD9F8002094F8FC104B
:1010500094F8FE5008468D429ABF4D1BEDB2002514
:10106000D4F800B00592049101F030F8039094F8A0
:10107000FD0001F041F8DDE90412039B00905648A1
:10108000D847D9F800202846D4F800B0039201F0E0
:101090001DF8039A034629465048D84794F8FF1094
:1010A000D4F800210846D4F800B00492039101F06E
:1010B0000DF8DDE9031203464948D84794F8FD309E
:1010C00094F8FC20D9F80010002001F0DBF8002390
:1010D000524608A94846FFF7CDFE04460028AED088
:1010E000029B93F8783013F0050F0BD013F0040F28
:1010F0000CBF00220222374B93F83210914218BFE6
:1011000083F83220FF22002108A807F0B5F8D9F8AB
:1011100000104FF47A792A460823012001F0B2F832
:1011200009FB07F1A1F51C414039B1FBF9F106A813
:101130000694FCF77FFFFF22434608A94FF44D7049
:10114000FFF7EAFE421C05463FF479AF002821492B
:101150001ADD0E68FCF756FE234602462946214852
:10116000B047B8F1000F02D0012388F80330002304
:10117000529A9D42136005DDE9B208A801F0B2FE63
:10118000529B186001205BE791F8FF200823D1F8FB
:101190000011012001F076F809FB06F1A1F51C41D0
:1011A0004039B1FBF9F107A80794FCF743FF434628
:1011B000FF2208A94FF44D70FFF7AEFE431C054611
:1011C0003FF43DAF0028D2DDB8F1000FCFD00223AD
:1011D000CBE700BFB00000209CE40108CFE4010889
:1011E000F6E401081DE5010870B5C2B001ABFF22AD
:1011F00002A94FF47A60FFF78FFE061E1EDD114D27
:10120000F1B26A6D02A801F04DFC0446B0B103785A
:10121000052B01D0032B0DD10021204600F074F9DD
:10122000204600F035F92046019900F0A3FB2B6C15
:10123000204613B901F0DEFA00E09847304642B08C
:1012400070BD00BFB000002038B5074B0546DB6815
:1012500018209847044620B11422002107F00CF80A
:101260006561204638BD00BFB000002010B50446BF
:1012700050B1406901F0BEFA00236361034B204680
:10128000BDE810401B69184710BD00BFB00000202A
:10129000037807B5052B4FF00003019006481A4666
:1012A00001A90CBF806C406CFBF7CEFC431E58427A
:1012B000584103B05DF804FBB000002007B5037887
:1012C00001900948052B4FF000024FF0010301A9DE
:1012D0000CBF806C406CFBF7B7FC431E5842584172
:1012E00003B05DF804FB00BFB0000020002213B57E
:1012F000084C01A9A06C0192FBF700FE019B33B9D9
:1013000094F836201AB901A9606CFBF7F7FD019833
:1013100002B010BDB0000020064B10B5DB68A02065
:101320009847044618B1A022002106F0A5FF2046E8
:1013300010BD00BFB000002070B5044690B1D0F8D9
:101340008000094D08B12B699847D4F8980020B166
:1013500001F050FA0023C4F898302B692046BDE80C
:101360007040184770BD00BFB00000201FB50E4C84
:101370000190E06CFBF7F4FF024638B903A9E06C7A
:10138000FBF7BCFD10B10398FFF7D6FF002301A9BE
:101390001A46E06CFBF758FC20B94FF4B4710348CF
:1013A000F5F784FB04B010BDB0000020EAE30108AB
:1013B000F8B50423437003780546032B0ABF144B8A
:1013C0000469DC6BFFF7A8FF0646B0B940F277115D
:1013D0001048F5F76BFB104B104A4FF4BC710D48E9
:1013E00006F0F4FD31466868A0473046FFF7A4FFD9
:1013F000FA20FCF75FFE3846F8BD01272B7807700E
:101400004370002CEED1FFF7B1FF2046F4E700BF98
:10141000B0000020EAE301088AE3010858E401086B
:10142000F8B503780646032B08BF154B0F460CBFD3
:10143000DC6B0469FFF770FF0546B0B94FF4C87163
:101440001048F5F733FB104B104A40F291110D484C
:1014500006F0BCFD29467068A0472846FFF76CFFE0
:10146000FA20FCF727FE0120F8BD02230370337831
:1014700047604370002CEDD1FFF778FF2046F3E77B
:10148000B0000020EAE301088AE3010874E40108DF
:1014900008B5104A10B1002382F8093192F82230C1
:1014A000BBB192F8093192F80A118B4211D95B1A3B
:1014B00092F80B1193FBF1F201FB12334BB900F0E0
:1014C00083FC30B900F08EFC18B9BDE8084000F08C
:1014D00099BC08BDB00000200A4B93F822207AB1D5
:1014E000027A42F00102027293F8092193F80A315C
:1014F0009A4205D9037A43F002030372FEF7B6BE9F
:10150000704700BFB000002070470000064A137803
:10151000FD2BDFBF00780549C8540133DABF012035
:1015200013700020704700BF395000203A4F002050
:1015300038B10078032803D0431F58425841704700
:1015400001207047052307B50DF107008DF807301E
:10155000FFF7DCFF0248FFF7D9FF03B05DF804FB9B
:10156000384F0020037A70B51B09D61804460F2E99
:1015700000F10C001546184409DC06F055FE012068
:10158000237A05EB131565F30713237270BDC3F1BE
:101590000F0206F049FE237A002043F0F003237285
:1015A000F4E7000037B5114C0546227822B1104906
:1015B000FFF7D8FF002323700E4C94F807213AB1AF
:1015C0000823012201A928468DF80430FFF7CAFF3D
:1015D00094F8083143B140F20113022201A92846D0
:1015E000ADF80430FFF7BEFF03B030BD3950002026
:1015F0003A4F0020B00000200122044B00F00F0001
:1016000083F80E0183F80721704700BFB000002067
:101610002DE9F04F814693469A4600258BB09DF800
:101620005080B44E0291454502D30BB0BDE8F08F17
:101630001AF805300AEB0507013B1F2B00F29881D1
:10164000DFE813F0200096012B003B01C600AE003E
:10165000FF0036013B011D0196013D018B00550144
:1016600064019601960196019601960196019601F4
:1016700096019601960196019601960196019601B2
:1016800096018301A8EB0503DBB2012B4FF00004A8
:101690001BD086F80841022417E00024A8EB0503BC
:1016A000DBB201938DF81C40019A231D934202DAAC
:1016B0003B5D032B0BD044B1032308A88DF82030E9
:1016C000FFF724FF07A8FFF721FF2C447AE0391920
:1016D0004B78A01C1A09384403F00F0305910492BB
:1016E0000393F8F7A2FF0599049A09790534062AAD
:1016F000C1F3021CE4B201F00F01039B21D90F2AB0
:1017000005D19DF81C2042F002028DF81C205A1EC3
:10171000062A19D90F2B05D19DF81C3043F004037C
:101720008DF81C3009B186F80C11BCF1000F0ED1F8
:1017300000F034FC9DF81C3043F001038DF81C30A0
:10174000B2E786F8FC20DCE786F8FD30E4E7BCF180
:10175000060FA9D14FF6FF70EAE7A8EB0503DBB24D
:10176000052B40F20381781CF8F755FF002197F90B
:101770000530002BACBF604B604BC31841F1000239
:10178000002196F80E01C31841EB0202BBF1020FD3
:1017900002D1013342F10002C9E91C32062494E768
:1017A000062307A88DF81C30FFF7B0FE029B5448B3
:1017B00003F01F038DF82030FFF7A8FE08A8FFF7FD
:1017C000A5FE6C1CE4B2A5423FF42FAF25462AE7E4
:1017D000A8EB0503DBB2042B40F2C880D7F8012048
:1017E000484C0892D2B2C2F3021386F8FE30237836
:1017F000C2F30302052A43F0040394BF43F002033B
:101800006FF341030DF1210098BF86F8FF2023708C
:101810006427F8F702FF47433846F9F719FC60B12F
:101820002378C6F8007143F0010301222370364B80
:101830001A70FFF787FE052447E7237860F300035B
:10184000F3E7A8EB0503DBB2052B40F28F806421A0
:1018500057F8010F3A79030A59430890C0B28DF83E
:10186000242000F033FB07238DF8180007A88DF81B
:101870001C30FFF74BFE06A8FFF748FE8EE7A8EBEB
:101880000503DBB2042B71D96421D7F80100030AE8
:101890005943C0B200F04CFB0A238DF81C0008A885
:1018A0008DF82030FFF732FE07A8FFF72FFEC2E7C2
:1018B000787800F00F00FFF79FFEAC1C82E7A8EBE2
:1018C0000503DBB2012B51D001237A7808A8110956
:1018D00002F00F0203FA01F1934086F80B310C235A
:1018E00086F80A118DF82030FFF710FED3E6EC1CC5
:1018F00068E700BFB00000206E3DD5126F3DD512E5
:10190000BD010020384F0020394F0020A8EB05030F
:10191000DBB2012B2AD0B3687C78984701222309D7
:101920000A3302FA03F3C6F818310F23C6E944015B
:1019300004F00F0408A8C6F81C418DF81C208DF88F
:101940002030FFF7E3FD07A8CEE7A8EB0503DBB2E5
:10195000012B0BD07B780BB1022B07D196F83320EB
:101960009A423FF498AE86F8333094E60024ACE611
:101970002C4628E730B585B003910446174B30B9A3
:101980001B7803B305B0BDE83040FFF7DBBD002591
:101990009DF90E109DF80F201D70FFF7C9FD90B145
:1019A0000F48237A90F822502DB113F0010518BF8B
:1019B000012580F806511B0907D0009304F10C03A0
:1019C0002046FFF725FE05B030BD637F002BFAD11E
:1019D000237F002BF7D00093A36EF1E7394F00204F
:1019E000B000002010B5044678B1836A012B0CD1F9
:1019F000C36A1BB910210648F5F758F8E36A58780E
:101A000002288CBF0020012010BD0020FCE700BF91
:101A100051E501082DE9F047054686B018B1037875
:101A2000033B012B03D92221BC48F5F73FF86B6932
:101A30000BB11B781BB12321B848F5F737F84FF0ED
:101A40000009B74C94F8FD60D4E93F8700F0ACF989
:101A500000F0B2F9304603AAB249CDF80C90FDF778
:101A6000C3FD064620B92846FFF7A2FC01260AE07E
:101A7000039BA3B1FDF75EFD0399042907D928460E
:101A8000FFF7CEFC4E46304606B0BDE8F0874FF477
:101A90007A73A5484843B0FBF3F0FCF70BFBAB6847
:101AA00094F820200133102AAB602FD1012B09D1EB
:101AB000D4F8F0300133C4F8F0309C4B5B699847A0
:101AC000A4F8E800B4F8E8300133A4F8E8304FF0A7
:101AD000000905AB019304AB0093314641F27073EA
:101AE00041F28832686994F8FFA0CDF8109084F82C
:101AF000FF90FFF795FA0646A8B92846FFF758FC6D
:101B0000049800F077FE84F8FFA0AFE7112A05D112
:101B1000636987489847A4F8E800D8E750217F48D0
:101B2000F4F7C4FFD3E7049B84F8FFA013B11A783D
:101B3000012A06D02846FFF73BFC049800F05AFE25
:101B4000A1E794F82020102A40F09780102384F811
:101B500050300023049AD16802F1530C616502F100
:101B6000630E002B00F09980112384F850306346F7
:101B7000DFF8C0A1D146186859680833A9E8030006
:101B80007345CA46F6D1DFF8B09102F1230302F1A2
:101B9000330ACE46186859680833AEE80300534547
:101BA000F146F6D1DFF8949102F1430ACE46186867
:101BB00059680833AEE803005345F146F6D1DFF823
:101BC0008091CE46186859680833AEE80300634533
:101BD000F146F6D19368A363137CC3F3030384F83F
:101BE000FF30137CC3F3021384F8FE30507CFFF700
:101BF00003FD049894F83120437C1230012B4FF000
